:020000040800F2
:1000000000000220693A0108B1990008B39900087C
:10001000B5990008B7990008B999000800000000D8
:10002000000000000000000000000000BB99000874
:10003000BD99000800000000BF990008C1990008A0
:10004000AD3A0108AD3A0108AD3A0108AD3A0108F0
:10005000AD3A0108AD3A0108AD3A0108AD3A0108E0
:10006000AD3A0108AD3A0108AD3A0108697C0008D3
:10007000AD3A0108AD3A0108AD3A0108AD3A0108C0
:10008000AD3A0108AD3A0108AD3A0108AD3A0108B0
:10009000AD3A0108AD3A0108AD3A0108FD9B0008F0
:1000A000AD3A0108AD3A0108AD3A0108AD3A010890
:1000B000BD9B0008AD3A0108AD3A0108AD3A010810
:1000C000AD3A0108AD3A0108AD3A0108AD3A010870
:1000D000AD3A0108AD3A0108119D0008AD3A01089A
:1000E000AD3A0108AD3A0108C5990008AD3A0108DA
:1000F000AD3A0108AD3A0108AD3A0108AD3A010840
:10010000AD3A0108AD3A0108AD3A0108AD3A01082F
:10011000AD3A0108AD3A0108AD3A0108AD3A01081F
:10012000AD3A0108AD3A0108AD3A0108AD3A01080F
:10013000AD3A0108AD3A0108AD3A0108AD3A0108FF
:10014000AD3A0108AD3A0108AD3A0108F599000849
:10015000AD3A0108AD3A0108AD3A0108AD3A0108DF
:10016000AD3A0108AD3A0108AD3A0108AD3A0108CF
:10017000AD3A0108AD3A0108AD3A0108AD3A0108BF
:08018000AD3A0108AD3A010897
:100188004CBF050800000020300C0020300C002077
:10019800843D002008B5074B186809F08FFB0EF066
:1001A800EFFA054B054806221A70BDE8084001F031
:1001B800C6BD00BFE4260020712600204C10002098
:1001C80008B5034801F0BBFD024B00221A7008BDB8
:1001D800A01800207126002008B5054B0122002038
:1001E8001A7005F0FFFF0348BDE8084001F0A7BDFD
:1001F800FC2C0020101600202DE9F041144C20465C
:1002080004F073F900201349134A03F025FF13493A
:10021800134A0746002003F01FFF1249124A0646F8
:10022800002003F019FFD22105463A462346F6205E
:1002380004F02AF8D22132462346A62004F024F8F6
:100248005620D2212A462346BDE8F04104F01CB8C6
:10025800241400202EAB0508C901000837AB050897
:10026800E101000840AB05089D01000808B502F04F
:10027800B5FC034801F063FD024B00221A7008BD6B
:10028800A018002071260020034B0D224FF4864051
:100298001A700FF097BA00BF71260020034B0D2289
:1002A8004FF402401A700FF08DBA00BF712600207B
:1002B8000F4B0D2270B51A7000240BE0A8B2002273
:1002C8003146013505F0FEF8B5F5A07FF6D10134C9
:1002D800CE2C02D00025A6B2F0E70D2000F09EFC3F
:1002E8004FF441400FF0E2FABDE8704004F036BB2D
:1002F800FC2C00202DE9F347234D0024284604F068
:10030800F4F8234622464FF6FF71204800940194E2
:1003180003F0AAF91E491F4A8146204603F09CFEB5
:100328001D491E4A0746204603F096FE1C491D4AF1
:100338008046204603F090FE1B491C4A064620468C
:1003480003F08AFE214682464A462B46204603F0A1
:100358009BFF64213A462B460A2003F095FF8C2127
:1003680032462B460A2003F08FFFB42142462B4623
:100378000A2003F089FFF620D22152462B4602B00C
:10038800BDE8F04703F080BFA80F002049AB05087F
:1003980055AB0508A502000864AB0508B9020008BA
:1003A80073AB0508910200082EAB0508750200081A
:1003B80008B5054B012200201A7005F013FF034809
:1003C800BDE8084001F0BBBCFC2C00201016002042
:1003D80008B5034801F0B3FC024B00221A7008BDAF
:1003E800A01800207126002008B5054B07221A70B6
:1003F8000EF0C6F90348BDE8084001F0A0BC00BFF4
:1004080071260020241400202DE9F041144C2046C8
:1004180004F06BF800201349134A03F01DFE13493A
:10042800134A0746002003F017FE1249124A0646EF
:10043800002003F011FED22105463A462346F62055
:1004480003F022FFD22132462346562003F01CFF38
:10045800A620D2212A462346BDE8F04103F014BF66
:100468004C1000202EAB0508D903000882AB050804
:10047800F103000837AB0508B9030008014801F08B
:100488005EBC00BF3812002010B5094C204604F0AD
:100498002CF800200749084A03F0DEFDD221024665
:1004A80023464FF48270BDE8104003F0EDBE00BF54
:1004B800581700208BAB05088504000870B50C4C54
:1004C8000C4D20684FF6E076314603F009F92068B4
:1004D800294603F0B3F86068314603F001F9606813
:1004E800294603F0ABF8BDE8704004F037BA00BF06
:1004F800300C00208CB1050838B52B4CFFF7DEFF17
:10050800002005F06FFE237A23B90A203221274AFA
:1005180005F076FF637A23B90A206421244A05F09E
:100528006FFF214CA37A23B90A209621214A05F0AE
:1005380067FFA37A1C4DFBB16B7AEBB12B7ADBB169
:1005480000232B726B72AB721B4B286801221A7046
:100558004FF6E07103F0C4F82868184903F06EF804
:100568006868174903F06AF80BF0E5FC04F0F6F93F
:10057800144804F037FA0DE00B4C4FF4784120682A
:1005880003F0AEF82068104903F058F860680F4986
:1005980003F054F8FFF792FF00200BF08FFC0C4893
:1005A800BDE8384001F0CBBB300C002092AB050809
:1005B800A0AB0508AFAB050871260020BDAB050848
:1005C8008DB1050880969800D1AB05088FB1050854
:1005D800A018002008B500200BF070FC0248BDE808
:1005E800084001F0ACBB00BFA018002038B5FFF7E9
:1005F80065FF0EF0DDF83C213F220023DF2005F0E7
:10060800E1FE4FF480600EF017FE124C3E223C21B2
:10061800DF20002305F0D6FE012323720E4B4FF690
:10062800E075186809F04AF92068294603F058F877
:1006380020680A4903F002F86068294603F050F878
:100648006068074902F0FAFF04F088F9054B0022B8
:100658001A7038BD300C0020E4260020E3AB0508F2
:10066800F6AB05087126002038B5FFF727FF0EF016
:100678009FF86E213F220023DF2005F0A3FE4FF4F0
:1006880086400EF0D9FD124C3E226E21DF20002359
:1006980005F098FE012363720E4B4FF6E07518685B
:1006A80009F00CF92068294603F01AF820680A496D
:1006B80002F0C4FF6068294603F012F86068074931
:1006C80002F0BCFF04F04AF9054B00221A7038BD4D
:1006D800300C0020E426002009AC05081AAC0508F7
:1006E8007126002010B5FFF7E9FE0EF061F8A02191
:1006F8003F220023DF2005F065FE4FF402400EF094
:100708009BFD114C3E22A021DF20002305F05AFE5C
:100718000123A3720D4B186809F0D0F820684FF632
:10072800E07102F0DDFF2068094902F087FF606888
:10073800084902F083FF04F011F964200BF07EFAF7
:10074800054B00221A7010BD300C0020E426002052
:100758002BAC05088DB10508712600202DE9F74F4F
:100768003A4D3B4E0024284603F0BFFE224623465E
:100778004FF6FF7137480094019402F075FF4FF669
:10078800E0780427F0604146224623463248009725
:10079800019402F069FF23463060414622462F4803
:1007A8000097019402F060FF2D4970602D4A2046A1
:1007B80003F052FC2C492D4A0746204603F04CFC16
:1007C8002B492C4A8046204603F046FC2A492B4AEE
:1007D8008146204603F040FC29492A4A83462046A0
:1007E80003F03AFC21468246F2682B46204603F085
:1007F8004BFD5A2132682B460A2003F045FD6E2135
:1008080072682B460A2003F03FFD9B213A462B468F
:10081800FA2003F039FD692142462B46FA2003F0FD
:1008280033FD37214A462B46FA2003F02DFDC82117
:1008380052462B46AA2003F027FDF020C8215A462D
:100848002B4603B0BDE8F04F03F01EBDC8140020CE
:10085800300C00203FAC050847AC05085AAC050829
:1008680069AC0508ED06000871AC050871060008BA
:1008780061AC0508F505000879AC0508DD05000838
:1008880080AC05080105000838B50C4C4FF6E0753A
:100898002068294602F024FF2068094902F0CEFEAC
:1008A8006068294602F01CFF6068064902F0C6FE2F
:1008B80004F054F8BDE8384004F050B8300C00207B
:1008C80047AC050887AC050870B52DED028B9FED88
:1008D800248A88B00A26F0EE488A03E0B0EE608ADF
:1008E800F0EE418A0CF031FE8DED000ACDED010AE3
:1008F8009DE8030004AB83E80300F0EE680AB0EE5D
:10090800480A9DED041ADDED051A8DED028ACDED3C
:10091800038A0CF0BBFBCDED010A8DED000A9DE8C2
:10092800030002AD85E80300013E6C46DDED020AD6
:100938009DED031AD2D19FED0B0A0CF0FDFD8DED54
:10094800000ACDED010A9DE8030085E80300DDED0E
:10095800030A9DED020A08B0BDEC028B70BD00BF12
:1009680000000000CDCCCC3D2DE9F74F564D574C3B
:10097800DFF86491DFF864814FF6E07005F006FC5B
:10098800286811F075FF064668680F4611F070FF79
:100998003246CDE900013B464946204616F046FE60
:1009A800224600230520372105F02AFD2869484FF3
:1009B800484E11F05DFF824668698B4611F058FF7A
:1009C8005246CDE900015B463946204616F02EFE18
:1009D800224600230520692105F012FD286B11F03D
:1009E80047FF8246686B8B4611F042FF5246CDE9BD
:1009F80000015B464146204616F018FE00230520FC
:100A08009B21224605F0FCFC31462A6C204616F054
:100A18000DFE224600239B21A22005F0F1FC4FF495
:100A2800FC6005F0B3FBA86811F022FF8246E86875
:100A38008B4611F01DFF5246CDE900015B46494641
:100A4800204616F0F3FD224605205021002305F02C
:100A5800D7FCA86911F00CFF8246E8698B4611F0B3
:100A680007FF5246CDE900015B463946204616F09D
:100A7800DDFD224600230520822105F0C1FCA86B7C
:100A880011F0F6FE8246E86B8B4611F0F1FE5246F5
:100A9800CDE900015B464146204616F0C7FD00231C
:100AA8000520B421224605F0ABFC31466A6C20468D
:100AB80016F0BCFDA220B4212246002303B0BDE8F5
:100AC800F04F05F09DBC00BF103B0020400C0020FB
:100AD800ACAC0508CFAC05089AAC0508BEAC050857
:100AE80008B5002005F07EFB0A4B1B780B2B0BD8B2
:100AF800DFE803F00A0A0A0A0A0A08060A0A0A0AC2
:100B0800054802E0054800E00548BDE8084001F056
:100B180016B900BF71260020241400204C100020B4
:100B2800A01800202DE9F14F2D4C204603F0DDFCE4
:100B380000202C492C4A03F08FFA2C492C4A814674
:100B4800002003F089FA2B492B4A0746002003F0BE
:100B580083FA2A492A4A0646002003F07DFA2949E1
:100B6800294A0546002003F077FA2849284A804692
:100B7800002003F071FA2749274A8246002003F033
:100B88006BFAD22183464A462346E62003F07CFBD3
:100B980028203A462346014603F076FB4621324692
:100BA8002346282003F070FB64212A462346282088
:100BB80003F06AFB822142462346282003F064FBA7
:100BC800524623462820A02103F05EFB28205A46DF
:100BD800BE21234601B0BDE8F04F03F055BB00BF6E
:100BE800101600202EAB0508E90A0008D4AC050849
:100BF80019160008DFAC0508F5150008E9AC05086A
:100C0800D1150008F4AC0508AD150008FFAC0508BF
:100C18008915000809AD050865150008023810B5E2
:100C28000B2800F26E84DFE810F04F005300140127
:100C3800AF016702FD01120363036C04D3032704A9
:100C48000C0000204FF6E0710BF038FB19204FF430
:100C5800FC610BF033FB4B204FF6E0710BF02EFBE1
:100C68007D204FF6E0710BF029FBAF204FF6E071C5
:100C78000BF024FB4FF6FF7005F088FAC82100231B
:100C88005020A94A05F0BCFB4EF29C7005F07EFA94
:100C9800052001210023A54A05F0B2FB05201A21F1
:100CA8000023A34A05F0ACFB05204C210023A14AF0
:100CB80005F0A6FB05207E219F4A002305F0A0FB36
:100CC80005209E4AB02160E0BDE810400BF0A0B9B5
:100CD80000204FF6E0710BF0F1FA64204FF6E07156
:100CE8000BF0ECFAC8204FF6E0710BF0E7FA4FF67C
:100CF800FF7005F04BFA00237D20DC21904A05F0B7
:100D08007FFB4EF29C7005F041FA8E4B1C78022C4A
:100D180040D0052C6CD0012C40F0F383B4204FF464
:100D2800F0610BF0CBFA05202146874A002305F035
:100D380067FB05205221854A002305F061FBB62197
:100D48007B4A0023052005F05BFB4FF4F06005F0BB
:100D58001DFA40F2131021467B4A002305F050FB90
:100D680040F213105221724A002305F049FB784AD9
:100D780040F21310B621002305F042FB4EF29C709E
:100D880005F004FA0520A221724A0023BDE81040AC
:100D980005F036BBA0204FF4F0610BF08FFA052068
:100DA80001216A4A002305F02BFB052052216A4ADB
:100DB800002305F025FBB6215D4A0023052005F038
:100DC8001FFB4FF4F06005F0E1F940F21310012128
:100DD8005E4A002305F014FB40F213105221544AD6
:100DE800002305F00DFB40F21310B6215B4AC2E761
:100DF80064204FF4F0610BF061FA20460121584A53
:100E0800002305F0FDFAB621494A0023204605F0E3
:100E1800F7FA4FF4F06005F0B9F940F21310012128
:100E28004F4A002305F0ECFA40F213105221404AD1
:100E3800002305F0E5FAB62140F21310494A0023D1
:100E480005F0DEFA4EF29C7005F0A0F9204652211A
:100E58009AE700204FF6E0710BF030FA31204FF698
:100E6800E0710BF02BFA63204FF6E0710BF026FAD5
:100E780095204FF6E0710BF021FAC7204FF6E0718C
:100E88000BF01CFA4EF29C7005F080F90520012148
:100E98000023354A05F0B4FA052020210023334AFF
:100EA80005F0AEFA052052210023314A05F0A8FAD0
:100EB8000520842100232F4A05F0A2FAB621052037
:100EC8001B4A002305F09CFA4FF4F06005F05EF928
:100ED800012140F213100023234A05F091FA40F251
:100EE80013102021244A002305F08AFA40F2131037
:100EF80052210F4A002305F083FA40F2131084218F
:100F08001E4A002305F07CFAB6211D4A40F2131050
:100F1800002305F075FA4FF6FF7005F037F97D20CC
:100F2800DC21184A31E700BF0EAD050823AD0508DE
:100F380005B3050827AD05082BAD05082FAD050835
:100F4800DFAC05081C03002034AD05083DAD0508DD
:100F580033AD050867AD050838AD05083CAD050893
:100F680042AD050841AD05085BAD050846AD05086D
:100F780056AD05084BAD050850AD050855AD05083B
:100F88005AAD0508E9AC050800204FF6E0710BF0F2
:100F980095F927204FF6E0710BF090F94F204FF6A6
:100FA800E0710BF08BF977204FF6E0710BF086F9C2
:100FB8009F204FF6E0710BF081F9C7204FF6E071E2
:100FC8000BF07CF94EF29C7005F0E0F80520012149
:100FD8000023AC4A05F014FA052016210023AA4A7A
:100FE80005F00EFA05203E210023A84A05F008FA6C
:100FF800052066210023A64A05F002FA8E21002367
:101008000520A44A05F0FCF90520A34AB6210023CF
:1010180005F0F6F94FF6FF7005F0B8F87D20DC21F1
:101028009E4AB2E600204FF6E0710BF047F93120F6
:101038004FF6E0710BF042F963204FF6E0710BF0C8
:101048003DF995204FF6E0710BF038F9C7204FF6BF
:10105800E0710BF033F94EF29C7005F097F805201B
:10106800012100238E4A05F0CBF905202021002319
:101078008C4A05F0C5F90520522100238A4A05F05B
:10108800BFF9052084210023884A05F0B9F9B62163
:1010980005207C4A002305F0B3F94FF4F06005F011
:1010A80075F8012140F213100023814A05F0A8F9D0
:1010B80040F2131020217F4A002305F0A1F940F2E5
:1010C800131052216F4A002305F09AF940F21310C9
:1010D8008421794A002305F093F9B621774A40F232
:1010E8001310002305F08CF94FF6FF7005F04EF849
:1010F8007D20DC21724A48E6724B1C78022C32D0E3
:10110800052C5DD0012C40F08B8000204FF6E0715B
:101118000BF0D4F834204FF6E0710BF0CFF86420D0
:101128004FF6E0710BF0CAF84FF6E07198200BF01B
:10113800C5F84EF29C7005F029F805202146624A50
:10114800002305F05DF905202021604A002305F001
:1011580057F9052050215E4A002305F051F9052072
:1011680084215C4A59E000204FF6E0710BF0A6F8A4
:1011780052204FF6E0710BF0A1F890204FF6E07185
:101188000BF09CF84FF6E071B4200BF097F84EF294
:101198009C7004F0FBFF052001214F4A002305F055
:1011A8002FF905203E214A4A002305F029F9052098
:1011B8007C21484A002305F023F90520A0212BE0D3
:1011C80000204FF6E0710BF079F82E204FF6E07111
:1011D8000BF074F87F204FF6E0710BF06FF84FF6C4
:1011E800E071AD200BF06AF84EF29C7004F0CEFF6F
:1011F80020460121394A002305F002F92046322110
:10120800334A002305F0FCF820466B21314A0023BD
:1012180005F0F6F820469921314A002305F0F0F848
:101228004FF4F06004F0B2FF2E4A00230520B621E7
:1012380005F0E6F84FF4FC61C8200BF03FF84FF6D4
:10124800FF7004F0A3FF8720DC21274A9DE50020DA
:101258004FF6E0710BF032F863204FF4FC610BF0AD
:101268002DF84FF6E071C7200BF028F84FF6FF7005
:1012780004F08CFF002005F08BF8A520D7211B4A2D
:1012880083E500BF05B305085EAD050827AD050871
:1012980062AD05082BAD050866AD05086AAD050801
:1012A80076AD05087AAD050897AD05087EAD050849
:1012B80087AD050883AD050882AD050886AD05082C
:1012C8008BAD05081C03002042AD050863AD050879
:1012D80024AD0508A6AD050867AD050828AD0508C5
:1012E80096AD05081CB4050809AD0508A5B10508A3
:1012F800042005F04DF800204FF6E0710AF0DEFFFB
:1013080031204FF6E0710AF0D9FF63204FF6E07103
:101318000AF0D4FF95204FF6E0710AF0CFFFC720FE
:101328004FF6E0710AF0CAFF4EF29C7004F02EFFEF
:10133800052001210023734A05F062F805202021C9
:101348000023714A05F05CF80520522100236F4AFA
:1013580005F056F80520842100236D4A05F050F861
:101368000520B6216B4A002305F04AF84FF6E070D5
:1013780004F00CFF40F20B100121674A002305F02E
:101388003FF840F22B102021644A002305F038F87A
:1013980040F223105221624A002305F031F840F24E
:1013A8001B1084215F4A002305F02AF8B6215E4A03
:1013B800002340F2131005F023F84FF6FF7004F0F5
:1013C800E5FE002004F0E4FF6E20D221574A90E0A9
:1013D800042004F0DDFF00204FF6E0710AF06EFFF4
:1013E80027204FF6E0710AF069FF4F204FF6E071B1
:1013F8000AF064FF77204FF6E0710AF05FFF9F2044
:101408004FF6E0710AF05AFFC7204FF6E0710AF074
:1014180055FF4EF29C7004F0B9FE0520012100230F
:10142800434A04F0EDFF052016210023414A04F049
:10143800E7FF05203E2100233F4A04F0E1FF052095
:1014480066213E4A002304F0DBFF05208E213C4A3A
:10145800002304F0D5FFB6213A4A0023052004F002
:10146800CFFF4FF6FF7004F091FE002004F090FFCC
:101478006420D221344A3CE0042004F089FF002093
:101488004FF6E0710AF01AFF43204FF6E0710AF0B8
:1014980015FF85204FF6E0710AF010FF4FF6E07156
:1014A800C7200AF00BFF4EF29C7004F06FFE052077
:1014B8000121264A002304F0A3FF05204521244AE0
:1014C800002304F09DFF052087211E4A002304F015
:1014D80097FFB6211F4A0023052004F091FF4FF61D
:1014E800FF7004F053FE002004F052FF1A4A7D20DA
:1014F800D221002304F084FF0420BDE8104004F04A
:1015080047BF10BD9AAD0508A6AD0508A5AD0508ED
:10151800A8AD0508ACAD0508B1AD05085BAD05087B
:10152800B8AD0508BCAD0508C1AD0508C7AD0508CF
:10153800CDAD050883AD050888AD0508D2AD050811
:1015480030AD050867AD0508D5AD0508DEAD050861
:1015580042AD050805B3050879B2050810B5064C73
:1015680006480623237000F0EAFB2078FFF756FBB5
:10157800BDE810400DF034BEFC2C0020FC17002004
:1015880010B5064C06480723237000F0D8FB2078D6
:10159800FFF744FBBDE810400DF022BEFC2C0020F4
:1015A800FC17002010B5064C06480523237000F0F0
:1015B800C6FB2078FFF732FBBDE810400DF010BEE7
:1015C800FC2C0020FC17002010B5064C064804230C
:1015D800237000F0B4FB2078FFF720FBBDE8104033
:1015E8000DF0FEBDFC2C0020FC17002010B5064CA9
:1015F80006480323237000F0A2FB2078FFF70EFBB8
:10160800BDE810400DF0ECBDFC2C0020FC170020BC
:1016180010B5064C06480223237000F090FB207892
:10162800FFF7FCFABDE810400DF0DABDFC2C0020F5
:10163800FC17002038B5094C05464FF6E0712068C4
:1016480002F04EF820680DB1054900E0054901F0A7
:10165800F5FFBDE8384003F081B900BF5C0C0020FD
:10166800E2AD0508F5AD0508194B10B51C78012C3D
:1016780005D006D3022C0CBF3024002402E000243D
:1016880000E0102404F1C80006F040FB11490246AE
:10169800114815F0CBFF04F1CC0006F037FB0D49DB
:1016A80002460E4815F0C2FF04F1D00006F02EFBEA
:1016B800084902460A4815F0B9FF04F1D40006F0BB
:1016C80025FB044902460748BDE8104015F0AEBFA7
:1016D8001C0E0020CFAC0508B4260020D826002018
:1016E800EE2C0020A026002010B5E82006F00EFB06
:1016F8000F4C024621460F4815F098FFEC2006F0E3
:1017080005FB214602460C4815F090FFF02006F034
:10171800FDFA21460246094815F088FFF42006F034
:10172800F5FA024606482146BDE8104015F07EBF8E
:10173800CFAC0508B4260020D8260020EE2C0020C7
:10174800A02600200E4A012310B513700D4A00246C
:1017580014700D4A204613700AF0B0FB204604F0BE
:1017680041FD0A4B03221A700AF006FF0BF087FCB2
:10177800074B08481C70BDE8104000F0E0BA00BFF5
:10178800FC2C0020770D0020750D0020712600200C
:10179800E4380020DC12002038B50D4B0D4D002434
:1017A8001C700D4B28681C700C4B4FF6E0711C70B8
:1017B80001F096FF28680A4901F040FF03F0CEF8CF
:1017C800204604F00FFD0748BDE8384000F0B7BADE
:1017D800D40D00205C0C0020770D0020712600201D
:1017E80091B10508A018002007B50E4B0E481A78CD
:1017F800D2F1010238BF00221A700C4B05221A7070
:1018080000F09DFA022201238DE80C00B02060212F
:10181800102232230DF082FE03B05DF804EB03F0D2
:101828009DB800BFD40D002094110020712600201F
:101838002E4A002310B513702D4A13700DF0C8FA04
:101848000446002842D02B4C4FF6E071206801F086
:1018580047FF2068284901F0F1FE60684FF6E07103
:1018680001F03EFF6068254901F0E8FEA0684FF6E8
:10187800E07101F035FFA068214901F0DFFE03F0B7
:101888006DF84FF47A600AF0D9F920684FF6E071E4
:1018980001F026FF20681B4901F0D0FE60684FF672
:1018A800E07101F01DFF6068164901F0C7FEA068ED
:1018B8004FF6E07101F014FFA068124901F0BEFE76
:1018C80003F04CF8BDE8104003F048B80CF058FF9E
:1018D800204604F087FC0C4B0C4804221A7000F0D8
:1018E8002EFABDE81040FEF7CFBF00BFD40D002090
:1018F800770D00205C0C002008AE05081CAE05081A
:101908002CAE050890B1050871260020C8140020E7
:101918002DE9F04F6A4DDFF8F4916A4E85B0002446
:101928004FF6FF78284602F0E0FD4146224623465E
:1019380065480094019401F097FE042703904146FE
:101948002246234648460097019401F08DFE414601
:1019580030602246234648460097019401F084FEF1
:10196800414670602246234648460097019401F09C
:101978007BFEA8F50048B0604146224623465348FE
:101988000097019401F070FE4146F060224623461C
:101998004F480097019401F067FE414630612246A6
:1019A80023464C480097019401F05EFE234670617F
:1019B8004146224648480097019401F055FE4749A0
:1019C800B061474A204602F047FB4649464A8046EE
:1019D800204602F041FB4549454A8246204602F02E
:1019E8003BFB4449444A0746204602F035FB43493D
:1019F800434A8146204602F02FFB4249424A834629
:101A0800204602F029FB21468446039ACDF808C0F7
:101A18002B46204602F038FC052132682B46A020D0
:101A280002F032FC692172682B46782002F02CFC07
:101A38007D21B2682B46782002F026FC2821F26826
:101A48002B46052002F020FC4B2132692B4605204D
:101A580002F01AFC052072696E212B4602F014FC74
:101A68009121B2692B46052002F00EFCD2213A469C
:101A78002B46052002F008FCD22142462B46562070
:101A880002F002FCD2214A462B46A62002F0FCFBBB
:101A9800D22152462B46F62002F0F6FBB4215A46D4
:101AA8002B46052002F0F0FBDDF808C05620B421D3
:101AB80062462B4605B0BDE8F04F02F0E5BB00BF1B
:101AC8006C1500205C0C00203CAE050846AE0508ED
:101AD8004DAE050853AE050859AE05085FAE0508BA
:101AE800391800082EAB0508A117000868AE0508CC
:101AF800F117000871AE05084D1700087AAE050801
:101B0800F116000883AE0508711600088DB10508A6
:101B1800664A00232DE9F04713700125644ADFF86F
:101B2800C0811370A842014688F8005003D00228EB
:101B380040F0B68041E04FF4747006F0CEF80AF039
:101B480041FC5C4B5C4A1B68934209DD5B4A5C497B
:101B580012688A4207DD5B498A4204DC022210E0EF
:101B6800B3F5FA5F1DDB554A574912688A4201DC12
:101B7800002206E055498B4213DD554B9A4210DC92
:101B88000122544B01201A7005F07EFA022005F05C
:101B98007BFA0120FFF74EFD4E4B1978012901D140
:101BA80007E0FEE702D302297AD102E040200021B3
:101BB80000E0402007F090FA72E0C82006F0A6F88E
:101BC8000446CC2006F0A2F80746D02006F09EF87E
:101BD8000646D42006F09AF881460AF0F3FB354B06
:101BE80036491A68A242184602DB0B68BB4213DD6D
:101BF800394B04601E60394B0F60C3F800900AF03F
:101C08001DF9374B01221A70364A0520B4210023EA
:101C1800BDE8F04704F0F4BB944218D19F4216D1B6
:101C28002D4B1B689E4212D12C4B1B6899450ED137
:101C38004FF47470294688F8005006F04EF82A4B85
:101C480000221A60294B4FF07E521A6028E0244B7C
:101C580002251D7029464FF4747006F03EF8154BA6
:101C68001B6806EE906A1C1BF8EEE67A06EE904AB0
:101C7800B8EEE67A1C4B87EE277A284683ED007A81
:101C8800154B1B6806EE903AB8EEE67A174BC7EE8E
:101C9800277AC3ED007A05F0F7F90020FFF7CAFCB0
:101CA8000AF02BFBBDE8F04702F058BED40D002027
:101CB800770D0020F02600205FE31600082D002095
:101CC8007FD1F0088074D21A50DA11001FA10700E2
:101CD80080D1F0081C0E0020E42C00209C26002057
:101CE800C90100208CAE05086C260020AC26002017
:101CF80008B500F055FFFEF77FFA00F051F800F044
:101D080071F8FEF72BFDFEF77FFBFEF70BFF01F0E6
:101D180077FBFFF7FDFDFEF7EDFA01F037F9FEF767
:101D2800B3FB01F069FA00F073FB00F087FD00F0E7
:101D380091FE00F065FABDE8084000F033BB10B52D
:101D4800044628B90F48104A104B552103F02EF8C5
:101D58000F4B1868844213D010B1C369002198470B
:101D6800002004F03FFA002004F026FA4FF6FF7036
:101D780004F00CFAE369204601219847044B1C60E3
:101D880010BD00BFA0AE05081C2C0408BCAE050899
:101D9800780C00200048D2E7A01800200CF0D8BF2B
:101DA80010B5084C204602F0A0FB00200649074A5F
:101DB80002F052F9D22102462346FA20BDE810402B
:101DC80002F062BA600E0020DAAE0508A51D000810
:101DD800024B034801221A70FFF7B1BF7126002099
:101DE8006C1500202DE9F743374D384F384E002445
:101DF800284602F07AFB2246234647F6FF7135480B
:101E08000094019401F030FC4FF6FF78814641467A
:101E18002246234638460094019401F025FC4146A9
:101E280030602246234638460094019401F01CFC99
:101E3800414670602246234638460094019401F0DA
:101E480013FC2346B060414622463846009401946C
:101E580001F00AFC2049F060204A204602F0FCF814
:101E68001F49204A0746204602F0F6F821468046D8
:101E78004A462B46204602F007FA3C2132682B4698
:101E8800192002F001FA5A2172682B46192002F033
:101E9800FBF97821B2682B46192002F0F5F9962152
:101EA800F2682B46192002F0EFF9D2213A462B4668
:101EB800EC2002F0E9F99C20D22142462B4603B0DF
:101EC800BDE8F04302F0E0B9DC1200208DB105084E
:101ED8007C0C0020CCAE0508D9AE0508D91D000839
:101EE800E2AE0508B520000870B5474E474C327879
:101EF80047492DED028B142592B005FB02420C32A6
:101F08000FA815F093FB33780E2B05FB03F504EBB4
:101F1800050332D8D3ED016A9B6807EE103A63597E
:101F2800B8EEE68A06EE903ADFED3A7AF8EEC78A1E
:101F3800B8EEE67A88EE278AC8EEA78AC7EE277A2F
:101F480017EE900A10F094FC02460B466846324998
:101F580015F06CFB18EE100A10F08AFC02460B46CE
:101F680005A82E4915F062FB18EE900A10F080FCC7
:101F780002460B460AA82A4929E093ED017A9B6894
:101F880007EE903A635906EE903AF8EEE78AF8EED3
:101F9800E67AB8EEC78A17EE900A10F069FC024696
:101FA8000B4668461F4915F041FB18EE100A10F061
:101FB8005FFC02460B4605A81B4915F037FB18EED7
:101FC800900A10F055FC0B46184902460AA8184C0E
:101FD80015F02CFB2068174901F030FB20680FA989
:101FE80001F02CFB6068694601F028FBA06805A990
:101FF80001F024FBE0680AA901F020FB02F0AEFC26
:1020080012B0BDEC028B70BDEA2600200000002053
:10201800EBAE050800007A44F6AE050807AF0508E0
:1020280018AF050829AF05083AAF05084BAF0508F2
:102038007C0C002096B1050808B5144B144A1B788F
:102048000D2B01D8012104E00E2B01D1022100E063
:1020580000211170142253430E49C858CA184FF46E
:102068007A730D4958430860516892684B430B498D
:102078000B600B4B1A6009F0E1FE0A4B0A4801227B
:102088001A70BDE80840FFF75ABE00BFEA260020D4
:102098001C0E002000000020F0260020082D002043
:1020A800E42C0020712600206C150020C4E700BF36
:1020B8004FF6FF7070474FF6FF7070471FB5002945
:1020C80047D04FF2DE7004F08DF8002004F060F97C
:1020D8000F2004F05BF81F4C1F4A412101230A20FE
:1020E80004F08EF9042004F053F92368282096217F
:1020F800042B24DC0123194A04F082F903A90DF109
:102108000E02206804F004FC0F2004F03FF8BDF82C
:102118000C00BDF80E1014380F242822002380B2BA
:10212800009404F063F8BDF80E10BDF80C0000949C
:10213800143989B22822012304F058F809E0084A22
:10214800012304F05DF91E20A521064A012304F0AD
:1021580057F91FBD8C0C00205CAF05086FAF050850
:102168008BAF0508A1AF050837B51E4C2368042BB3
:1021780005462BDC01A80DF1060104F0C7FBBDF8EC
:102188000630BDF80420184904200DF025FC23680A
:10219800002B04DA1548164A164B592105E0042B82
:1021A80005DD1248124A144B5A2102F0FFFD04EBD8
:1021B8008302BDF8041001339180BDF80610236036
:1021C800052BD18008D1201D04F022FC00230B48E8
:1021D8002360FFF7B4FD03E028460121FFF76EFFF7
:1021E8003EBD00BF8C0C0020B8AF0508FDAF050848
:1021F8002E2C04081FB0050836B00508B4160020B8
:1022080037B50B4C204602F070F90A4B0A49009387
:1022180000250120094A0A4B019502F00EF82946CB
:1022280002462346284603B0BDE8304002F02CB8E9
:1022380080130020C5200008B9200008BF2000082E
:10224800712100084FF6FF7070474FF6FF70704716
:1022580030B54FF6E07087B003F0C4FF002004F0FB
:1022680097F80F2003F092FF00212C4A2C4C0123F1
:102278000A2004F0C5F8002003F088FF042004F0C9
:1022880087F80A201921274A012304F0B9F82521E3
:10229800254A01230A2004F0B3F81F2003F076FF33
:1022A80001230A203721214A04F0AAF82378002BB9
:1022B80031D001231E2096211D4A04F0A1F862881E
:1022C8001C4902A815F0B2F901231E20A22102AA76
:1022D80004F096F8A288184902A815F0A7F9AE21CB
:1022E80002AA01231E2004F08BF80F2003F04EFFF2
:1022F8006088A188143880B20F2528220023009511
:1023080003F074FFA18860880095143989B22822E7
:10231800012303F06BFF07B030BD00BF64B00508B0
:10232800A40C002076B0050896B00508B6B00508DC
:10233800D9B00508EBB00508F8B0050801B187E782
:10234800704713B50DF1060101A804F093FA144B78
:1023580001221A705988BDF80420891A0E311C29E7
:1023680019460AD89C88BDF80600201A0E301C2889
:1023780003D899680131996001E000238B60084B0C
:102388009968012905DD00229A601A70FFF702FD9D
:1023980005E05A80BDF806209A80FFF759FF1CBD5A
:1023A800A40C002037B50B4C204602F09EF80A4BCF
:1023B8000A49009300250120094A0A4B019501F0BA
:1023C8003CFF294602462346284603B0BDE8304074
:1023D80001F05ABFB4160020452300084D2200081A
:1023E800532200084B23000808B5064B00221A7038
:1023F800054B186814F0B0FD0448BDE80840FFF725
:102408009EBC00BF71260020D0360020A0180020F6
:102418002DE9F04F514D524E85B00024284602F068
:1024280064F82246234647F6FF714E48009401940B
:1024380001F01AF94FF6FF770390394622462346F2
:1024480049480094019401F00FF93946306022465A
:10245800234646480094019401F006F94FF001081C
:102468007060224623464FF6E0714148CDF800805F
:10247800019401F0F9F82346B060394622463D48F8
:10248800CDF80080019401F0EFF83B49F0603B4A39
:10249800204601F0E1FD3A493A4A0746204601F054
:1024A800DBFD3949394A8046204601F0D5FD3849D7
:1024B800384A8146204601F0CFFD3749374A8246DF
:1024C800204601F0C9FD3649364A8346204601F0C8
:1024D800C3FD21468446039ACDF808C02B46204602
:1024E80001F0D2FE3C2132682B46142001F0CCFECC
:1024F8003C2172682B46EC2001F0C6FEB421B2687C
:102508002B460F2001F0C0FED2213A462B46E6208A
:1025180001F0BAFE642142462B46052001F0B4FEC4
:102528004A462B460520872101F0AEFE52462B462F
:102538000520D22101F0A8FED2215A462B46502070
:1025480001F0A2FEDDF808C09B20D22162462B468E
:1025580005B0BDE8F04F01F097BE00BF040F0020A2
:10256800B00C002005B105080FB1050889AE0508B3
:102578008BB105088DB10508D9AE0508F12300080F
:1025880061AC0508D925000871AC0508D9260008F2
:1025980018B10508E127000820B105089D270008A3
:1025A80028B105085927000808B50CF001F94FF4BF
:1025B80041400CF041FE044B186807F07FF9034BCB
:1025C80009221A7008BD00BFE426002071260020E9
:1025D80010B50C4CFFF7E8FF0B4A0023B420052187
:1025E80003F00EFFA0684FF6E07101F079F8A068DB
:1025F800064901F023F80CF0DBF8BDE8104002F0C2
:10260800ADB900BFB00C002093B1050830B1050882
:10261800264B2DE9F7431888C00014F095FC0546B1
:1026280028B90520B421224A2B4603F0E9FE214BA4
:10263800DFF878801D6000240CF0BAF826461E4F9B
:10264800DFF8889023E009F02BFA3B68D9F80000FE
:1026580045F8083C7B6845F8043C184B1B68C018D3
:1026680007F02CF9164B186809F0E8FAB8F80000DA
:1026780094FBF0F080B24FF4FC63009328210246EB
:10268800322303F00FFD04F59E7401360334B8F8C5
:1026980000300835B342D6DA0A4B186807F00EF94D
:1026A800094B09221A70BDE8FE8300BFDC3A0020FE
:1026B80049B10508D03600209C3800206826002043
:1026C8009C260020E426002071260020D836002011
:1026D80010B5094CFFF79CFFA0684FF6E07100F0B9
:1026E800FFFFA068054900F0A9FF0CF061F8BDE8FC
:1026F800104002F033B900BFB00C002057B10508F4
:1027080010B5074C4FF6E071A06800F0E9FFA0682B
:10271800044900F093FFBDE8104002F01FB900BF64
:10272800B00C002071B1050810B5074C4FF6E071E8
:10273800A06800F0D5FFA068044900F07FFFBDE85D
:10274800104002F00BB900BFB00C002087B105089B
:1027580010B50C4C0B2323700B4B01221A70002070
:1027680003F00EF80948FFF7EAFA2078FEF756FA60
:10277800074B032093ED000A0CF029F8BDE8104040
:10278800D2E700BFFC2C00207A0D0020FC170020A7
:102798002403002038B50C4D0C232B700B4B01245F
:1027A8001C70002002F0ECFF0948FFF7C8FA2878EF
:1027B800FEF734FA074B204693ED000A0CF007F8B1
:1027C800BDE83840B0E700BFFC2C00207A0D00209F
:1027D800FC1700202403002010B50C4C092323709B
:1027E8000B4B01221A70002002F0CAFF0948FFF7BC
:1027F800A6FA2078FEF712FA074B022093ED000A9A
:102808000BF0E5FFBDE810408EE700BFFC2C002070
:102818007A0D0020FC170020240300200CF05EBB7A
:10282800034A044800231370034A1370FFF787BA5A
:10283800E4380020A0180020712600202DE9F74375
:10284800384D394EDFF8FC800024284601F04DFE53
:102858002246234647F6FF7134480094019400F05D
:1028680003FF4FF6FF778146394622462346304814
:102878000094019400F0F8FE394630602246234661
:1028880040460094019400F0EFFE394670602246FD
:10289800234640460094019400F0E6FE2346B060CB
:1028A8003946224640460094019400F0DDFE214955
:1028B800F060214A204601F0CFFB2049204A074614
:1028C800204601F0C9FB214680464A462B46204651
:1028D80001F0DAFC3C2132682B46282001F0D4FCB8
:1028E8005A2172682B46192001F0CEFC7821B26873
:1028F8002B46192001F0C8FC9621F2682B461920B6
:1029080001F0C2FCD2213A462B46EC2001F0BCFC77
:102918000520D22142462B4603B0BDE8F04301F022
:10292800B3BC00BFF0100020C00C0020A1B1050806
:10293800A9B10508D9AE050829280008B4B10508C9
:10294800252800088DB1050870B5064600200D46FB
:10295800144603F01DFD4FF6FF7003F017FCF2B2AA
:1029680073208621002303F02DFDEAB27320AE21E7
:10297800002303F027FDE2B27320D6210023BDE82F
:10298800704003F01FBD08B5084B20201860084BA5
:102998001860084B58221A600146FFF7D5FF064811
:1029A800064B1860BDE8084006F088BFD801002033
:1029B800D4010020D0010020C0E1E40090260020CE
:1029C80008B5094B20201860084B58211960084B9E
:1029D80002461860FFF7B8FF0648074B1860BDE8C5
:1029E800084006F06BBF00BFD8010020D4010020CA
:1029F800D0010020809698009026002008B5094B49
:102A080058201860084B20211960084B0A461960A5
:102A1800FFF79AFF0648074B1860BDE8084006F024
:102A28004DBF00BFD8010020D4010020D0010020F4
:102A3800404B4C0090260020034A044800231370A2
:102A4800034A1370FFF77BB9E4380020A018002070
:102A5800712600202DE9F74F444D454EDFF83C81A3
:102A68000024284601F041FD2246234647F6FF711F
:102A780040480094019400F0F7FD4FF6FF77834635
:102A88003946224623463C480094019400F0ECFD68
:102A9800394630602246234640460094019400F0AF
:102AA800E3FD39467060224623464046009401946F
:102AB80000F0DAFD2346B0603946224640460094CD
:102AC800019400F0D1FD2D49F0602D4A204601F017
:102AD800C3FA2C492C4A0746204601F0BDFA2B4977
:102AE8002B4A8046204601F0B7FA2A492A4A8146ED
:102AF800204601F0B1FA214682465A462B46204626
:102B080001F0C2FB3C2132682B46192001F0BCFBC6
:102B18005A2172682B46192001F0B6FB7821B26859
:102B28002B46192001F0B0FB9621F2682B4619209C
:102B380001F0AAFBD2213A462B46EC2001F0A4FB77
:102B4800822142462B46192001F09EFBAA214A46C3
:102B58002B46192001F098FB19205246D2212B460A
:102B680003B0BDE8F04F01F08FBB00BF441900204F
:102B7800D00C0020BCB10508CAB10508D9AE0508BB
:102B8800412A0008D7B10508052A0008E0B1050860
:102B9800C9290008E9B105088F2900088DB1050881
:102BA80010B50B4C204601F0A0FC0020014622463F
:102BB80000F0BAFD00200749074A01F04DFAD2217A
:102BC800024623464FF48270BDE8104001F05CBB1A
:102BD800FC170020F2B10508092C000870B5C924BB
:102BE8000AE0A8B200223146013502F06BFCF02D54
:102BF800F7D10134EF2C02D00025A6B2F1E770BD61
:102C080010B51A4C2378092B08D1194A00231370E0
:102C1800184A1370FFF7E2FF174823E00A2B0ED17A
:102C2800164B186814F098F9154A00231370114AC6
:102C38001370144A1370FFF7D1FF134812E00020F5
:102C480002F09EFD114A00231360114A13800D4BB8
:102C580002221A700F4B186806F030FE22780E4BCD
:102C68000E481A70BDE81040FFF769B871260020B9
:102C78007A0D0020770D0020040F0020D0360020A8
:102C88007B0D0020E4380020F0100020C40D002047
:102C9800D20D0020E42600208E26002038120020C5
:102CA800034B01224FF4FC601A7003F06FBA00BFA7
:102CB800770D0020044B054800221A70044B0C22A3
:102CC8001A70FFF73CB800BF770D002044190020A8
:102CD80071260020044B054800221A70044B0D226F
:102CE8001A70FFF72CB800BF770D0020A80F00203E
:102CF8007126002007B50A4A0023137004228DE8C4
:102D08000C00C6201022232356210CF007FC054B8B
:102D180005480A221A7003B05DF804EBFFF70FB8F4
:102D2800770D002071260020F010002007B50A4A10
:102D38000023137004228DE80C009720102223230F
:102D480056210CF0EBFB054B054809221A7003B01D
:102D58005DF804EBFEF7F3BF770D00207126002025
:102D6800040F002007B50B4B00221A70082203231A
:102D78008DE80C004920102223233D210CF0CEFBC6
:102D8800054B064801221A7003B05DF804EBFEF704
:102D9800D6BF00BF770D0020712600206C150020DB
:102DA80008B50D4B002018700C4B18700C4B1870A0
:102DB8000C4B08221A700C4B187003F013FA0B4BCB
:102DC800012119704FF080400EF001FE0848BDE85F
:102DD8000840FEF7B4BF00BF95260020D40D0020A0
:102DE800770D002071260020FC2C0020E8360020FA
:102DF800600E002070B51F4C1F4E20684FF6E0751E
:102E0800294600F06DFC20681C4900F017FC60683A
:102E1800294600F065FC6068194900F00FFCA068BD
:102E2800294600F05DFCA068164900F007FC01F097
:102E380095FD4FF47A6008F001FF2068294600F0FC
:102E48004FFC2068314600F0F9FB6068294600F025
:102E580047FC6068314600F0F1FBA068294600F0A5
:102E68003FFCA068314600F0E9FBBDE8704001F086
:102E780075BD00BFE00C002090B1050808AE05083C
:102E88001CAE05082CAE05080C4B10B500241C70B0
:102E98000B4B01221A70204609F010F8204603F067
:102EA800A1F9084B0B221A7009F066FB0AF0E7F843
:102EB8000548BDE81040FEF742BF00BF770D00206F
:102EC800FC2C002071260020101600200F4A002339
:102ED80010B513700E4A13700BF07AFF044628B130
:102EE800FFF788FFBDE8104001F038BD03F07AF91C
:102EF80009F068FA074B1C70074B07221A7009F093
:102F08005BFA0648BDE81040FEF719BFD40D002053
:102F1800770D0020FC2C00207126002024140020AE
:102F2800144A002310B51370134A1370134A137010
:102F38000BF04EFF28B1FFF75DFFBDE8104001F030
:102F48000DBD03F04FF90E4B01241C7009F03AFA3D
:102F580006F022FD0B4B06221A7009F02DFA4FF0ED
:102F6800804021460EF033FD0748BDE81040FEF7CB
:102F7800E6BE00BF95260020D40D0020770D002066
:102F8800E8360020712600204C1000202DE9F04F73
:102F9800734DDFF830928BB000244FF6FF78284647
:102FA80001F0A3FA4146224623466E480094019454
:102FB80000F05AFB4FF6E07604270390314622468C
:102FC800234669480097019400F04EFB314604906F
:102FD8002246234665480097019400F045FB414688
:102FE80005902246234648460097019400F03CFB92
:102FF8005F4E41463060224623464846009701947A
:1030080000F032FB2346706041462246484600974E
:10301800019400F029FB5749B060574A204601F057
:103028001BF85649564A8046204601F015F855497E
:10303800554A0746204601F00FF85449544A81463C
:10304800204601F009F85349534A8246204601F0C8
:1030580003F85249524A8346204600F0FDFF514981
:10306800514A84462046CDF808C000F0F5FF4F4984
:1030780006904F4A204600F0EFFF4E4907904E4A0F
:10308800204600F0E9FF4D4908904D4A204600F0DF
:10309800E3FF21460990039A2B46204601F0F4F8F5
:1030A8002146049A2B46C82001F0EEF80A21059A19
:1030B8002B46C82001F0E8F8552132682B467820C5
:1030C80001F0E2F8692172682B46782001F0DCF8FB
:1030D800B2682B467D21782001F0D6F828213A469F
:1030E8002B46052001F0D0F8962142462B460520B4
:1030F80001F0CAF8D2214A462B46052001F0C4F84F
:10310800D22152462B46562001F0BEF8D2215A460B
:103118002B46A62001F0B8F8DDF808C0B4216246B5
:103128002B46052001F0B0F8B421069A2B4656200C
:1031380001F0AAF8B421079A2B46A62001F0A4F8BA
:10314800B421089A2B46F62001F09EF8099AF62039
:10315800D2212B460BB0BDE8F04F01F095B800BF67
:10316800A0180020F7B1050800B205080DB205083F
:10317800E00C002018B20508DD2C000826B205086E
:103188006D2D00082EB20508912E000837B20508EB
:10319800292F000840B20508D52E000849B20508B5
:1031A800A92D000852B20508352D00085BB20508A4
:1031B800FD2C000864B20508BD2C00086CB2050897
:1031C800A92C00088DB1050807B5032308228DE84E
:1031D8000C004920102223233D210CF09FF9044BB9
:1031E800044801221A7003B05DF804EBFEF7A7BD8E
:1031F800712600206C1500202DE9F743314E324F1F
:10320800324D0024304601F070F92246234647F635
:10321800FF712F480094019400F026FA4FF6FF78CA
:10322800814641462246234638460094019400F0E0
:103238001BFA4146286022462346384600940194EA
:1032480000F012FA41466860224623463846009448
:10325800019400F009FA2346A86041462246384600
:103268000094019400F000FA1A49E8601A4A2046CE
:1032780000F0F2FE214607464A463346204601F052
:1032880003F83C212A683346192000F0FDFF5A2133
:103298006A683346192000F0F7FF7821AA68334698
:1032A800192000F0F1FF9621EA683346192000F052
:1032B800EBFFEC20D2213A46334603B0BDE8F04399
:1032C80000F0E2BF941100208DB10508EC0C00203D
:1032D80074B20508D9AE0508D13100081C4B1A781C
:1032E8001C4B10B51A7009F04DF91B4B1B4A0024F2
:1032F8001C6002202346CA2103F082F8204608F009
:10330800DDFD174B1C80174B1C70174B1B78023BBD
:10331800052B1CD8DFE803F003070B13170FBDE8D4
:103328001040FEF775B9BDE81040FEF75FB9BDE87B
:103338001040FEF749B9BDE81040FEF721B9BDE8D5
:103348001040FEF72FB9BDE81040FEF707B910BDD1
:103358008E26002071260020C40D00208CB105089F
:10336800E4360020E4380020FC2C002008B5084B87
:10337800186806F0A3FA002002F034FF09F0FCF800
:10338800044B05480B221A70BDE80840FEF7D7BC6D
:10339800E42600207126002010160020114B10B5DD
:1033A80000241C70104B186806F088FA204602F0BA
:1033B80019FF0E4B1B780B2B0ED8DFE803F006061F
:1033C8000D0D0D0D0A080D0D0D06094802E00948FE
:1033D80000E00948FEF7B3FC084B1C70BDE810403C
:1033E80009F0CAB8FC2C0020E42600207126002031
:1033F800A0180020241400204C100020E4380020DD
:103408002DE9F041144C204601F06FF800201349D3
:10341800134A00F021FE1349134A0746002000F022
:103428001BFE1249124A0646002000F015FED22162
:1034380005463A462346E62000F026FF4B21324651
:103448002346642000F020FF642069212A46234691
:10345800BDE8F04100F018BF381200202EAB050877
:10346800A53300087CB205087533000888B2050842
:10347800E532000808B508B143682BB90348044A87
:10348800044B9B2101F092FC586908BD95B20508D0
:10349800402C0408B7B2050808B5FFF7EBFF8068B1
:1034A800123080B208BD08B5FFF7E4FF4068063067
:1034B80080B208BD2DE9F84F04468846FFF7DAFFC9
:1034C8006689E589074606F1030905F10F0AB8F18F
:1034D800000F1FD01F2002F059FE2046FFF7DCFF27
:1034E80083462046FFF7DFFF294603465FFA8BF243
:1034F800F0B202F08BFE042002F04AFF0B364FF6C2
:10350800FF70033502F042FEB0B2A9B23A68012357
:1035180002F076FF3D69204641464A465346A84791
:10352800BDE8F88F13B504460DF1060101A803F0B4
:10353800A1F92046FFF79EFF6389BDF80410BDF886
:103548000620C91AE389D21A0339C3680F3A2046FC
:1035580098471CBDF7B5044614200D4616461F466D
:1035680013F0F2FC089BC7600361064B0649074A43
:1035780080E8700000930190054B002000F05DFE8C
:10358800FEBD00BFBD340008AF340008A1340008F8
:103598002D350008704708B508B143682BB90448B1
:1035A800044A054BAD2101F001FC586908BD00BF74
:1035B800D6B20508582C0408B7B20508F8B5054670
:1035C8000E46FFF7E8FF836B04461BB128463146D9
:1035D800984700E018466F8994F83C30ED890EB999
:1035E800034310D0208E02F0D1FD608E02F0E4FD7E
:1035F80094F8350002F0CCFE94F834303846294669
:10360800224602F0FDFE002384F83C30F8BD08B5E0
:10361800FFF7C1FF90F83500BDE8084002F0CDBEC5
:1036280038B5FFF7B8FF044614F086F8054694F855
:10363800350002F0BDFE684380B238BD38B50D468E
:10364800FFF7A9FF29462E22044614F0A5F850B129
:10365800204629462E2214F0F1F8002384F82E3053
:10366800012384F83C3038BD2DE9F7430746402054
:103678000E461546984613F067FC044628B91148CB
:10368800114A124B4E2101F091FB114B114A12497C
:103698008DE818000020114B00F0CFFD3946814617
:1036A800FFF7CCFF9DF82830268684F835300B9B31
:1036B8006586A363002384F8348084F83C30484648
:1036C800BDE8FE83D6B20508702C0408F4B20508DC
:1036D800C535000817360008293600089D3500084A
:1036E80010B50C46FFF757FF0123048680F83C30DD
:1036F80010BD00BF4FF4A0707047C82070477047D6
:10370800074B1B78022B07B508D1064B1B78022BF9
:1037180004D001A80DF1060103F0ACF80EBD00BFFE
:10372800E4380020FC2C002073B50A4B06460D46F1
:103738001446009300200849084A094B019000F0FC
:103748007CFD294602462346304602B0BDE870405B
:1037580000F09ABD07370008FD3600080337000857
:103768000937000813B502AB03E90600436843B103
:10377800027C0124082A9C7004D11B6921469847C1
:1037880000E01C4620461CBD30B500282BD0058B18
:10379800002425E0036A1A7C012A05D15B681A888F
:1037A8008A421BD1187F30BD052A06D15B681A886A
:1037B8008A4213D193F82C0030BD032A06D15B68E6
:1037C8001A888A420AD193F8250030BD062A05D105
:1037D8005B681A888A4201D1D87A30BD0134043036
:1037E800AC42D7D3002030BD08B1817501207047A5
:1037F800F8B504460D46D0B1E175D0F89830984731
:10380800012D0DD12746002606E0F86900F10802CF
:10381800436906CA98470136238B04379E42F4D37E
:10382800D4F898302046294698470120F8BDF8BDBD
:10383800F8B50546084617460E4613F07DFF013FCA
:10384800B84234BF04463C463CB12846314622467D
:1038580013F0F4FF00232B55F8BD2C70F8BDF7B515
:10386800044600200090019000296CD00E8B68E07F
:1038780000F1080351F823301D7C042D04D15D6844
:103888002D88954247D0013000F1080351F82330C4
:103898001D7C012D04D15D682D8895423BD00130F7
:1038A80000F1080351F823301D7C052D04D15D6813
:1038B8002D8895422FD0013000F1080351F82330AC
:1038C8001D7C032D04D15D682D88954223D00130DD
:1038D80000F1080351F823301D7C022D04D15D68E6
:1038E8002D88954217D0013000F1080351F8233094
:1038F8001D7C072D04D15D682D8A95420BD00130BF
:1039080000F1080351F823301D7C062D08D15D68AD
:103918002D88954203D103F10801204615E00130B6
:1039280000F1080351F823502B7C082B09D16F684C
:103938003F88974204D105F1080120461A4605E060
:103948000130B04294D320466946082213F0ACFDFA
:103958002046FEBDF8B505460F461646002830D06D
:103968004388032B2FD0202013F0EEFA04460028BA
:103978002BD040F80C5B39460C22FFF759FF182072
:10398800E66113F0E1FA0646B8B102230374012395
:1039980063760F4B446063600E4BA360002323766D
:1039A8006B8805EB830201339BB2012B50606B805F
:1039B8000CD16A685268137608E0204613F0CCFAF6
:1039C80004E0064602E0002600E006463046F8BD60
:1039D800BCAB04085AA8040837B5456802AB03E92C
:1039E80006003DB3037C0124042B85F8314022D125
:1039F800688E02F0CBFB95F8300002F0C9FC95F810
:103A0800343043B9BDF80200BDF80610AA1C23469D
:103A180002F0F6FC0FE0012B03D1084840F23951BF
:103A280004E0022B07D1054840F24151044A054BF6
:103A380001F0BCF92C4620463EBD00BF07B305087F
:103A48003077040805B30508F8B504460F4616464E
:103A580010B3838A0A2B20D0202013F075FA05466C
:103A6800E8B14460102200F108003946FFF7E0FE93
:103A78004FF6FF73A08A2B801F236B8000232B76C1
:103A8800831D013080B20128EE6144F82350A082E2
:103A980007D1A3691876F8BDF8BD0020F8BD01204C
:103AA800F8BD0120F8BD2DE9F3471D464B1C98428F
:103AB80082460C461746BDF828600DDD95420BDCA2
:103AC80001320AF101035B1A521BC8B2D2B29BB28F
:103AD8002946009602F092FBAAF1020A3046C4EB8E
:103AE8000A0A02F053FB4FF000084FF001091FFAD1
:103AF8008AFA0BE0601C08EB050180B289B25246D5
:103B08000023009602F072FB09F101097B1B08F102
:103B1800010899451FFA88F8ECD3BDE8FC87F8B589
:103B2800C7B2144638461E460D4602F071FB621EA7
:103B380092B23846294602F06BFB304602F026FB6B
:103B4800022606E0A21B92B23846294602F060FB24
:103B58000136A642F6D3F8BD73B504460E4600F109
:103B68001E001546009200233C2280B21E3E02F041
:103B78003DFBB1B220463C220123009502F036FB02
:103B88007CBD73B504460E460138154600920023E5
:103B9800032280B2013E02F029FBB1B22046032283
:103BA8000123009502F022FB7CBDF7B5089D2E7B12
:103BB800EF7A1C463604AB7A06EB0726F618431A4A
:103BC800687B06EB00602D1800200190121B084648
:103BD8002146009501F002FFFEBD30B5456885B06D
:103BE80004AB03E906007DB101242C736D68BDF8B0
:103BF8000800BDF80A109DF80C209DF80E300095BD
:103C0800FFF7D3FF204600E0284605B030BD2DE978
:103C1800F04385B004AB03E906004468BDF80860CA
:103C2800BDF80C70002C41D0012384F8263094F89C
:103C380025300BB9A26800E06268FFB2BDF80A102F
:103C48009DF80E30009230463A46FFF7AEFF04F179
:103C58000C08022002F09CFB404613F06DFD05465F
:103C680000B1451E0F3F0024153E1FFA87F90DE0ED
:103C780002F098FB02F09CFB04FB106189B24846F5
:103C88002022002302F0D6FB0134E4B2AC42EFD389
:103C9800002002F07BFAB8B2B1B24246012302F02A
:103CA800C9FB002002F074FB012000E0204605B0AB
:103CB800BDE8F0832DE9F04385B004AB03E90600C5
:103CC8004568BDF80860BDF80C70002D3CD0012394
:103CD8006B762B7EBDF80A10012B0CBF6A68AA68A8
:103CE8009DF80E300092FFB23A463046FFF75DFF6E
:103CF8000C35022002F04CFB284613F01DFD0E3F48
:103D080081460024163E1FFA87F80DE002F04AFBB0
:103D180002F04EFB04FB106189B2404620220023CA
:103D280002F088FB0134E4B24C45EFD9002002F0E0
:103D38002DFAB8B2B1B22A46012302F07BFB00206B
:103D480002F026FB012000E0284605B0BDE8F0831C
:103D58002DE9F04F85B00546DDF8409002914846C0
:103D68009046039313F0E8FCDDF838A0DDF83CB08A
:103D78000646294600242F4611E024B1B4420CBF60
:103D88005B46534600E0039B01F10805ADB2009382
:103D98002846029A4346FFF708FF01342946B442F1
:103DA800EBDD002002F0F2F9022002F0F1FA7D1DAD
:103DB80008F10508A8B21FFA88F14A46012305B0A0
:103DC800BDE8F04F02F01CBB70B5406886B006AB8A
:103DD80003E9060000282ED0012380F82D308668DC
:103DE800164BF21A534243EB020390F82C205AB1B7
:103DF800002B134D134B144A08BF1D46134B00F1FB
:103E08001C0418BF13460AE0002B0D4D0D4B0E4A3B
:103E180018BF1D460D4B00F10C0408BF1346BDF832
:103E28001200BDF81410BDF81620009601950294F2
:103E3800FFF78EFF012006B070BD00BFA080040808
:103E4800DC7C040882820408BE7E040864840408BA
:103E580070B5446886B006AB03E9060004B30123D5
:103E68006377A668104B227FF11A4B4243EB01039C
:103E78000AB10BB904E01BB966680C4D0C4B01E0A4
:103E88000C4D0D4BBDF81200BDF81410BDF81620EE
:103E980000960C3401950294FFF75AFF012000E0C8
:103EA800204606B070BD00BFEC8B040828880408C3
:103EB8000A8A0408C28D0408988F04082DE9F04383
:103EC80085B004AB03E906004468BDF80860BDF896
:103ED8000A90BDF80C50BDF80E80002C00F08C80C4
:103EE8000123A3740220676802F052FA4FF6FF70AC
:103EF80002F062F9002002F049F9EDB25FFA88F8A1
:103F0800A6F1160189B230462A4643460097FFF7C4
:103F18004CFE277A002F2ED1A28A234600E00137D3
:103F2800974204D29969097E04330029F7D002F038
:103F380039FA02F03DFAA9F116091FFA89F90E219A
:103F480001FB10914FF6FF7208F101085FFA88F340
:103F580089B2009248462A46FFF7A5FD022002F0E2
:103F680017FA1F2002F012F9A38A002B38D0103D4F
:103F7800E8B2303E2CE0E3685C68A28A2346013A46
:103F8800002700E00137974204D29969097E04337B
:103F98000029F7D002F006FA02F00AFA0E2101FB16
:103FA80010914FF6FF7208F101085FFA88F389B2A1
:103FB800009248462A46FFF776FD022002F0E8F90B
:103FC8001F2002F0E3F8A38A53B1103DE8B21A3E6D
:103FD8000637B1B254F827200123083202F02AFA32
:103FE800002002F0D5F94FF6FF7002F0E5F81F2027
:103FF80002F0CCF8012000E0204605B0BDE8F083CF
:104008002DE9F04105463620884614461F4612F031
:104018009BFF0646E0B120F8025B41462E22FFF7DF
:1040280007FCBDF8183086F8344073861820012341
:1040380086F8307086F8313012F086FF044618B1E1
:1040480004234660037404E0304612F085FF00E064
:1040580004462046BDE8F081F8B5064624200F4600
:10406800154612F071FF0446D8B10F4B06808360E5
:104078000E4B39464360102200F10C00FFF7D8FBC5
:1040880001260023182025622377667712F05CFF4B
:10409800054610B14460067404E0204612F05CFF47
:1040A80000E005462846F8BDEC8B0408468604085F
:1040B800F8B506462C200F46154612F045FF044673
:1040C800E8B120F80C6B39461922FFF7B1FB0D4B0C
:1040D800A562A3600C4B6360002384F82530182088
:1040E800012384F8263012F02FFF054618B1032368
:1040F8004460037404E0204612F02EFF00E00546F9
:104108002846F8BDF8A4040896A1040810B504468A
:10411800142012F019FF20B100234380014B0480C2
:10412800036110BD5D39000838B50546442012F01A
:104138000BFF0446C0B10E4B058243600D4B036074
:10414800012383740023037283820B4B03641820BA
:1041580012F0FAFE054618B107234460037404E020
:10416800204612F0F9FE00E00546284638BD00BF9B
:104178008C9D040882990408513A00082DE9F04101
:1041880005463420884614461F4612F0DDFE0646D2
:1041980020B3144B05808360134B414643601022C3
:1041A80000F10C00FFF744FB214606F11C00102229
:1041B800FFF73EFB002386F82C30182001233763D5
:1041C80086F82D3012F0C0FE044618B1052346606B
:1041D800037404E0304612F0BFFE00E004462046B7
:1041E800BDE8F081A0800408FA7A04082DE9F041BE
:1041F800044614200D461646984612F0A5FE0746BA
:10420800B8B1069B048003610023C3720123456093
:10421800068180F80A800373182012F095FE044680
:1042280018B106234760037404E0384612F094FE80
:1042380000E004462046BDE8F0812DE9F04104463F
:1042480018200D461646984612F07EFE0746B8B16D
:1042580001238370069B04800361079B4560866089
:10426800C0F80C804361182012F06EFE044618B1A5
:1042780008234760037404E0384612F06DFE00E03E
:1042880004462046BDE8F0812DE9F34198461B8B92
:104298001D2B05460C4617464FF0000000F2B4806F
:1042A800B5F5A07F0090019000F2AE80F02900F2F1
:1042B800AB80127CADF80610511EADF802500729EC
:1042C80000F28A80DFE801F045595E04456A1476F9
:1042D8007B684E4A7A611A8893F834303A80013BF9
:1042E800DBB2012B7FD8ADF80240ADF806507AE07A
:1042F80005F11602ADF8002004F11602ADF804200D
:1043080002AE434A16E903007A6107F1080282E81F
:10431800030003F10802013348F82270A8F81830A6
:104328007B681A8A187A3A8000286CD1FFF7FCFE5D
:104338003849436859603849DF600126163D1960DD
:1043480002461E72A8B2E1B24346FFF79DFF30460F
:104358005AE0012A0CBF314B314B78687B6130F849
:104368000C3B3B8013F0E8F9431CDB001A34ED18D2
:10437800ADF80440ADF8005035E07B68294A1B6869
:104388007A6102E0284A7B687A611B8814353B8091
:10439800ADF800501434ADF8044024E07B68234A9B
:1043A8007A611A883A801A899B7AAD18ADF800505C
:1043B800E418F0E77E681E4B7B61338838463B8003
:1043C80073689847013D4519ADF80050B368384601
:1043D8009847013C0419DEE71648174A174B40F284
:1043E8001A3100F0E3FC02AA12E9030007F10803FE
:1043F80083E80300B8F8183003F10802013348F8DD
:104408002270A8F818300120BDE8FC81E1390008C5
:10441800C53E0008789504086E910408593E0008C6
:10442800D13D0008BD3C0008173C0008E33B0008EC
:104438006D37000807B305084077040805B3050879
:10444800F8B51646002834D01378002B2ED0028BEE
:10445800002327E0046A257C042D21D165682F8874
:104468008F421DD195F8313053B16F8E01F0B4FEF3
:1044780004F1080268866369204606CA98476F8671
:10448800A81C31462E22FFF7D3F995F831307BB1BD
:1044980004F108026369204606CA98470120F8BD5E
:1044A800013304309342D5D30020F8BD1846F8BD37
:1044B8000120F8BD70B5B8B1068B0446002310E0A2
:1044C800256A287C04280AD16D682888884206D184
:1044D8001046A91C2E22FFF7ABF9012070BD01334D
:1044E8000434B342ECD3002070BD38B5044620B381
:1044F800134BC361134BC0F89830134BC0F89C3072
:10450800124B00257822C0F8A0308575C575058343
:10451800294600F1200013F009F8D4F89830204615
:10452800294698470A4A1388312B07D8094941F880
:10453800234001331380012038BD38BD284638BDDB
:10454800F9370008F1370008913700086738000884
:10455800FC0C0020E81900202DE9F0410446002851
:1045680000F0B380078B02460025A8E0136A1E7C82
:10457800042E00F08780012E23D1586803888B42CF
:1045880040F09B8005F1080712F0E6FC54F827007C
:104598004FF00008C0F8048012F0DEFC228B531E96
:1045A8009D4208D00732238354F8221044F827107C
:1045B80044F8228002E044F8278025833046BDE88D
:1045C800F081052E5ED0032E5CD0022E13D15B68DD
:1045D800186803888B4270D14388013B9BB24380A3
:1045E8000BB912F0B9FC05F1080654F826305868E2
:1045F80012F0B2FC4EE0072E21D15E68338A8B425E
:104608005BD1002706E0BB1D013756F8230012F0E6
:10461800A3FCFFB2B38ABB42F5D80027B78205F1E5
:10462800080654F82630586812F096FC54F826000C
:1046380033E044F8267025830120BDE8F081062E7A
:104648001ED1586803888B4237D105F1080612F04D
:1046580083FC54F826000027476012F07DFC228B6B
:10466800531E9D4209D00833013A54F8231022837F
:1046780044F8261044F82370DEE744F826701AE060
:10468800082E1AD1586803888B4216D112F064FCA0
:1046980005F1080654F826000027476012F05CFC74
:1046A800228B531E9D42C4D0073254F8221044F87E
:1046B800261044F822702383BEE701350432BD4238
:1046C800FFF454AF0020BDE8F081BDE8F08170B57B
:1046D800044600282AD0068B751E083600EB86068D
:1046E8001EE056F8043D1A7C042A13D0012A11D082
:1046F800052A0FD0032A0DD0022A02D15B681B6855
:1047080009E0072A02D15B68198A05E0062A01D068
:10471800082A04D15B6819882046FFF71DFF013D70
:10472800681CDED100232383012070BD70BDF0B565
:1047380028B30023068B1A461EE0046A257C072D41
:1047480018D16468258A8D4214D1A78A002504EB04
:1047580083040DE004EB050C0435DCF818C09CF864
:1047680018C0BCF1010F03F1010301D1D8B2F0BDAB
:10477800BB42EFD301320430B242DED30020F0BD99
:1047880070B508B3048B00231BE0026A157C072D63
:1047980015D15268158A8D4211D10023958A114688
:1047A8001C46012007E013B99669307601E08E694E
:1047B800347601330431AB42F5D3012070BD0133A7
:1047C8000430A342E1D3002070BD2DE9F04128B3A5
:1047D8000023078B1A461EE0046A257C072D18D192
:1047E8006468258A8D4214D1B4F814C0002504EBFE
:1047F80083040CE066190435B66996F81880B8F198
:10480800010F03D106F10800BDE8F08101336345CB
:10481800F0D301320430BA42DED30020BDE8F08183
:104828002DE9F04700282FD00023B0F818C01D4606
:1048380027E0046A267C072E21D16468268A8E42E6
:104848001DD1B4F81480002604EB830915E009EBA8
:104858000604A7693C7E012C0DD192F800A0BAF19C
:10486800000F08D007F1080011461022FEF7E0FFFC
:104878002046BDE8F087013304364345E7D30135C8
:1048880004306545D5D30020BDE8F087F0B5B0B158
:10489800068B002510E0046A277C062F0AD164687D
:1048A80027888F4206D123819DF814306260A37255
:1048B8000120F0BD01350430B542ECD30020F0BD35
:1048C80010B500210446FEF793FF20460121BDE8FC
:1048D8001040FEF78DBF38B598B1048B024600230F
:1048E8000CE0106A058804328D4206D100F10802F6
:1048F800436906CA9847012038BD0133A342F0D363
:10490800002038BD10B50C460021FEF771FF204687
:104918000121BDE81040FEF76BBF13B502AC04E9F6
:104928000C00BDF80230834206D8BDF8003083423F
:1049380034BF0020012000E00020BDF806308B4283
:1049480006D8BDF804308B4234BF0021012100E0B5
:104958000021002818BF0846C0B21CBD38B5114B4D
:10496800114A1988002319E052F8045FA87D01282C
:1049780012D100240CE004F1080355F82300037C4D
:10498800082B03D1436800211B6998470134A4B25E
:104998002B8BA342EFD838BD01339BB28B42E3D1B6
:1049A80038BD00BFFC0C0020E4190020704770B52A
:1049B800094CA5787DB9094B1E78012E0BD1636887
:1049C800013363606268064B9A4204D9284601F0B5
:1049D800A1FCA670656070BDFC0C00209801002049
:1049E80040420F00054A9060134602E09968013979
:1049F800996091680029F9D1704700BFFC0C00202C
:104A0800F0B585B001F034FF002800F04981002599
:104A180002A80DF10A01ADF80850ADF80A5001F0EE
:104A280029FF03A80DF10E01ADF80C50ADF80E509A
:104A380001F06CFFBDF80C10BDF808200091BDF81E
:104A48000E10BDF80A3001912C46964D9649082063
:104A58000AF0C2FFA878012803D101F05BFCAC7012
:104A680019E1924B5B78012B40F01581AB78002B54
:104A780040F011816B6029888D4A09E152F8046F72
:104A8800B07D012840F002810025FAE005F1080315
:104A9800BDF8080056F82340BDF80A1004F10803D1
:104AA8000CCBFFF73AFF002800F0E980237C013B9C
:104AB800062B00F29F80DFE803F00429159D1F9D57
:104AC8004C006668012304F10805337795E8060071
:104AD800636920469847002333772046636995E841
:104AE800060086E0636893F8252012F1FF3218BFAC
:104AF800012283F8252077E0636893F82C2012F1CF
:104B0800FF3218BF012283F82C206DE06268137E03
:104B18001568002B6ED16E882F462946184606E088
:104B280051F804EFDEF804E001338EF81800B342C0
:104B3800F6D301231376002607E057F8040F00F197
:104B48000802436906CA984701366B889E42F4D327
:104B580050E0656820892E68A37B227B0096A0F12F
:104B6800160189B2FFF721F81420FFF73BFF2B7AD3
:104B7800C3B9AF8A29461A461E4609E0886990F8E3
:104B880018E00676BEF1010F08BF13460431013262
:104B9800BA42F3D301220BB9AB6924E0053355F8C7
:104BA800233020E06368DB685A680023908A154642
:104BB80019461F4609E0AE6996F818E03776BEF147
:104BC800010F08BF0B46043501318142F3D3411E62
:104BD8008B4203D1053052F8203003E004D207336A
:104BE80052F8233001221A7604F1080206CA6369D2
:104BF80020469847237C013B072B4CD8DFE803F07D
:104C08000410074B0A0D123A63681B6A34E06368A4
:104C18009B6A2DE063681B6B2AE063681B6927E0C9
:104C2800636824E063681A7A7AB9988A1946013861
:104C380000E00132824204D28C69247E0431002CC7
:104C4800F7D0063253F8223011E0DB685A68908AB0
:104C580011460138002300E00133834204D28C69F5
:104C6800247E0431002CF7D0063352F82330DB6958
:104C7800984710E06368DB68204698470BE00135E9
:104C8800ADB2338BAB423FF601AF04E001339BB2C8
:104C98008B427FF4F3AE01F031FE0F20FFF7A2FE46
:104CA80005B0F0BDFC0C00202DB3050898010020CC
:104CB800E4190020034B9A6812B19A68013A9A6085
:104CC800704700BFFC0C00202DE9F3470120DFF8F6
:104CD800D080DFF8D09001460CF018FA01240025A6
:104CE8004FF4807602274046694600968DF8047096
:104CF8008DF805408DF806508DF807400BF05EFEE4
:104D08004046082122460BF0D9FE244BDFF8988054
:104D18001A6844F2A243B2FBF3FA0AF1FF3A2046BA
:104D280021461FFA8AFA0CF021FAC8F804A048466E
:104D38004146A8F80050A8F80250A8F8085088F88A
:104D48000A500CF0AFFD7023A8F80C300423A8F823
:104D580010300AF1FF3A6323642203FB0AF3B3FB22
:104D6800F2F39BB2C8F8143008F10C014846A8F8D1
:104D78000E40A8F81870A8F81A50A8F81C60A8F8EF
:104D88001E500CF0ADFE484621460CF020FE484669
:104D980021460DF026F9BDE8FC8700BFE40100209C
:104DA80000000240000001400C0D002083B50E46B3
:104DB8000746154910201C4615460AF00DFE10201E
:104DC80012490AF009FE102011490AF005FE1020C8
:104DD8000E490AF001FE002310200E4901930AF043
:104DE800FBFD334610200C493A460AF0F5FD102029
:104DF8000A492A460AF0F0FD1020094922460AF01D
:104E0800EBFD019B0133E7E767B305086CB30508C1
:104E18008CB305089CB30508ACB30508C1B30508F5
:104E2800D2B3050808B5164B1A6A01321A621A6A13
:104E3800012A1A4603D0134840F21E210FE0586297
:104E4800194602E04B6A013B4B62506A0C4B002842
:104E5800F8D11A6A012A06D00A4840F229210A4ADA
:104E68000A4BFFF7A3FF1A6A013A1A621B6A2BB1B1
:104E78000448054A064B40F22B21F2E708BD00BF63
:104E88000C0D0020E3B305081EAF04080DB4050897
:104E98001EB4050810B5084C0221002220460BF06C
:104EA80002FE44F6FF70FFF7BDFF204602210122F3
:104EB800BDE810400BF0F7BD000402400C4B0D4953
:104EC8001A6844F2A2436428B2FBF3F3D4BF20EA81
:104ED800E0706420013B9BB24B60013B5843642265
:104EE800B0FBF2F080B2486103480C310CF07BBD96
:104EF800E40100200C0D00200000014010B5134B08
:104F080093F828202AB11248124A134B40F209316B
:104F18000EE0012283F8282066234FF0C042013BAF
:104F2800DBB2108033B90A480A4A0C4B40F21331FD
:104F3800FFF73CFF1488A4B28442F0D1084B1980D3
:104F4800024B002283F8282010BD00BF0C0D002062
:104F5800E3B3050828AF04082FB4050805B305080E
:104F68000000026010B5FFF7AFFE6420FFF7A6FF50
:104F780021210720FFF7C2FF3220FFF753FF01214D
:104F88000020FFF7BBFF3220FFF74CFF232107204B
:104F9800FFF7B4FF3220FFF745FF00211020FFF78D
:104FA800ADFF41F28830FFF73DFF33210720FFF7BF
:104FB800A5FF3220FFF736FF112046F63001FFF734
:104FC8009DFF3220FFF72EFF4FF4C0610220FFF74C
:104FD80095FF3220FFF726FF122046F6EB41FFF738
:104FE8008DFF3220FFF71EFF03204AF6A401FFF7CA
:104FF80085FF3220FFF716FF00210C20FFF77EFF08
:105008003220FFF70FFF0D2040F60C01FFF776FF67
:105018003220FFF707FF0E204FF42C51FFF76EFFE9
:105028003220FFF7FFFEB0211E20FFF767FF322076
:10503800FFF7F8FE012042F63F31FFF75FFF32200D
:10504800FFF7F0FE05200021FFF758FF3220FFF799
:10505800E9FE00210620FFF751FF3220FFF7E2FEAC
:1050680016204EF61C71FFF749FF3220FFF7DAFED3
:10507800172040F20311FFF741FF3220FFF7D2FE5D
:1050880000210B20FFF73AFF3220FFF7CBFE00216B
:105098000F20FFF733FF3220FFF7C4FE4120002125
:1050A800FFF72CFF3220FFF7BDFE42200021FFF75B
:1050B80025FF3220FFF7B6FE00214820FFF71EFF2C
:1050C80040F23F143220FFF7ADFE21464920FFF79A
:1050D80015FF3220FFF7A6FE00214A20FFF70EFF3A
:1050E8003220FFF79FFE00214B20FFF707FF3220F9
:1050F800FFF798FE44204FF46F41FFF7FFFE322080
:10510800FFF790FE00214520FFF7F8FE3220FFF759
:1051180089FE21464620FFF7F1FE3220FFF782FE86
:10512800302040F20771FFF7E9FE3220FFF77AFEE0
:1051380031204FF40171FFF7E1FE3220FFF772FED4
:1051480032204FF40171FFF7D9FE40F202543220A9
:10515800FFF768FE21463320FFF7D0FE3220FFF725
:1051680061FE342040F20751FFF7C8FE3220FFF7F6
:1051780059FE35204FF40171FFF7C0FE3220FFF7CA
:1051880051FE36204FF40171FFF7B8FE3220FFF7C9
:1051980049FE21463720FFF7B1FEA4F500743220FE
:1051A800FFF740FE21463A20FFF7A8FE3220FFF71E
:1051B80039FE2F2041F2BE21FFF7A0FE3220FFF773
:1051C80031FE21463B20FFF799FE3220FFF72AFEE9
:1051D80000212320FFF792FE3220FFF723FE002153
:1051E8002420FFF78BFE3220FFF71CFE25204FF40A
:1051F8000041FFF783FE3220FFF714FE00214F2005
:10520800FFF77CFE3220FFF70DFE4E200021FFF74E
:1052180075FE3220BDE8104004E608B5124B93F83D
:1052280029202AB11148124A124B40F223310FE0CB
:10523800012283F82920222166234FF0C042013B36
:10524800DBB2118033B90948094A0B4B4FF44F714F
:10525800FFF7ACFD108880B22228F0D1024B002263
:1052680083F8292008BD00BF0C0D0020E3B3050812
:1052780035AF04082FB4050805B3050810B51B4B56
:10528800032826D8DFE800F0021A080E1C8841F22D
:10529800280246F628000AE01C8841F2080246F671
:1052A800080004E01C8841F2300246F6300049F25A
:1052B80041318C4214BF014611460BE0188846F66E
:1052C800200249F24131884214BF11464FF48151FE
:1052D80000E000211A8848F689139A4202D1112069
:1052E800FFF70CFEBDE8104097E700BF9A010020C9
:1052F800014B18800A2095E5000002604FF0C0437A
:10530800188003F500331A881A88188880B2704705
:105318004FF0C04322221A8003F5003382B01A8866
:1053280092B2ADF806201B889BB2ADF80630BDF8E6
:10533800060080B202B07047072040F27311DDE525
:1053480007200021DAE582B0044BADF80600BDF86D
:10535800062092B25A8502B0704700BF0C0D00209B
:1053680082B0044BADF80600BDF8062092B25A8010
:1053780002B070479A010020014B80B21880704734
:10538800000002604FF0C04380B218807047024BA3
:1053980080B21880704700BF000002604FF0C04321
:1053A80080B218807047024B80B21880704700BFE7
:1053B8000000026082B0044B0190019ADA62DA6A56
:1053C800002AFCD102B070470C0D002070B54FF0D8
:1053D800C0452A242C800A4C060AC0B226802080A8
:1053E800100AD2B2208022802B222A800A0A228028
:1053F800C9B21A0ADBB221802280238070BD00BFA7
:105408000000026010B50B4614460246FFF7DEFFA7
:105418004FF0C0432C22A0B21A80BDE8104067E7C5
:105428000B4B1A8848F689139A4210B504460AD1DC
:10543800C1F1EF014E2089B2FFF760FD4F202146F0
:10544800BDE810405AE502460B46BDE81040BDE7EE
:105458009A01002008B5FFF7E3FF0F4B1B78012BDB
:105468004FF0C0420D4B0FD12E2111801A881A8897
:105478001B8892B202F0FC0002F4784242EAC000B3
:10548800C3F3C423184308BD222111801A881A883F
:10549800188880B208BD00BFB81A0020000002605A
:1054A80070B5074D0646012421463046FFF7D2FF66
:1054B8000134A4B2C82C25F8020FF5D170BD00BF85
:1054C800E638002010B5084B1B78012B144602D192
:1054D800BDE8104096E7FFF7A3FFFFF79EFE2046C2
:1054E800BDE8104004E700BFB81A002070B5074DAA
:1054F800064601242146013435F8022F3046A4B26D
:10550800FFF7E0FFC82CF5D170BD00BFE6380020DA
:1055180070B505460E46FFF7C3FF01242146013446
:1055280028463246A4B2FFF7CDFFC82CF6D170BD8D
:105538002DE9F84F0C4693460546C718DFF82CA00E
:105548000AE0BAF82A20B1B292B24046FFF7BAFF91
:1055580001364E45F5DB0135BD4205DA264604EB3A
:105568000B091FFA85F8F4E7BDE8F88F0C0D002049
:105578002DE9F04104460D461646BDF81880032B68
:1055880039D8DFE803F00B351927381980B22946D6
:1055980042460137FFF796FFBFB200E00027B74247
:1055A800F3D1BDE8F081E01B80B2294642460137BD
:1055B800FFF788FFBFB200E00027B742F3D1BDE88C
:1055C800F081E91B89B2204642460137FFF77AFF8E
:1055D800BFB200E00027B742F3D1BDE8F0817919E6
:1055E80089B2204642460137FFF76CFFBFB200E0A0
:1055F8000027B742F3D1BDE8F08170B5194B1A4ABC
:10560800598E92F9004064180025A4B28AB0AC42C1
:1056180008BF0124C62C28BFC62415700F264FF6D4
:10562800FF721E865C865A8519202B4600922146F9
:105638000A22FFF79DFF21463046FFF70BFF22465F
:1056480003460A4902A811F0F1FF02AA06A8084970
:1056580011F0ECFF3220D22106AA2B4600F0D0FE32
:105668000AB070BD0C0D0020251B002044B40508AD
:105678004CB405082DE9F341BDF820500C4690467E
:105688001F461A46002306460095FFF771FF611E64
:10569800414430463A46002389B20095FFF768FF37
:1056A80030462146424601230095013EFFF760FF40
:1056B800BF19B8B2214642460123089502B0BDE899
:1056C800F04155E770B50D461C490446088848F670
:1056D800891188422CD1C5F1F001661E9E198A1ADB
:1056E800C5F1EF0392B29BB29A422CBF11461946FC
:1056F800EF2928BFEF219A4238BF134643EA012118
:10570800B6B289B24420FFF7F9FBA64234BF31464E
:1057180021464520FFF7F2FBA64238BF264640F255
:105728003F139E4234BF314619464620FFF7E6FB39
:1057380020462946BDE8704072E600BF9A01002065
:1057480000200146F0224FF4A073BBE770B54FF07C
:10575800C0452A242C80094C060A26802080080A85
:10576800208021802B212980110A218022801A0A79
:10577800228023802C232B8070BD00BF0000026094
:1057880070B5114B1B78012B044607D1002040F25D
:105798003F110246EF23FFF7D9FF04E0FFF7D0FFE0
:1057A8000020FFF76BFDF02509E0013E2046B6B268
:1057B800FFF79EFD002EF8D1013DADB215B14FF4B3
:1057C800A076F2E770BD00BFB81A00202DE9F04FAF
:1057D8001C463E4B87B01B78039183469DF84410C6
:1057E80010980591012B039B049092461FFA8BF0A9
:1057F8009AB208D1411E531E0919534489B29BB26B
:10580800FFF7A4FF09E01FFA8AF51146A3B22A465A
:10581800FFF758FF0020FFF731FD0027DDF80C8067
:105828003E4640F23F1CA14639E0BBF1000F2EDB9B
:1058380065452CDC0398002829DBB8F1EF0F26DC3E
:10584800220702D1002CC8BF013621492140002976
:1058580003DA013961F00F010131059A0AB1C1F18A
:105868000F01049830F8162003FA01F10A4012B229
:105878006AB118494A8D029392B2A8B21FFA88F108
:10588800CDF804C0FFF71EFEDDF804C0029B01340A
:1058980001354C45C9DB0136013708F10108574588
:1058A80003DA5D4600240123F3E7084B1B78012B3C
:1058B80008D1002040F23F110246EF2307B0BDE8AF
:1058C800F04F43E707B0BDE8F04F39E7B81A0020BA
:1058D8000F0000800C0D00202DE9F74F1F463B4BB1
:1058E800DDF830801B7816469DF83420012B0446DD
:1058F80001920D4680B28AB208D1411E531EC919C1
:105908009B1989B29BB2FFF721FF09E01FFA86FEB7
:105918001146BBB27246FFF7D5FE0020FFF7AEFC7A
:105928004FF0000BDA463DE0002C30DB09EB0403B6
:1059380040F23F1293422ADC002D28DB0BEB0503D3
:10594800EF2B24DC19F00F0F04D1B9F1000FC8BFF9
:105958000AF1010A1E4B09EA0303002B03DA013B93
:1059680063F00F030133019A0AB1C3F10F03012257
:1059780002FA03F338F81A2013401BB213B1154B7F
:10598800588D01E0144A508880B2FFF7B1FC09F144
:10599800010901E04FF00009B945C5DB0AF1010A28
:1059A8000BF1010BB345F5DB084B1B78012B08D134
:1059B800002040F23F110246EF2303B0BDE8F04F4C
:1059C800C4E603B0BDE8F04FBAE600BFB81A00203D
:1059D8000F0000800C0D00209A0100202DE9F041F5
:1059E8001C4F069C3F789DF81C60012F02FB03F5B5
:1059F80080B28FB209D1411ECB1899B27B1E9A187A
:105A080093B23A46FFF7A2FE07E092B29BB239463C
:105A1800FFF758FE0020FFF731FC002709E034F8B3
:105A2800020B1EB1030A43EA002080B2FFF760FCB4
:105A38000137AF42F3DB074B1B78012B07D100205E
:105A480040F23F110246EF23BDE8F0417EE6BDE893
:105A5800F04175E6B81A00202DE9F0431F2093B0F5
:105A6800FFF78EFE4FF47840FFF78AFE4FF6E07599
:105A78004FF4FC60FFF784FE2846FFF781FE002004
:105A8800514CFFF77DFE00204FF6FF790146642256
:105A98000346A4F82A90CDF80090FFF769FD00208E
:105AA8000A2164220346CDF80090FFF761FD00202B
:105AB8000146642201234FF4784765850095FFF776
:105AC80057FD7720EF21C82200234FF4FC66678535
:105AD8000097FFF74DFDBD213222012340F23F1010
:105AE80066850096FFF744FDA02032220023782126
:105AF80067850097FFF73CFDA0207821322201231B
:105B08004FF01F0866850096FFF732FDA020782128
:105B180032220223A4F82A80CDF80080FFF728FD5E
:105B2800A02078213222032365850095FFF720FD08
:105B3800264B2749A3F8028002AD3C22284611F0E3
:105B4800B3FCEB20C3210522302300950025A4F8DF
:105B58002A900195FFF7C0FE32210A2096220B46B3
:105B680067850097FFF786FD32213C2096220B4679
:105B780066850096FFF77EFD32210B4696226E2041
:105B8800A4F82A80CDF80080FFF774FDFFF7D8FB52
:105B9800FFF7D2FB3220FFF791F92846FFF78EF97D
:105BA8006420FFF78BF90B4B03F110028DE82400FA
:105BB80028465A681B682946FFF710FF1195119B64
:105BC80001331193FBE700BF0C0D00209A01002060
:105BD8004AAF040808D401082DE9F14FFFF774F81B
:105BE8004FF0C0456420FFF769F90127FFF752F924
:105BF8004FF028096D48FFF715F92F800520A5F803
:105C0800009003F05BFACF232B80694B0026832298
:105C18001E801A8030221A80ED222A804FF06408F4
:105C28000322A3F800801A8012221A8081221A8087
:105C3800E8222A8085221A8079221F801A80CB22A6
:105C48002A8039221A804FF0340C02242C21F722A2
:105C580019801E80A3F800C01C802A8020221A8088
:105C6800EA222A80C0221E80C1211E802A80262284
:105C78001A80298011211980C52129803521198090
:105C88003E211980C7212980BE211980362129800B
:105C98003A205521A3F8009028801980B121298045
:105CA8004FF0100BF2211E80A3F800B029800821C4
:105CB80019802A80E0221F804FF01F092A801A22AB
:105CC800A3F800904FF0180A1A800F210A22A3F8AF
:105CD80000A01A8019800621198045211980872182
:105CE80019803221198007211A804FF0E10E19809E
:105CF8001C80052419801C801E80A5F800E04FF048
:105D0800250E1E80A3F800E04FF0270EA3F800E050
:105D18001C80A3F800B04FF0090BA3F800B04FF0B7
:105D2800780B1880A3F800B04FF04D0BA3F800B023
:105D38001C800D24A3F800A01C8038241C80188027
:105D48002A20A3F80090EF2428802B201E801E8094
:105D58001E801C8028803F201E801E801F80188087
:105D6800B720A5F800C028801980B62129801A809C
:105D780082221A801122A3F800E040461E802927BB
:105D88002A8003F09BF940462F8003F097F90948D1
:105D9800FFF748F82C232F8030462B8040F23F1124
:105DA8003246234601B0BDE8F04FCFE4400D030072
:105DB8000000026040420F002DE9F041022098B037
:105DC800012100240BF0A2F901250226804816962D
:105DD80016A98DF85D408DF85E408DF85F408DF80E
:105DE8005C500AF0EBFD182029460BF08FF9284685
:105DF80029460BF0A3F921460C2276480AF05EFEEC
:105E08000C22744829460AF059FE04210C227148D4
:105E18000AF054FE05210C226E480AF04FFE0721B5
:105E28000C226C480AF04AFE08210C2269480AF044
:105E380045FE09210C2267480AF040FE0A21654800
:105E48000C220AF03BFE0B2162480C220AF036FEB7
:105E58000E210C225F480AF031FE0F210C225D480A
:105E68000AF02CFE07210C225B480AF027FE0821C5
:105E78000C2259480AF022FE09210C2256480AF041
:105E88001DFE0A210C2254480AF018FE0B210C2290
:105E980051480AF013FE0C210A464F480AF00EFE3C
:105EA8000D210C224C480AF009FE0E210C224A480A
:105EB8000AF004FE0C2248480F210AF0FFFD4CF6B8
:105EC800B3734448169316A98DF85C608DF85E404C
:105ED8008DF85F408DF85D500AF070FD16A94FF6F9
:105EE80080733D4816938DF85C608DF85E408DF8A0
:105EF8005F408DF85D500AF061FD40F6B830FEF75E
:105F080091FFFEF7C7FF40F6B830FEF78BFF0F236F
:105F180011934FF4805310270DF13C0809936846FC
:105F28004FF400231094129414941594009401943F
:105F38000294039704940694079408940A94059489
:105F48000B940C93CDF834800F9513950AF0AFFAA3
:105F58000523684611930F9610941294149415947F
:105F6800CDF8388013950AF0A2FA294620460AF09F
:105F78001EFB40F6B830FEF755FF2046FFF7BEF986
:105F880004461649164E3846224609F025FD41F2C8
:105F980089239C4248F68918124F01D044450ED1F6
:105FA800FEF7E0FF00233B70A6F8008010200E49A2
:105FB80048F6891241F2892309F00EFD05E0FFF742
:105FC8000BFE49F241333D70338018B0BDE8F081D3
:105FD80000040240000C02400010024051B40508C1
:105FE8009A010020B81A002068B405084FF0C04391
:105FF80036221A8003F50033012814BF6820482090
:106008001880704770B5244B01228CB01A70002498
:106018000AE0A9B21F2230460135FFF753FA642D72
:10602800F7D10134642C02D00025A6B2F1E7322062
:10603800014602460346FFF7C9F94FF0C0432E2236
:106048001A8003F5003300201E881C881D88A4B21E
:10605800B6B200F09BF8ADB223461049009532461F
:1060680003A811F0E3FA00230A20C82103AA00F0CC
:10607800C7F904F0FC0204F4784444EAC20242EA94
:10608800D522074903A811F0D1FA0A20DC2103AA76
:10609800002300F0B5F9FEE7B81A0020A7B40508F8
:1060A800BFB405082DE9F04F40F23F19484534BF09
:1060B80004464C46EF2B34BF98464FF0EF084A454C
:1060C80038BF9146EF2934BF0D46EF25C4EB090AC6
:1060D800C5EB080785B0BAF1000FB8BFCAF1000ACE
:1060E800002FB8BF7F424FF6FF734C452CBF1A46AE
:1060F80001221FFA8AFA454538BF0123BFB202932D
:106108000FFA8AF63BB29E42BDF838B0019202DD22
:10611800C6F34F0607E0022693FBF6F67642B6B2C0
:1061280001E01E4603E00FFA8AF35B420393144A28
:106138001378022B204629465A4602D1FDF721FD45
:1061480001E0FFF7BFF94C4501D1454514D0039A4A
:1061580033B2934205DD019AF31BA4189BB2A4B293
:1061680000E0334636B23AB29642DADA029A53443B
:10617800AD189BB2ADB2D4E705B0BDE8F08F00BF53
:10618800FC2C002000487047C01A002082B0064B43
:10619800ADF80600BDF8062092B21A80188880B2C1
:1061A80002B0FFF7D0B800BFBC1A0020014B188816
:1061B80080B27047BC1A002082B0064BADF80600CA
:1061C800BDF8062092B21A80188880B202B0FFF794
:1061D800C7B800BFBE1A0020014B188880B27047AC
:1061E800BE1A0020FFF7CCBAFFF76CBA10B5BDF89D
:1061F80008400294BDE81040FFF7BAB910B5BDF8E1
:1062080008400294BDE81040FFF734BAFFF790B990
:106218002DE9F04F4FEA420800253D4C85B08246F3
:106228008B46C8F1030817462E461FFA87F909EB73
:106238000B0C228805EB0A031FFA8CFC9BB2614603
:10624800184692B2CDF804C00293FFF73BF9C9EBA8
:106258000B0292B20392029B22880399184692B2CB
:10626800FFF730F9DDF804C02288C5EB0A039BB2BA
:106278006146184692B20293FFF724F9029B2288DE
:106288000399184692B2FFF71DF905EB0B0292B27B
:10629800039209EB0A03228803999BB2184692B22B
:1062A8000293FFF70FF9029B2288C5EB0B0C1FFA2C
:1062B8008CFC1846614692B2CDF804C0C9EB0A09B5
:1062C800FFF700F9228803991FFA89F992B2484624
:1062D800FFF7F8F82288DDF804C092B24846614614
:1062E800FFF7F0F8B8F1000F04DA08EB860808F1B8
:1062F800060805E0F31B08F10A0808EB8308013FCC
:1063080001360135BE42ADB28FD905B0BDE8F08F78
:10631800BC1A002008B9FFF713B8012801D1FFF70C
:106328000BB87047704700200146F0224FF4A07365
:10633800FFF7C8B9704708B505280CD8DFE800F0A2
:10634800121403050709094808BD094808BD09488A
:1063580008BD094808BD0948094A0A4B40F24111DD
:10636800FEF724FD084808BD084808BD880100203C
:10637800780100207001002068010020CAB40508D7
:1063880086AF040805B305089001002080010020AD
:1063980010B50446FFF7CFFF014B18601C7110BD04
:1063A800A0010020014B1879704700BFA001002010
:1063B80008B5FFF7C0FF808808BD08B5FFF7BBFF29
:1063C800C08808BDF7B51F460B4B0C4E1D68144618
:1063D800EA882B68203C5443A4B2AE1B03EB440468
:1063E80018BF0126AB888DE8500017B1FFF7EEF90A
:1063F80001E0FFF771FAFEBDA00100209001002026
:106408002DE9F0410F46984615460446084E08E027
:10641800204643463946FFF7D5FF33689B88E41882
:10642800A4B215F8012B002AF2D1BDE8F08100BF13
:10643800A001002010B5044608462146BDE81040DA
:10644800DEE7094B70B5044618790E461546FFF786
:10645800B4FFC6F1F001091A89B220462A46002382
:10646800BDE87040CCE700BFA0010020704700BF26
:10647800044B1A680AB9044A1A601A681018186096
:1064880010467047400D0020843D00204FF0FF303B
:10649800704708B50248034A034B3721FEF786FCCC
:1064A800E9B405089CAF040805B305080120704746
:1064B80010B504460A4802210BF0AEF80028F9D0BE
:1064C800074821460BF071F8054801210BF0A4F8A4
:1064D8000028F9D00248BDE810400BF063B800BFAF
:1064E8000038004010B5194802210BF095F8002833
:1064F800F9D0164800210BF058F8144801210BF088
:106508008BF80028F9D011480BF04CF80402A4B21B
:10651800002301E001339BB2002BFBD00B48022182
:106528000BF07AF80028F9D0084800210BF03DF864
:10653800064801210BF070F80028F9D003480BF049
:1065480031F82043C0F3CB0010BD00BF0038004035
:106558002DE9F0478AB00AAF0A2001210AF0D6FDDA
:106568004FF4604347F8143D474EDFF824A1012457
:1065780000254FF00208304639468DF81A508DF83C
:1065880018808DF819808DF81B400AF017FA3046EC
:106598000D2105220AF092FA30460E2105220AF052
:1065A8008DFA052230460F210AF088FA21464FF469
:1065B80080400AF0CFFD50460AF0AAFE4FF48273DD
:1065C800ADF802304FF40073ADF80A303823ADF857
:1065D8000C30504607236946ADF81030ADF800502E
:1065E800ADF80450ADF80650ADF80850ADF80E50AF
:1065F8000AF0C0FE504621460AF057FFA9468DF81A
:106608001A5030464FF48055394605958DF8184094
:106618008DF819808DF81B400AF0D0F930462946CC
:106628000AF03DFA4025394618488DF818908DF83B
:1066380019808DF81A908DF81B4005950AF0BEF95F
:1066480021464FF480400AF091FD062103200BF00B
:106658001BF80C2307A88DF8213007958DF820909A
:106668008DF8224009F09EFE17238DF8243009A8E2
:106678000F238DF825308DF826308DF8274002F04D
:106688003BFF0AB0BDE8F08700040240000C02405E
:1066980000380040014B1878704700BF440D0020B7
:1066A800024B5A889B8802800B807047440D00205B
:1066B800014B00221A707047440D0020F0B593B0CA
:1066C80068460021482210F031FF6D4600246448D6
:1066D8004FF480510AF0E5F9002301E001339BB241
:1066E800002BFBD09020FFF7E3FE002301E00133ED
:1066F8009BB2002BFBD0FFF7F5FE4FF48051074605
:1067080057480AF0CCF9002301E001339BB2002B73
:10671800FBD053484FF480510AF0C3F9002301E03D
:1067280001339BB2002BFBD0D020FFF7C1FE002322
:1067380001E001339BB2002BFBD0FFF7D3FE4FF4EF
:106748008051064646480AF0AAF945F8047B013408
:106758002E6244484021E4B20AF08FF910B9092C9E
:10676800B5D101E0092C78D19DE80C00D218029B24
:1067780003980699D218049BC018059BC018079B5C
:10678800CB180899032490FBF4F092FBF4F25B1801
:1067980093FBF4F3151AC11A9C1A002DB8BF6D4269
:1067A8000029B8BF4942002CB8BF6442502D03DD10
:1067B800502909DD502C50DC8D4205DAAC424FF0EF
:1067C800020405DB111806E08C424FF0020401DADE
:1067D800D11800E0C1180A9B099A0C980F9DD2188D
:1067E8000B9BD2180D9BC0180E9BC018109BEB1862
:1067F800119D91FBF4F1032492FBF4F290FBF4F069
:106808005B1993FBF4F3161AC41A9D1A002EB8BF2D
:106818007642002CB8BF6442002DB8BF6D42502E9E
:1068280089B203DD502C09DD502D16DCA64205DAAD
:10683800B5424FF0020405DB131806E0A5424FF0FD
:10684800020401DAD31800E0C318074A93FBF4F3F3
:106858009BB2938001235180137013B0F0BD00BF29
:1068680000040240000C0240440D0020000000001B
:10687800FFF710BFF7B505460C4601A80DF1060154
:10688800FFF70EFF1B4BBDF80660BDF8040093E848
:106898000600724301FB002299685218164992FBC0
:1068A800F1F207EE102AF8EEC77A40F23F17FCEE35
:1068B800E77A17EE902A92B2B2F5207F28BF3A46BF
:1068C8002A801D69DA685B696E4302FB0060C018A4
:1068D80090FBF1F107EE101AF8EEC77AFCEEE77AB2
:1068E80017EE903A9BB2B3F5F07F28BFEF232380D1
:1068F800FEBD00BF4C0D002040420F00FFF7D8BE80
:10690800014B187E704700BF4C0D0020FFF7C8BE32
:10691800042808B505D90748074A084B7D21FEF722
:1069280045FA054B03EB8000038B0B80438B1380E8
:1069380008BD00BF0AB50508A2AF040828B50508B8
:1069480008B5082001F0BAF942F69643C31A58422E
:1069580040EB030008BD10B50A2001F0D7F90C4C34
:1069680020600E2001F0D2F96060122001F0CEF90B
:10697800A060162001F0CAF9E0601A2001F0C6F9FB
:1069880020611E2001F0C2F901236061237610BD49
:106998004C0D002010B5FFF7DBFD01F06DFA044641
:1069A80001F076FA074903462246202009F014F838
:1069B800FFF7C6FF28B101F079FA10B9BDE8104019
:1069C800C9E710BD64B5050810B5104C0A20216848
:1069D80001F083F961680E2001F07FF9A1681220A7
:1069E80001F07BF9E168162001F077F921691A2096
:1069F80001F073F961691E2001F06FF9082042F671
:106A08009641BDE8104001F04BB900BF4C0D002085
:106A18002DE9F04F0346A7B0B0F800C01C8986885E
:106A2800DF885D89CDF810C0B249B0F802C0B3F86C
:106A38000C90B3F80E80CDF824C00FFA84FB30B266
:106A480001220FFA87FE0BEB000C0A7629B20FFA27
:106A580089FACDF888C001EB0E0C0FFA88F2CDF850
:106A680090C00AEB0B0CCDF830C002EB010CCDF84E
:106A780058C0B3F810C05B8ACDF800C00FFA8CFC80
:106A880006910CEB00010A9102930CEB0A011BB270
:106A9800239103EB0E010E9199182591049900FAA0
:106AA80081F0584450446044DDF824C006990EFA39
:106AB8008CFEDDF810C01FFA80FB1CFB0CF08E4426
:106AC80016FB0600964414FB0400009A19FB090003
:106AD8009E4412FB02001FFA8EFA0BF0A7FEDDF8A7
:106AE80024C0029ACDE912011CFB0CF017FB070029
:106AF80015FB050018FB080012FB02000BF096FEC0
:106B0800DDF824C0029ACDE9140104991CFB01F3B5
:106B180017FB063615FB0466009B18FB096612FB7B
:106B280003600BF083FEDDE91423CDE90001DDE904
:106B380012010BF0F1FE04460D46DDE900010246A4
:106B48000B460BF0E9FE02460B46204629460BF0A1
:106B58002FFDCDE9180158460BF078FECDE910015C
:106B6800DDE91023DDE900010BF0D6FECDE90601D1
:106B780050460BF06BFE804689464246DDE912011D
:106B88004B460BF0C9FEDDE91023CDE91C01DDE918
:106B980014010BF0C1FE002206460F46564BDDE9F4
:106BA80018010BF0B9FE424604460D464B46DDE996
:106BB80006010BF0B1FE02460B460BF0FBFC024649
:106BC8000B46204629460BF0F5FC424604460D4686
:106BD8004B46DDE91C010BF09FFE02460B462046A2
:106BE80029460BF0E5FCDDE9102304460D46304646
:106BF80039460BF091FE02460B46204629460BF01B
:106C0800D7FCDDF828C0CDE902014FEA8C10DDF889
:106C180030C000EB0C20DDF810C0A0241CFB0400E1
:106C28000BF004FEDDF838C0CDE90A014FEA8C10FC
:106C3800DDF858C000EB0C20DDF824C01CFB040074
:106C48000BF0F4FDCDE90C0150460BF0EFFDDDE94A
:106C58001023CDE91601DDE90C010BF05DFE42467B
:106C6800CDE91E014B46DDE90A010BF055FE42460F
:106C7800CDE920014B46DDE900010BF04DFE32461F
:106C88003B460BF095FCCDE90E0158460BF0CEFDC6
:106C9800DDE91C23CDE91A01DDE906010BF088FCCA
:106CA800DDF88CC0C024CDE9060104FB0CF0DDF84A
:106CB80088C0302505FB0C00DDF810C078261CFBC9
:106CC80006000BF0B3FDDDF894C0824604FB0CF01F
:106CD800DDF890C005FB0C00DDF824C01CFB0600A5
:106CE8008B460BF0A3FDDDE9102306460F460BF09B
:106CF80013FE03E04C0D0020000014404246CDE98D
:106D080004014B46504659460BF006FEDDE91423B4
:106D180080468946DDE90A010BF0FEFDDDE9002326
:106D280004460D46DDE90C010BF0F6FD02460B4664
:106D3800204629460BF03CFC0022A14B0BF0ECFD51
:106D4800DDE9202304460D46DDE91E010BF030FC89
:106D580002460B46DDE916010BF0DEFD02460B4646
:106D6800204629460BF026FC002204460D46954B8A
:106D7800DDE90E010BF0D0FD02460B462046294600
:106D88000BF018FCDDE902230BF0F0FE88A3D3E931
:106D980000230BF0C1FD0CF059F88B490860DDE9C0
:106DA8001223DDE90C010BF0B7FDDDE900230446F1
:106DB8000D46DDE90A010BF0AFFD02460B46204601
:106DC80029460BF0F5FB00227D4B0BF0A5FDDDE914
:106DD8001E2304460D46DDE920010BF0E9FB0246BF
:106DE8000B46DDE91A010BF097FD02460B462046DB
:106DF80029460BF0DFFB002204460D46714BDDE906
:106E080006010BF089FD02460B46204629460BF089
:106E1800D1FBDDE902230BF0A9FE65A3D3E900232A
:106E28000BF07AFD0CF012F8674A5060DDE90E238A
:106E3800DDE90A010BF070FDDDE9062304460D4685
:106E4800DDE90C010BF068FD02460B462046294699
:106E58000BF0B0FB002204460D465A4BDDE9180141
:106E68000BF05AFD02460B46204629460BF0A2FBC2
:106E7800DDE902230BF07AFE4DA3D3E900230BF0E2
:106E88004BFD0BF0E3FF504B59469860DDE91423A6
:106E980050460BF041FDDDE9002304460D4630461F
:106EA80039460BF039FD02460B46204629460BF0C1
:106EB8007FFB0022424B0BF02FFD424604460D4655
:106EC8004B46DDE904010BF073FB02460B46DDE996
:106ED80016010BF021FD02460B46204629460BF011
:106EE80069FB35A3D3E9002304460D46DDE90E010D
:106EF8000BF012FD02460B46204629460BF05AFBC2
:106F0800DDE902230BF032FE29A3D3E900230BF0BD
:106F180003FD0BF09BFFDFF8B0C0DDE91223CCF8CE
:106F28000C00394630460BF0F7FCDDE90023044637
:106F38000D46504659460BF0EFFC02460B462046DC
:106F480029460BF035FB00221D4B0BF0E5FCDDE973
:106F5800042304460D46404649460BF029FB0246E9
:106F68000B46DDE91A010BF0D7FC02460B4620461A
:106F780029460BF01FFB10A3D3E9002304460D4656
:106F8800DDE906010BF0C8FC02460B4620462946FF
:106F98000BF010FBDDE902230BF0E8FD04A3D3E9B5
:106FA80000230BF0B9FC0BF051FF074908610DE015
:106FB8000000000080842E410000000000C08240D4
:106FC80000001440000089404C0D0020DDE90E232C
:106FD800504659460BF0A0FCDDE9062304460D4651
:106FE800304639460BF098FC02460B4620462946A7
:106FF8000BF0E0FA11A3D3E9002304460D46DDE9BE
:1070080018010BF089FC02460B46204629460BF076
:10701800D1FADDE902230BF0A9FD0AA3D3E9002385
:107028000BF07AFC0BF012FF034A506127B0BDE861
:10703800F04FC9E4AFF300804C0D002000000000C1
:1070480000C082400000000080842E41AFF3008021
:10705800064A074B1A60074A074B1A60074A084B4B
:107068001A60084B64221A60704700BF40420F0044
:10707800F026002080C3C901082D0020A086010049
:10708800E42C00209C260020012808B503D05AD300
:10709800022851D13CE02C4B1B78012B03D013D391
:1070A800022B49D121E0294BC820196800F015FEB0
:1070B800274BCC20196800F010FE264BD020196809
:1070C80000F00BFED42033E0204BD820196800F0E4
:1070D80004FE1F4BDC20196800F0FFFD1D4BE0206B
:1070E800196800F0FAFDE42022E0184BF82019682E
:1070F80000F0F3FD164BFC20196800F0EEFD154B6F
:107108004FF48070196800F0E8FD4FF482700FE0CA
:107118000E4BE820196800F0E0FD0D4BEC201968D3
:1071280000F0DBFD0B4BF020196800F0D6FDF420D1
:10713800094B196800F0D1FD04F0F2FE18B9BDE85A
:10714800084004F0FEBE08BD1C0E0020F0260020FA
:10715800082D0020E42C00209C26002008B52E4B8A
:107168001B78012B02D0022B55D140E02B4B1B780A
:10717800012B03D013D3022B4DD121E0C82000F0FE
:10718800C5FD274B1860CC2000F0C0FD254B1860CA
:10719800D02000F0BBFD244B1860D42022E0D8207A
:1071A80000F0B4FD1E4B1860DC2000F0AFFD1D4B55
:1071B8001860E02000F0AAFD1B4B1860E42011E0E5
:1071C800F82000F0A3FD164B1860FC2000F09EFD8F
:1071D800144B18604FF4807000F098FD124B186043
:1071E8004FF4827000F092FD104B186008BDE82043
:1071F80000F08CFD0A4B1860EC2000F087FD094B6D
:107208001860F02000F082FD074B1860F42000F0B1
:107218007DFD064B186008BDC90100201C0E00202A
:10722800F0260020082D0020E42C00209C260020B9
:1072380008B504F075FE10B1BDE808408EE7BDE85A
:10724800084005E7064B07495960C021002219721A
:107258001E211A70D9601A745A611A76DA61704759
:10726800EC1A002040787D0110B50321FF22C020D0
:1072780001F02AFC1F4C102180222060C02001F060
:1072880023FC112180222060C02001F01DFC122166
:1072980080222060C02001F017FC1321802220608A
:1072A800C02001F011FC142180222060C02001F0D0
:1072B8000BFC152180222060C02001F005FC8022F3
:1072C80020601621C02001F0FFFB2060C02017219C
:1072D800802201F0F9FB80222060B721C02001F054
:1072E800F3FB054B00221A745A611A76DA610122FF
:1072F8001A7010BDC4260020EC1A002038B5C02032
:107308000321FF2201F0E0FB0B4D00242B19615DE6
:107318005A78C020023401F0D7FBC82CF6D1B1212D
:10732800AC22C02001F0D0FBC0200321002201F0D4
:10733800CBFB002038BD00BFCEAF04082DE9F347D2
:1073480006460F4692461D461AB90C1FE40191469F
:1073580035E005EE902A06EE903AB8EE657AF8EE3A
:10736800667AFC01C7EE277AA4F500749FED5C7A73
:1073780067EE877A17EE900A0BF07AFA41EC100B59
:107388000DF0F2FB59EC108B494640460BF086FD98
:1073980024184FEACA100BF049FACDE90001284633
:1073A8000BF044FA4B4642460BF0B6FA02460B463F
:1073B800DDE900010BF0FCF80BF070FD8146002EB2
:1073C80014BF4FF022084FF01A08C5F307224146B0
:1073D800C02001F079FB08F10101EAB2C02001F0F8
:1073E80073FBC4F3014208F10201C02001F06CFBF9
:1073F800C4F3072208F10301C02001F065FBE2B2E3
:1074080008F10401C02001F05FFBC9F3034305F450
:10741800702243EA123208F10501C02001F054FB42
:1074280008F10601C9F30722C02001F04DFB08F15D
:1074380007015FFA89F2C02001F046FBC020B121A4
:10744800A02201F041FB07EE107A264CF8EEC77A2D
:107458000EBBD4ED015A06EE90AAB8EE657A05EE99
:10746800905AB8EE666AF8EE656A0123C6EE266A97
:10747800237477EEA67A67EE277A17EE900A0BF058
:10748800F7F941EC100B0DF06FFB51EC100B0BF002
:1074980005FD606120E005EE90AAD4ED016AB8EE22
:1074A800656A05EE905AB8EE667AF8EE656A0123C9
:1074B800C6EE266A237677EEA67A67EE277A17EE67
:1074C800900A0BF0D5F941EC100B0DF04DFB51EC87
:1074D800100B0BF0E3FCE0610020BDE8FC8700BF67
:1074E80000000043EC1A00200022012326E70128AF
:1074F80038B50D4604D002280CBF3C242C2400E0EB
:1075080034242146C02001F059FB05F0070200F0A1
:107518000F0040EA02122146C020BDE8384001F0C1
:10752800D3BA2DE9F3470A9C1D4607468A461646F4
:10753800524B01E06D0864089C42FBD82DB906F156
:107548000076043EF601A94634E006EE905AB8EEFD
:10755800667A06EE904AF8EE667AF601C7EE277A62
:10756800A6F500769FED467A67EE877A17EE900AC1
:107578000BF07EF941EC100B0DF0F6FA59EC108B7C
:10758800494640460BF08AFC3618E8010BF04EF9E4
:10759800CDE9000120460BF049F94B4642460BF075
:1075A800BBF902460B46DDE900010BF001F80BF0D0
:1075B80075FC8146022F9BBF324BDB194FF0000848
:1075C80093F8C880C4F307224146C02001F07CFA32
:1075D80008F10101E2B2C9B2C02001F075FA08F160
:1075E8000201C9B2C6F30142C02001F06DFA08F1E8
:1075F8000301C9B2C6F30722C02001F065FA08F1F9
:107608000401C9B2F2B2C02001F05EFA04F4702499
:10761800C9F3034308F1050143EA1432C9B2C02093
:1076280001F052FA08F10601C9B2C9F30722C020D5
:1076380008F1070801F048FA5FFA89F25FFA88F161
:10764800C02001F041FABAF1010F0CBF2F220F221E
:107658000DB942F04002012F06D002D3022F0AD101
:1076680005E0C020102104E0C020112101E0C02065
:10767800122101F029FA0020BDE8FC87FFFF0F0066
:1076880000000043CEAF040807B501230093002390
:10769800FFF747FF0EBD00280CBFFF22002208B5E8
:1076A800C020032101F010FA002008BD08B5C02051
:1076B800B121AC2201F008FA002008BD08B5042069
:1076C800012109F023FD4FF480700121BDE8084035
:1076D80009F04CBD07B50223009303238DF804304D
:1076E8000348002369468DF8073009F067F90EBD95
:1076F8000008024030B5124D8BB0002406A806944D
:1077080007940894099408F027FB00948DF8044026
:107718008DF8054002940394049428460124694690
:107728008DF8144008F0E9FA28460B212246062372
:1077380008F05EFB2846214608F028FB0BB030BD58
:107748000020014010B5002104460122302001F03C
:10775800BBF9C0B9012001F0B1FC002CB8BF40341E
:10776800E4B210212246302001F0AEF9012001F0E8
:10777800A5FC30201121224601F0A6F90120BDE820
:10778800104001F09BBC10BD10B500210446012239
:10779800302001F099F9C0B9012001F08FFC002CCC
:1077A800B8BF4034E4B212212246302001F08CF9EF
:1077B800012001F083FC30201321224601F084F9D6
:1077C8000120BDE8104001F079BC10BD38B5012298
:1077D80005460C463020002101F076F9F0B9012069
:1077E80001F06CFC25EAE5725F2AA8BF5F223B2105
:1077F800D2B2302001F068F9012001F05FFC24EAE0
:10780800E4725F2AA8BF5F22D2B230203C2101F087
:107818005BF90120BDE8384001F050BC38BD302884
:1078280010B504460ADC10F17F0F02DB002802DBEA
:1078380005E06FF07E0404F5807400E03024002138
:1078480030200A4601F040F9A8B90120E4B201F05D
:1078580035FC41212246302001F036F9012001F0A3
:107868002DFC30204221224601F02EF90120BDE8EE
:10787800104001F023BC10BD282810B5044609DCCF
:1078880010F1180F02DB002802DB04E06FF0170488
:107898007F3400E02824002130200A4601F014F942
:1078A800A8B90120E4B201F009FC53212246302096
:1078B80001F00AF9012001F001FC30205421224690
:1078C80001F002F90120BDE8104001F0F7BB10BD3E
:1078D80008B530200021012201F0F6F860B9012036
:1078E80001F0ECFB30203321402201F0EDF80120BB
:1078F800BDE8084001F0E2BB08BD10B5302000210A
:10790800012201F0E1F8044660B9012001F0D6FB3C
:1079180030203321224601F0D7F80120BDE810407D
:1079280001F0CCBB10BD10B530200021012201F0C0
:10793800CBF80446A0B9012001F0C0FB342122464F
:10794800302001F0C1F8012001F0B8FB30203721C8
:10795800224601F0B9F80120BDE8104001F0AEBBA5
:1079680010BD4020EEE640200EE708B500210122B8
:10797800302001F0A9F8012001F0A0FB30203421CB
:10798800024601F0A1F8012001F098FB30203721D0
:10799800024601F099F80120BDE8084001F08EBBCD
:1079A80008B500210122302001F08EF8012001F0F5
:1079B80085FB302034210C2201F086F80120BDE837
:1079C800084001F07BBB00002DE9F04F984B994A25
:1079D8001968994B002914BF91469946974B2DED8C
:1079E800048BC3F80090964B0025002287B01A80BC
:1079F800AA46AB46A8465AE0A2004046CDF804C0C5
:107A080002920AF035FF0746584601F100460AF08F
:107A18002FFF02460B46384631460AF0C9FD39F9B0
:107A2800243007EE103AF8EEC77A064617EE900AA9
:107A38000F460AF01DFF02460B46304639460AF04B
:107A4800B9FD0BF04BFA074650460AF011FF044601
:107A5800284601F100460AF00BFFCDE90401DDE9F3
:107A68000423204631460AF0A3FD029A09EB0203DB
:107A78000446B3F9023007EE103AF8EEC77A0D461D
:107A880017EE900A0AF0F4FE02460B4620462946F5
:107A98000AF090FD0BF022FADDF804C0684A0CF1F8
:107AA800010CC3465546A2F800C08246B846644B4E
:107AB800B3F800C00FFA8CF4B32C9DDD58460AF0D9
:107AC800D7FECDE9020140460AF0D2FE0022064662
:107AD8000F465C4BDDE902010AF01EFF02460B4629
:107AE800304639460AF066FD0022574B0BF03EF847
:107AF8000BF0F4F94CA3D3E9002309EE900ADDE971
:107B080002010AF009FF00224F4B0BF02FF80BF08F
:107B1800E5F909EE100A28460AF0AAFE044650467E
:107B28000D460AF0A5FE002206460F4620462946C5
:107B3800444B0AF0F1FE02460B46304639460AF03D
:107B480039FD0022404B0BF011F80BF0C7F936A3B2
:107B5800D3E9002308EE900A294620460AF0DCFE05
:107B68000022394B0BF002F80BF0B8F908EE100AB6
:107B780069EE287A58EE297A17EE900A0AF078FE0C
:107B880068EE097A48EEA97A044617EE900A0D467F
:107B98000AF06EFE45EC104B41EC110B0DF0E8F8C5
:107BA80051EC100B0BF09AF928EE088A08EEA88A17
:107BB80007EE100A254B264CF1EE477AC3ED007A02
:107BC80018EE100A0AF054FE41EC100B0DF0DEF925
:107BD80029EE099A51EC100B09EEA99A0BF07EF9DF
:107BE800206019EE100A0AF043FE41EC100B0DF06C
:107BF800CDF951EC100B0BF071F9D4ED007A07EECA
:107C0800100A87EE877A134B1860134BFDEEE77A5C
:107C180083ED007A114BC3ED007A07B0BDEC048BFD
:107C2800BDE8F08FAFF30080912B50E67AB6EB3FBA
:107C3800141B002096230020F61D0020101B002096
:107C48001C1B00200000E03F000059400C2D0020C4
:107C5800242D0020182D0020142D0020181B002092
:107C680010B5084C204608F0F6FA074B1860FFF7E5
:107C7800ABFE064B0649012220461A80BDE810409B
:107C880008F06ABB10600240141B0020680D002039
:107C980020800010014B1868704700BF181B002097
:107CA80038B505460C460135C1F3072101F014FA31
:107CB800A8B2E1B201F010FA00B238BD38B50446F6
:107CC80001F044F801340546A0B201F03FF8EDB2E6
:107CD800C0B240EA052000B238BD37B50B0E8DF8AA
:107CE80004300B0C8DF805300B0A8DF806308DF832
:107CF8000710002400E0284601AB451CE15C013474
:107D080001F0EAF9042CADB2F5D13EBD37B5002437
:107D180000E02846451C01F019F801ABADB2E0546B
:107D28000134042CF5D19DF805009DF804300004B9
:107D380040EA03609DF8073018439DF8063040EA92
:107D480003203EBD37B500230193002400E02846F8
:107D5800451C00F0FBFF01ABADB2E0540134042C2C
:107D6800F5D19DED010A3EBD7047000038B50446C7
:107D7800642001F0A3F925786068AD00EDB22570A4
:107D880008F081FE237A40FA03F000F0030005436F
:107D9800104B257005F00F055A5D6378D218D2B2E2
:107DA800D3B20132D2B2022A637001D80022A27083
:107DB8005BB2012B03DD0123A3700023637094F9E8
:107DC8000130013303DAFF23A3700023637094F9B1
:107DD800020038BD9AB00408F7B504200121234FEA
:107DE80009F094F902AD01214FF48040012409F013
:107DF800BDF900264FF4B0733846694645F8083D8A
:107E08008DF804608DF8074008F0D8FD1020214651
:107E180009F07CF978236946154800938DF80460C9
:107E28008DF8074008F0CAFD0420214609F06EF9D4
:107E380021464FF4804009F099F91C2338466946D9
:107E480000938DF804608DF8074008F0B7FD022014
:107E5800214609F05BF9B02306488DF804606946AD
:107E68008DF80740009308F0A9FDFEBD0008024008
:107E78000010024000040240802108B5034808F0C1
:107E8800FCFDD0F1010038BF002008BD000402400D
:107E980008B54FF48071044808F0EFFDD0F10100F7
:107EA80038BF002008BD00BF0008024008B5FFF732
:107EB800E3FF08B1FFF7ECFFC0B208BD70B50028BA
:107EC8003AD01E4B1A7880181D4AC0B292F9002089
:107ED800187040B282421B4A02DD117801391970CC
:107EE80093F9001092F9002091FBF2F402FB1414AC
:107EF8001549E4B21C700A88144B1A80144B154AB1
:107F080018881080144A92F9000064B2013094FB7A
:107F1800F0F200FB1240114C2688114C258800FB1A
:107F2800065008800F4908880F49098802FB00128B
:107F38001A800E4B01221A7070BD00BFBE3A002095
:107F4800E9360020C4360020F43A00200A37002021
:107F5800BC3A0020BC380020F63A0020183800202F
:107F6800583B0020843B00209A380020BC36002073
:107F7800F0B5264A264C00231370264A2568167841
:107F8800254A12680FE0D45C2F197F7817F0040F88
:107F980007D0302C02D12023135431E01B4A137030
:107FA80003E00133DBB29E42EDDA184B1B788342C3
:107FB800194B16D9A9B11A68164C31211154302120
:107FC8000BE01A681518125C2E2A19D0303AD2B272
:107FD800092A88BF29700130C0B222788242F0DABB
:107FE8000EE01B681A5C79B12E2A0DD05118C9B25F
:107FF800392903D82F2998BF302100E03921195495
:10800800BDE8F040FCF7AABCF0BD00BF6C0D002035
:1080180048030020783C0020E03A002010B5642096
:1080280001F04CF88648FFF7A1FE864B1B78044602
:108038000C2B00F26981DFE813F00D000D006701D9
:108048007500750037008C008E00BE00C100DB0093
:108058008E004301FFF71CFF18B10120F9F758FD06
:1080680052E1794B1888794B1B88C01A784B1B88CA
:1080780090FBF3F0774B1A88774B1B88D31A774A13
:10808800128893FBF2F3DBB2C0B2032B00F2D38069
:10809800DFE803F002040608714A40E0714A3EE056
:1080A800714A3CE0714A3AE0FFF7F2FED8B100218C
:1080B8000A226F4810F00AFC6E4B002118600A2251
:1080C8006D4810F003FC6D4B18600420FEF760F952
:1080D800962005216A4A0023FEF792F90020FEF750
:1080E80057F907F0E1F8584B1888584B1B88C01A05
:1080F800574B1B8890FBF3F0564B1A88564B1B883E
:10810800D31A564A128893FBF2F3DBB2C0B21BB102
:10811800012B40F0908001E0554A00E0564A594B47
:108128001A6088E0002800F0EF80574B1A7806DDC7
:108138000132D2B2102A1A7008D9112205E0013A88
:10814800D2B2112A1A7001D900221A70F9F7CCFE9E
:10815800DAE04E4B1870002C00F0D6804C4B1B78A0
:10816800022B40F0D1804B4B1A78A418E4B20322BA
:10817800B4FBF2F102FB1144E4B21C70464B474ACF
:108188001B5D022B137009D0052B0CD0012B40F07E
:10819800BB804FF491706921414A08E04FF4917017
:1081A8006921404A03E0404A4FF491706921002355
:1081B800FEF726F9A8E0354B1870A5E0FFF768FE32
:1081C800A0B10021394810F0CDFA394B042083EDD5
:1081D800000AFEF7DDF8B4200521364A0023FEF731
:1081E8000FF9FAF78DFA0020FEF7D2F82F4A16E0B9
:1081F800FFF74EFE90B100212F4810F0B3FA2F4B35
:10820800042083ED000AFEF7C3F896200521294AC9
:108218000023FEF7F5F80020FEF7BAF8264A194BB6
:108228001A60094B1888094B1B88C01A084B1B8811
:1082380090FBF3F0C0B22146FFF79AFE64E000BF5E
:10824800A801002071260020F43A0020583B0020A5
:1082580018380020BC3A00209A380020843B0020BF
:10826800B4260020D8260020EE2C0020A0260020CE
:10827800603B0020C4010020D03A0020C00100204B
:108288009FB50508E03A0020EA260020EC3A0020D5
:10829800E4380020D50D0020300300201C03002006
:1082A800AFB50508B2B50508B5B50508DC36002038
:1082B80024030020B8B5050800370020200300205B
:1082C800FFF7E6FD08B107F0C7F914B1264B012204
:1082D8001A70264B1A68A41814F5967FB8BF244A5A
:1082E8001C60B8BF1A601B68B3F5967F03DD1F4B8F
:1082F8004FF496721A601C4C23782BB11D4B1868EA
:1083080001F0DCFA002323701B48FFF72FFD1B4BFD
:108318001B78013B0C2B25D8DFE803F00724242425
:1083280021161624121216241600FFF7C7FDFFF7B0
:10833800A3FD002816D00220BDE81040F9F7E8BBDD
:108348000F4B1B78022B0AD100280E4B01D1187055
:1083580010BD01DD012200E0FF221A7010BDBDE84A
:108368001040ABE510BD00BFEC260020F03A00201D
:10837800D4FEFFFF90260020B401002071260020C3
:10838800E4380020251B002010B58CB01E490F22B0
:1083980068460FF089F81D490F2204A80FF084F8E9
:1083A8001B490F2208A80FF07FF80021082230206F
:1083B80000F08AFB012000F081FE002404AB1DF8C8
:1083C8000420E15C302000F07FFB0134012000F044
:1083D80075FE0F2CF2D100210922302000F074FB29
:1083E800012000F06BFE002408AB1DF80420E15CBE
:1083F800302000F069FB0134012000F05FFE0F2CF3
:10840800F2D10CB010BD00BFACB00408BBB004087A
:10841800CAB0040810B58CB01E490F2268460FF088
:1084280043F81D490F2204A80FF03EF81B490F22FC
:1084380008A80FF039F800210822302000F044FB8A
:10844800012000F03BFE002404AB1DF80420E15C91
:10845800302000F039FB0134012000F02FFE0F2CF2
:10846800F2D100210922302000F02EFB012000F07B
:1084780025FE002408AB1DF80420E15C302000F044
:1084880023FB0134012000F019FE0F2CF2D10CB0AF
:1084980010BD00BFD9B00408E8B00408F7B004085C
:1084A80010B58CB01E490F2268460EF0FDFF1D491D
:1084B8000F2204A80EF0F8FF1B490F2208A80EF09F
:1084C800F3FF00210822302000F0FEFA012000F01E
:1084D800F5FD002404AB1DF80420E15C302000F019
:1084E800F3FA0134012000F0E9FD0F2CF2D100214C
:1084F8000922302000F0E8FA012000F0DFFD002416
:1085080008AB1DF80420E15C302000F0DDFA0134EE
:10851800012000F0D3FD0F2CF2D10CB010BD00BF2C
:1085280006B1040815B1040824B1040807B50220EF
:10853800012108F0EBFD012300938DF8043002239C
:108548008DF805300448002369468DF806308DF80B
:10855800073008F033FA0EBD0004024010B5084C8D
:1085680001210022204608F09EFA40F2FF4000F068
:10857800A5FD012120460A46BDE8104008F093BA3F
:108588000004024008B5FFF7E9FF00210A46302041
:1085980000F09AFA012000F091FD01210A463020EE
:1085A80000F092FA012000F089FD0021012230201C
:1085B80000F08AFA012000F081FD01210822302014
:1085C80000F082FA012000F079FD0221012230201A
:1085D80000F07AFA012000F071FD00210A463020EF
:1085E80000F072FA012000F069FD1B21CD22302035
:1085F80000F06AFA012000F061FD04210322302016
:1086080000F062FA012000F059FD0621092230200D
:1086180000F05AFA012000F051FD0721082230200D
:1086280000F052FA012000F049FD082170223020A4
:1086380000F04AFA012000F041FD1E213020B0224E
:1086480000F042FA012000F039FD05219122302086
:1086580000F03AFA012000F031FD0D21032230200C
:1086680000F032FA012000F029FD0E21002230200E
:1086780000F02AFA012000F021FD14218022302088
:1086880000F022FA012000F019FD0B218822302089
:1086980000F01AFA012000F011FD0C21822230208E
:1086A80000F012FA012000F009FD12218822302082
:1086B80000F00AFA012000F001FD13218C2230207D
:1086C80000F002FA012000F0F9FC00210A463020EF
:1086D80000F0FAF9012000F0F1FC3D2102223020DF
:1086E80000F0F2F9012000F0E9FCFFF74DFEFFF77A
:1086F80091FEFFF7D5FE30200021012200F0E4F9B9
:10870800012000F0DBFC3D216422302000F0DCF980
:10871800012000F0D3FC03210022302000F0D4F91E
:10872800012000F0CBFC04210022302000F0CCF91D
:10873800012000F0C3FC00210122302000F0C4F920
:10874800012000F0BBFC0C210822302000F0BCF90D
:10875800012000F0B3FC0D210822302000F0B4F90C
:10876800012000F0ABFC0E210822302000F0ACF90B
:10877800012000F0A3FC0F210822302000F0A4F90A
:10878800012000F09BFC00210A46302000F09CF9F3
:10879800012000F093FC02224021302000F094F9DF
:1087A800012000F08BFC30204121002200F08CF9E0
:1087B800012000F083FC3F21D422302000F084F90E
:1087C800012000F07BFC00210122302000F07CF920
:1087D800012000F073FC10210F22302000F074F902
:1087E800012000F06BFC11210F22302000F06CF901
:1087F800012000F063FC12210022302000F064F90F
:10880800012000F05BFC13210022302000F05CF90D
:10881800012000F053FC09213C22302000F054F9DB
:10882800012000F04BFC00210122302000F04CF91F
:10883800012000F043FC30203421024600F044F9C6
:10884800012000F03BFC30203721024600F03CF9C3
:10885800012000F033FC36210322302000F034F9E7
:10886800012000F02BFC39210322302000F02CF9E4
:10887800012000F023FC3B213C22302000F024F9A9
:10888800012000F01BFC3C210A46302000F01CF9B6
:10889800012000F013FC00210A46302000F014F9F2
:1088A800012000F00BFC5121C022302000F00CF90F
:1088B800012000F003FC52213020002200F004F9CE
:1088C8000120BDE8084000F0F9BB00BF2DE9F04FDA
:1088D800454E464D93B001214FF4001008F016FCA8
:1088E800304607F0B9FB4FF0C0630293404B039347
:1088F800404B002404934FF4B4794FF400334FF401
:1089080080684FF400674FF4005A4FF4807B30467C
:1089180002A90C9301930997CDF818900594079430
:10892800CDF82080CDF828A0CDF82CB00D9407F014
:108938001FFC22463046304907F075FC30460121BD
:1089480007F07BFC01210A464FF0402008F04CFE5E
:10895800284607F081FB294A019B0392284A0C9379
:1089680004922846402202A9059209970294CDF85C
:1089780018900794CDF82080CDF828A0CDF82CB019
:108988000D9407F0F5FB224628461E4907F04BFCDC
:108998002846012107F051FC42F2107701220221FA
:1089A800194808F021FE384600F088FB30460121BE
:1089B80007F019FC0121284607F015FC384600F09D
:1089C8007DFB0B238DF8443011A801238DF8454019
:1089D8008DF846408DF8473000F08EFD384600F09F
:1089E8006DFB13B0BDE8F08F106002408860024054
:1089F8000C40004096230020F61D00200C3C00404F
:108A0800C6200020261B0020003C00400248102100
:108A1800012207F05FBC00BF1060024013B50220BE
:108A2800012108F073FB4FF410730E4C00930223DE
:108A38008DF804308DF8053001238DF80630204676
:108A4800002369468DF8073007F0B8FF2046062155
:108A5800042208F033F820460921042208F02EF8F1
:108A68001CBD00BF0004024030B5154D85B0012182
:108A78004FF4001008F06EFB284608F035F8002384
:108A8800ADF804304BF6FF73ADF806303323ADF87C
:108A980008304FF48063ADF80A304FF48043ADF8E6
:108AA8000C3004AC074B2846012144F8103D08F06F
:108AB800BDF82846694608F045F805B030BD00BF46
:108AC80000540040801A060073B54FF4961306460A
:108AD8000D461446019304E0019B5A1E0192002B97
:108AE80057D031484FF4003108F0B8F90028F3D1D5
:108AF8002D48012108F0A6F84FF48053019304E0B3
:108B0800019B5A1E0192002B45D02748274908F09F
:108B180090F90028F4D024483146002208F0AAF839
:108B28004FF48053019304E0019B5A1E0192002BDD
:108B380033D01D481E4908F07CF90028F4D01A48A3
:108B4800294608F01AF94FF48053019303E0019B7A
:108B58005A1E01921BB31448164908F06AF90028F6
:108B6800F5D01148214608F008F94FF496130193FF
:108B780003E0019B5A1E01929BB10B480E4908F075
:108B88006DF90028F5D00848012108F067F80020A1
:108B980008E0012006E0022004E0032002E00420AF
:108BA80000E005207CBD00BF005400400100030028
:108BB80082000700800007000400001037B54FF45A
:108BC800961304460D46019305E0019B5A1E019237
:108BD800002B00F09B8056484FF4003108F03EF916
:108BE8000028F2D15248012108F02CF84FF48053A4
:108BF800019305E0019B5A1E0192002B00F088802A
:108C08004B484C4908F015F90028F3D0484821464C
:108C1800002208F02FF84FF48053019304E0019BE1
:108C28005A1E0192002B75D04148434908F001F9BA
:108C38000028F4D03E48294608F09FF84FF48053A6
:108C4800019304E0019B5A1E0192002B64D038481E
:108C58003A4908F003F90028F4D03548012107F013
:108C6800F1FF4FF48053019304E0019B5A1E0192D7
:108C7800002B53D02E482F4908F0DBF80028F4D0F9
:108C88002B482146012207F0F5FF4FF4805301934A
:108C980004E0019B5A1E0192002B41D0244C284924
:108CA800204608F0DBF80028F3D02046002107F022
:108CB800E9FF20460121238B07F0D0FF4FF48053B2
:108CC800019304E0019B5A1E0192002B2AD01848F8
:108CD8001C4908F0C3F80028F4D0154808F04FF8EC
:108CE8004FF480530193124A03E0019B591E0191EE
:108CF800D3B113889B05F8D4012104460C4807F02A
:108D0800C1FF0B48104908F0C3F80EE001240CE03D
:108D180002240AE0032408E0042406E0052404E011
:108D2800062402E0072400E0082420463EBD00BFD8
:108D380000540040010003008200070004000010F6
:108D480002000010400000100004001013B54FF49A
:108D580096130446019305E0019B5A1E0192002BCD
:108D680000F0AF8060484FF4003108F077F8002831
:108D7800F2D15D48012107F065FF4FF4805301935C
:108D880005E0019B5A1E0192002B00F09C8056487A
:108D9800564908F04EF80028F3D05348A021002285
:108DA80007F068FF4FF48053019305E0019B5A1EBA
:108DB8000192002B00F089804B484D4908F039F8A2
:108DC8000028F3D0210A484807F0D7FF4FF4805312
:108DD800019304E0019B5A1E0192002B77D0424870
:108DE800444908F03BF80028F4D0E1B23E4807F0C7
:108DF800C4FF4FF48053019304E0019B5A1E019273
:108E0800002B66D038483B4908F028F80028F4D0F1
:108E18003548012107F016FF4FF48053019304E011
:108E2800019B5A1E0192002B55D02F482F4908F05C
:108E380000F80028F4D02C48A121012207F01AFFDD
:108E48004FF48053019304E0019B5A1E0192002BBA
:108E580043D0254C2849204608F000F80028F3D0D4
:108E68002046002107F00EFF20460121238B07F042
:108E7800F5FE4FF48053019304E0019B5A1E0192C2
:108E8800002B2CD018481D4907F0E8FF0028F4D023
:108E9800154807F074FF4FF480530193124A03E01A
:108EA800019B591E0191E3B113889905F8D401215A
:108EB80004460D4807F0E6FE0B48114907F0E8FFA5
:108EC80010E001240EE002240CE003240AE004244C
:108ED80008E0052406E0062404E0072402E008244C
:108EE80000E0092420461CBD005400400100030096
:108EF800820007000400001002000010400000106B
:108F08000004001013B54FF496130446019305E0CE
:108F1800019B5A1E0192002B00F0AF8060484FF46D
:108F2800003107F09BFF0028F2D15D48012107F0CE
:108F380089FE4FF48053019305E0019B5A1E01926C
:108F4800002B00F09C805648564907F072FF002815
:108F5800F3D05348A021002207F08CFE4FF4805331
:108F6800019305E0019B5A1E0192002B00F08980B5
:108F78004B484D4907F05DFF0028F3D0210A4848C7
:108F880007F0FBFE4FF48053019304E0019B5A1E47
:108F98000192002B77D04248444907F05FFF002830
:108FA800F4D0E1B23E4807F0E8FE4FF48053019355
:108FB80004E0019B5A1E0192002B66D038483B49B9
:108FC80007F04CFF0028F4D03548012107F03AFE9D
:108FD8004FF48053019304E0019B5A1E0192002B29
:108FE80055D02F482F4907F024FF0028F4D02C48EB
:108FF800A121012207F03EFE4FF48053019304E0C3
:10900800019B5A1E0192002B43D0254C284920462B
:1090180007F024FF0028F3D02046002107F032FE95
:1090280020460121238B07F019FE4FF4805301934A
:1090380004E0019B5A1E0192002B2CD018481D49B0
:1090480007F00CFF0028F4D0154807F098FE4FF4FD
:1090580080530193124A03E0019B591E0191E3B129
:1090680013889C05F8D4012104460D4807F00AFE30
:109078000B48114907F00CFF10E001240EE0022410
:109088000CE003240AE0042408E0052406E0062492
:1090980004E0072402E0082400E0092420461CBD5F
:1090A8000054004001000300820007000400001083
:1090B80002000010400000100004001082B00023DD
:1090C80004E0019B01330193009B01330093009B53
:1090D8008342F6D302B0704737B54FF48053044645
:1090E8000D46019304E0019B5A1E0192002B6DD09E
:1090F8003C484FF4003107F0B1FE0028F3D139485D
:10910800012107F09FFD4FF48053019304E0019B78
:109118005A1E0192002B5BD03248334907F089FE72
:109128000028F4D02F48A021002207F0A3FD4FF417
:109138008053019304E0019B5A1E0192002B49D0F1
:1091480028482A4907F075FE0028F4D0210A254846
:1091580007F013FE4FF48053019304E0019B5A1E5D
:109168000192002B38D01F48214907F062FE0028E1
:10917800F4D0E1B21B4807F000FE4FF4805301938E
:1091880003E0019B5A1E019243B31648184907F0A1
:1091980050FE0028F5D01348294607F0EEFD4FF49D
:1091A8009613019303E0019B5A1E0192C3B10D4827
:1091B800104907F053FE0028F5D00A48012107F0AE
:1091C8004DFD0D48FFF77AFF00200AE0012008E076
:1091D800022006E0032004E0042002E0052000E06D
:1091E80006203EBD00540040010003008200070035
:1091F8008000070004000010A0860100F7B54FF4B6
:10920800805304460D461646019304E0019B5A1EFE
:109218000192002B74D040484FF4003107F01EFE35
:109228000028F3D13C48012107F00CFD4FF480538E
:10923800019304E0019B5A1E0192002B62D036482C
:10924800364907F0F6FD0028F4D03348A021002263
:1092580007F010FD4FF48053019304E0019B5A1E60
:109268000192002B50D02C482D4907F0E2FD002830
:10927800F4D0210A284807F080FD4FF48053019369
:1092880004E0019B5A1E0192002B3FD02248254939
:1092980007F0CFFD0028F4D0E1B21F4807F06DFDBC
:1092A8004FF48053019304E0019B5A1E0192002B56
:1092B8002ED019481B4907F0BCFD0028F4D0002423
:1092C8004FF4961710E0295D134807F056FD0197F3
:1092D80003E0019B5A1E0192E3B10F48124907F0BF
:1092E800BDFD0028F5D00134E3B2B342EBD30A4800
:1092F800012107F0B3FC0D48FFF7E0FE00200AE06B
:10930800012008E0022006E0032004E0042002E037
:10931800052000E00620FEBD0054004001000300C7
:10932800820007008000070004000010A0860100EA
:1093380013B50520012107F0E9FE184C4FF4E0535E
:10934800009302238DF804308DF805302046002361
:1093580069468DF806308DF8073007F02FFB204658
:109368000A21062207F0AAFB20460C21062207F054
:10937800A5FB062220460B21A4F5006407F09EFBFE
:109388004FF4004320466946009307F017FB204638
:109398000F21062207F092FB1CBD00BF0008024007
:1093A8001FB50446FFF7C2F8FFF75EFBFFF7EAF8C0
:1093B800FFF7BEFF01214FF4004007F0CBFE0294F7
:1093C8000F4C1023ADF80230204600236946ADF853
:1093D8000430ADF80C30ADF80030ADF8063007F0C9
:1093E800E8FF69464FF0402008F0B7F82046012111
:1093F80008F067F84FF04020012108F062F81FBD1F
:10940800003C004082B0002304E0019B013301933B
:10941800009B01330093009B8342F6D302B0704750
:1094280007B50420012107F071FE01214FF48040A7
:1094380007F09CFE4FF40073009300238DF804306E
:109448000348012369468DF8073007F0B7FA0EBDC7
:10945800000802400D4B07B51A680D484FF47A739F
:10946800B2FBF3F20B4B013A5A600B4AF02182F837
:10947800231000229A6007221A60084B084A0093BA
:109488000121084B02F012F80EBD00BFE4010020D4
:10949800F426002010E000E000ED00E000030020CA
:1094A800E40200204C020020054B1A6812B11A6829
:1094B800013A1A60034B1A6801321A60704700BFFC
:1094C800B0260020C826002082B0044B0190019AE3
:1094D8001A601A68002AFCD102B07047B026002032
:1094E800704700BF40F0BE60024B40F42020D860B7
:1094F800704700BF00ED00E0C37810B503B3164B0A
:109508004278DB688478DB43C3F30223C3F10401A8
:10951800C9B202FA01F10F2242FA03F2C9B222409B
:109528000A430E4B01781201CB18D2B283F80023FC
:1095380003780122590903F01F0302FA03F307E035
:1095480003780122590903F01F0302FA03F32031BB
:10955800024A42F8213010BD00ED00E000E100E0D1
:1095680021F0604121F07F01014B0843986070476A
:1095780000ED00E0044B1A6909B1104301E022EA4A
:1095880000001861704700BF00ED00E0044B1A6846
:1095980004280CBF42F0040222F004021A6070474B
:1095A80010E000E0014B93ED000A7047142D0020F5
:1095B800014B93ED000A70470C2D0020014B93EDF1
:1095C800000A7047202D0020014B93ED000A7047D8
:1095D800102D0020014B93ED000A7047242D002028
:1095E800014B93ED000A7047182D00200000000081
:1095F80008B5FDF739FE0020012324210246FDF7B6
:109608009DFE124B1B78013BDBB20020012B05D8D5
:109618000146FDF76CFF0120002104E00721FDF75A
:1096280066FF01200721FDF762FF63221221C02097
:10963800FFF74AFA02200121FDF759FFFEF736F835
:109648000120BDE80840FEF726B800BF1C0E002028
:109658000E4B1B78062B05D10D4B0E4A1968126864
:109668008A181A600C4B1B78013BDBB2012B084BA4
:10967800196805D8094A914207DD01321A60704716
:10968800074A914201DD01321A60704771260020B5
:10969800E82C0020682600201C0E00207FD1F0084E
:1096A800FF27ED080F4B1B78062B05D10E4B0F4AF1
:1096B800196812688A1A1A600D4B1B78013BDBB2D5
:1096C800012B094B05D80B4A1968914208DC1A602E
:1096D80070471A68B2F57A2FDCBF4FF47A221A6005
:1096E800704700BF71260020E82C00206826002063
:1096F8001C0E002020A107002DE9F04F6A4B6B4C8F
:109708001B688DB019220A9069485343B0FBF1F0E9
:109718001C190D4609F08AF841EC100B0BF024FADD
:1097280051EC100B09F0BAFB10F0010F804618BF7E
:1097380000F1FF3805FB08F009F078F806462046E6
:109748000F4609F073F802460B463046394609F0D1
:109758000DFA04460D4645EC104B0BF005FA57EC94
:10976800106B204632463B46294608F021FFCDE9DA
:1097780002013946304609F091FB47A3D3E900239B
:109788000B90DDE9020109F043FB002858D10120C4
:1097980000264FF01509314607464FF0000A4FF0F2
:1097A800000B03E030463946069E049FA7FB0A23B8
:1097B800541807FB0B333F4A43F100050023A2422C
:1097C800AB41CDE904453ED3A6FB0A23141806FB9A
:1097D8000B33384843F100050021A042A941CDE9E7
:1097E800064530D3DDE902012DA3D3E90023049C0B
:1097F800069D09F00DFB40BBDDE9022300202E4940
:1098080009F0B4F982468B464BEC10AB0BF0ACF97F
:109818005046594653EC102B8DED080B08F0C8FE46
:10982800CDE90201DDE9080109F006FE09F1FF3979
:109838005FFA89F982468B46B9F1000FB2D104E08C
:109848000125002401E035463C460B9A0A9BD1B21B
:109858005BB9184622462B46FDF770FD0A9801238E
:10986800009301464246034609E022462B46012062
:10987800FDF764FD01200090014642460023FDF7F4
:1098880050FEFDF713FF01200DB0BDE8F04FFDF7C6
:1098980002BF00BFAFF30080956479E17FFDA53D6D
:1098A800BBBDD7D9DF7CDB3DF03A002040787D0195
:1098B80000E9A435FFFF0F000000F03F2B4A2C4BB6
:1098C8001278012A10B518600BD12A4A904201DD9E
:1098D80001321A60284A1B6893420EDC244B1A6036
:1098E8000BE0022A09D1254A904201DD01321A60B3
:1098F800234A1B6893420FDC0CE01D4B214A196870
:10990800914201DD01321A601B68B3F57A2F03DC3E
:109918004FF47A22164B1A60154B1B4A19681B4BD9
:109928001B4C1B68CB18934223601ADC0020FFF7FE
:10993800E3FE01202168FFF7DFFE0C4B1B78013B9B
:10994800DBB20020012B05D80146FDF7D0FD012030
:10995800002104E00721FDF7CAFD01200721FDF7DA
:10996800C6FD034B1A680B4B1A6010BD1C0E002075
:10997800E82C00207FD1F00820A107007F74D21ABC
:1099880060E31600FF27ED0880D1F008002D0020C5
:10999800042D0020D8360020014B18688EE700BF40
:1099A800E4260020AFF300807047FEE7FEE7FEE7FD
:1099B800FEE770477047704702F036B910B5094C9A
:1099C800A37A4BB1084B1A6822F006021A6000F01D
:1099D80013F8204600F047FE4FF48020BDE8104001
:1099E80006F048BDF426002010ED00E0014801F023
:1099F80009B800BFF4260020364BD3F8882042F47B
:109A08007002C3F88820344B1A6842F001021A60C9
:109A180000229A60196821F0847121F4803119605C
:109A28002E495960196882B021F480211960DA60E2
:109A3800009201921A6842F480321A601A6802F49D
:109A480000320192009A01320092019A1AB9009AE2
:109A5800B2F5A06FF2D1204B1B6813F4003318BF86
:109A680001230193019B012B2ED11B4B1A6C42F051
:109A780080521A641A4A116841F4804111609A6848
:109A88009A609A6842F400429A609A6842F4A05236
:109A98009A60144A5A601A6842F080721A6019680B
:109AA8000D4A8901FBD5104B40F205611960936896
:109AB80023F003039360936843F002039360936871
:109AC80003F00C03082BFAD1024B4FF000629A60A6
:109AD80002B0704700ED00E000380240103000246A
:109AE8000070004008544007003C0240184B194AD7
:109AF800996801F00C01042903D0082903D0164BFA
:109B080019E0164B17E059685A6811F4800F596824
:109B180014BF124B104B02F03F02B3FBF2F30C4A96
:109B28005268C2F30142C1F38811013252004B431B
:109B3800B3FBF2F3074A1360054B9A68054BC2F36F
:109B480003129A181968127921FA02F21A607047FA
:109B580000380240E40100200024F40000127A00DA
:109B680037B51C230124002501A88DF804308DF891
:109B780005508DF806408DF80740FFF7BDFC2046DC
:109B8800214607F0E7FA0A4940F2E1434B6040F208
:109B98004F130B800D814D804FF0804007F082FEFF
:109BA8004FF080402146224608F041FA3EBD00BFF2
:109BB800282D002008B54FF08040012108F04CFA0C
:109BC80080B101214FF0804008F051FAFEF726FAE3
:109BD800054B064A11781A788A181A70044B1A88A5
:109BE80001321A8008BD00BF95260020EC3A0020FB
:109BF800780D002008B5402006F02EFC30B1FCF7A7
:109C08005DFD4020BDE8084006F034BC08BD0000FA
:109C1800014608B5044808F0E9FB0348402108F06C
:109C280092FC0028F9D008BD00440040F0B589B086
:109C38004FF4E1330120019300232B4CADF8083099
:109C48001E460146ADF80A30ADF80C30ADF81030BC
:109C58000C23ADF80E3007F059FA4FF4003001210B
:109C680007F078FA20680221072206F027FF07226A
:109C78006068032106F022FF0125022704232068DB
:109C8800059305A98DF81A608DF81B508DF818708A
:109C98008DF8197006F092FE08236068059305A9EF
:109CA8008DF8187006F08AFEA06801A908F0F4FA89
:109CB8002A4640F225510D4808F02CFC262307A817
:109CC8008DF81C308DF81D608DF81E608DF81F50C2
:109CD800FFF712FCA068294608F05BFB044A054B15
:109CE8001A6009B0F0BD00BFF80100200044004030
:109CF800199C00087C3C0020024B9868002108F061
:109D080048BB00BFF801002010B5094C40F22551AE
:109D1800204608F022FC50B1A288D2B2112A02D102
:109D2800044B01211970044B19884A401A8010BD50
:109D3800004400407F0D0020880D002070477047C8
:109D480073B50120014607F0E1F9264C4FF4D853CA
:109D58000093022303268DF8043020460023694629
:109D68008DF806308DF807308DF8056006F026FE70
:109D7800204608210A2206F0A1FE204609210A22CF
:109D880006F09CFE20460B210A2206F097FE0A22C6
:109D980020460C2106F092FE01254FF480632046F0
:109DA800694600938DF806508DF807508DF80560C8
:109DB80006F004FE0A210A46204606F07FFE2946E0
:109DC8004FF4804007F0D2F98020294607F0AAF91D
:109DD8004FF08050294607F0F9F9284606F04AFB6B
:109DE8007CBD00BF0000024007B54FF4C060FFF71C
:109DF80079FB43238DF804300322012301A88DF851
:109E080005308DF806208DF80730FFF775FB0EBD7D
:109E1800782358430723B0FBF3F000230133834230
:109E2800FCD970474FF47A735843F1E737B50023EC
:109E3800104C019305460320FFF7EAFFEB681A6907
:109E4800013C019213D0019A002AF4DA019A42F0F7
:109E580001020192019A1A61064A1969013A0191AF
:109E680002D00199C907F8D40320FFF7D1FF0020D9
:109E78003EBD00BF410D030010B5C47874B900EBB6
:109E8800820003339B10D0F8D000224603E051F83B
:109E9800044C0132046004319A42F8D1002010BD0C
:109EA800033230B59210D0F8D0400B46002003E0C2
:109EB8002568013043F8045C04339042F8D101EB83
:109EC800800030BD0122F0B50023827040220129B4
:109ED800C37082800CD108230370042343704FF4AD
:109EE800A073C38002230372C1724FF0A04309E03C
:109EF80041B90C230370062343704FF4A063C38059
:109F08001F4BC17203F500620261C36046780446C4
:109F180001461A46002508E002F5106C02F5306289
:109F28000A65C1F814C001353A460431B54202F158
:109F38002007F1D303F58062426103F58862C0F817
:109F4800CC20067803F5A0650146002203E0C1F89D
:109F58008C50013220350431B242F8D31946002220
:109F680002E0C4F8CC1001320434B24201F5805149
:109F7800F7D303F56063C0F80C310020F0BD00BFD3
:109F88000000044038B5037AC2680025012B044656
:109F980025D1936B417A65F3104309B143F48013DB
:109FA8009363D36823F4800323F0500343F0100332
:109FB8006FF3C3036FF3C7136FF351436FF3D343C7
:109FC800D3602046FFF732FFE378012B3ED105230B
:109FD80063F34405E36845F020059D6036E0D368E7
:109FE80043F04003D360FFF721FF237A627A032B03
:109FF80014BF4FF434134FF43C130AB143F48013E5
:10A00800E26814209363FFF70DFFE268217AD368B2
:10A01800032908BF43F48033D360237A032B15D177
:10A02800156B012363F39B656FF3D7552D2345F01B
:10A03800805563F316451563C820FFF7F3FEE36800
:10A0480045F400051D63C820FFF7ECFEE378012BFB
:10A0580007D1E3689D68052262F3440545F02005B1
:10A068009D60002038BDC3689A6842F001029A607A
:10A0780000207047C3689A6822F001029A600020A5
:10A08800704707B500230193019B43F02003019318
:10A09800019B61F38A130193019BC2681361064B0C
:10A0A8001169013B019102D001998806F8D4032077
:10A0B800FFF7AEFE00200EBD410D030007B50023DB
:10A0C8000193019B43F010030193019BC268136144
:10A0D800064B1169013B019102D00199C906F8D4D8
:10A0E8000320FFF795FE00200EBD00BF410D0300C1
:10A0F80008B5C268D36801296FF35D736FF39E7367
:10A1080002D143F0005302E009B943F08043322002
:10A11800D360FFF787FE002008BDC368586900F0C8
:10A1280001007047C3685B6913F0010F14BF00207A
:10A1380001207047C368586900F001007047C36880
:10A148005A69986910407047C3685868704703692E
:10A158001A6861F301021A607047C26800239361AC
:10A168004FF0FF335361536053610B4B9361C378D6
:10A178009169002B14BF4FF400634FF4016343F45B
:10A18800701343F4405343F0080321EA03010B43DF
:10A1980093610020704700BF00080080F8B5D0F830
:10A1A8000C3100221A60036915461A6865F3CC223F
:10A1B8001A60C37A012B04461BD10321FFF7C7FF9E
:10A1C800E36880214FF4800261F30F0259629A62BA
:10A1D800C02262F30F0561F31F454FF4A072C3F864
:10A1E800045162F30F056FF31F45C3F80851C3F814
:10A1F8000C5110212046FFF744FF2046FFF75EFF71
:10A20800226900234FF0FF311361204653611E4637
:10A218009161FF25D361214610E082691768C7F371
:10A22800076707F08007FFB2002F14BF4FF0904771
:10A2380000271760013316610430956062789342F5
:10A24800EBD300231D46FF2010E04A6D1668C6F3C5
:10A25800076606F08006F6B2002E14BF4FF090464F
:10A2680000261660013315610431906062789342CC
:10A27800EBD323691A6942F480721A61E278012AE1
:10A2880004D1054A402161F359421A632046FFF779
:10A2980064FF0020F8BD00BF0301010003699B684B
:10A2A800C3F34103013B022B9ABF024AD05C03204F
:10A2B800704700BF68B1040810B5036981699C68DC
:10A2C8000A68C4F34100022802D06FF30A0202E0D0
:10A2D800032060F30A020A605A6842F480725A60E6
:10A2E800002010BD30B54D780B780022012D00EB11
:10A2F800830405D105FA03F3A46963F30F0205E0AB
:10A30800012505FA03F3646D63F31F422368C3F361
:10A31800072505F08005EDB26DB98D6865F30A0370
:10A32800CD78C98865F3934361F3995343F080531B
:10A3380043F4004323600369D9690A43DA610020C2
:10A3480030BD30B54D780B780024012D224600EB46
:10A35800830105D105FA03F3896963F30F0205E068
:10A36800012505FA03F3496D63F31F4203696FF38F
:10A37800CF340C60D96921EA0202DA61002030BDCD
:10A38800F8B54F780B78012F00EB830349D19E690C
:10A398004C69356833692A4664F3120314B967F3C4
:10A3A800DC430BE08F68E419013CB4FBF7F7CC7889
:10A3B80067F3DC43012C08BF64F35E733361C37831
:10A3C800012B06D10B780C6900EB83039B695C6158
:10A3D8000CE0CB78012B09D04B693BB103690C78B1
:10A3E8005E6B012707FA04F434435C63CB78012BD6
:10A3F80007D103699B68DB0554BF45F0005245F05F
:10A4080080520B7800EB830342F004429B691A6088
:10A41800CB78012B38D10A788B8AC968FFF72CFDD5
:10A4280032E05E6D4F6935688C6833692A462FB90A
:10A4380064F31203012464F3DC430AE03F19013F8B
:10A44800B7FBF4F7BF05BF0D67F3DC437C4364F348
:10A4580012033361C378012B05D10B780C6900EB2B
:10A4680083035B6D5C61CB78012B06D14B7913B10B
:10A4780045F0005201E045F080520B7800EB830074
:10A4880042F00442436D1A600020F8BD73B54D7860
:10A49800012D3DD183694A691E681C690094E4B2A4
:10A4A80042B962F306048DF800409DF8024065F356
:10A4B800C4040EE08D68AA4286BF4D6165F30604A8
:10A4C80062F306048DF800409DF80240012262F311
:10A4D800C4048DF80240009A1A61C278012A05D195
:10A4E8000A780C6900EB82029269546146F00442D2
:10A4F8001A60C378002B34D14B69002B31D0036923
:10A508000A78586B012101FA02F202435A6328E0E3
:10A518000B784E698C6800EB83035B6D1A681D69C4
:10A528000095EDB206B14C6164F306059DF8024052
:10A538008DF80050012565F3C4048DF80240009C95
:10A548001C61C378012B05D10B780C6900EB8303E0
:10A558005B6D5C610B7800EB830042F00442436D55
:10A568001A6000207CBD4B78012B0B7800EB830030
:10A578000AD182691368C3F3076101F08001C9B287
:10A5880021B143F0804301E0426D136843F40013A6
:10A598001360002070474B78012B0B78C97800EBCB
:10A5A80083000CBF8269426D02391368C9B26FF328
:10A5B8005553012998BF43F080531360002070471A
:10A5C80003699A69D8691040000C704700EB810153
:10A5D80002694B6D9B685069184070470369986918
:10A5E800DB69184080B2704782B000230093C02313
:10A5F8008DF803300122002362F3C4038DF8023082
:10A6080018238DF80030009A436D1A61C278012A28
:10A6180006D100F5B96058611A684FF080221A60B7
:10A6280002B07047D0F8143110B50446D3B10369AD
:10A638009A68D20716D5827A42B1D0F80C21D0F8A0
:10A648000C116FF341026FF300020A605A6842F07E
:10A6580001025A600520FFF7E5FB23695A6822F0DA
:10A6680001025A6010BD837A63B103699B68D907F8
:10A6780008D5D0F80C31D0F80C216FF341036FF3F3
:10A68800000313607047012310B5002280F81231CF
:10A6980004460346FF2104E058698160186D0132C1
:10A6A8008160607804338242F6D3236900221A61FC
:10A6B8005A61DA614FF0FF329A612046FFF7FEFCDB
:10A6C80020461021BDE81040DBE44B78012B0B78C5
:10A6D80000EB83000FD183691868C0F3074000F0CE
:10A6E8002003DBB2CBB900F00200C0B200280CBFD7
:10A6F800302020207047436D1868C0F3074000F0F1
:10A708002003DBB25BB900F00200C0B200280CBF26
:10A718004FF440504FF400507047102070474FF4EA
:10A72800805070474B78012B0B7810B500EB8303F2
:10A738000AD19C69102A236802D1BDE8104012E7AB
:10A74800202A0CD0302A0FE05C6DB2F5805F2368B8
:10A7580002D143F400131BE0B2F5005F02D143F0CD
:10A76800006315E0B2F5405F0FD1C3F3074202F072
:10A778002002D2B222B100234B71BDE810400AE793
:10A7880043F0806343F0802302E00AB962F3CF33D9
:10A79800236010BDF8B50446FFF794FB012200239F
:10A7A80084F8122184F813312827164619464025C3
:10A7B8000CE007FB03F000F58C7022182354D380BB
:10A7C8005670D1709560D1605161013362789342BF
:10A7D800EFD300232826194640250CE006FB03F09A
:10A7E80000F55C7022182354D3805170D1709560A5
:10A7F800D1605161013362789342EFD32046FFF76D
:10A8080039FC2046FFF7BEFB00212046FFF770FC0D
:10A818002046FFF7C3FC2046BDE8F840FFF723BCFD
:10A8280070B5CDB20C464FF0280601F07F0106FB4B
:10A83800010115F0800F14BF01F58C7101F55C71F1
:10A8480004F07F04ED090C704D708A60CB7005B17F
:10A85800CC80022B01D100230B71FFF743FD0020B0
:10A8680070BD10B5CAB201F07F034FF0280404FB95
:10A87800030312F0800F14BF03F58C7303F55C73A8
:10A8880001F07F01D20919705A701946FFF759FD76
:10A89800002010BD38B501F07F0528246C4304F56D
:10A8A8005C7401194B6100238B614B70EBB203554B
:10A8B800CA60C478012C08BF0A6113B9FFF7E6FD26
:10A8C80001E0FFF75DFD002038BD70B501F07F04A1
:10A8D8002825654305F58C7541190126E4B2CA603F
:10A8E8000A6100224E7044558A614B6114B9FFF722
:10A8F800CDFD01E0FFF744FD002070BDCAB212F0A3
:10A90800800F10B54FF0280306D001F07F0403FB39
:10A91800040303F58C7303E003FB010303F55C7385
:10A92800D209012401F07F0119709C705A701946F0
:10A93800FFF719FE002010BDCAB212F0800F10B543
:10A948004FF0280306D001F07F0403FB040303F54E
:10A958008C7303E003FB010303F55C730024D20945
:10A9680001F07F0119709C705A701946FFF713FEA9
:10A97800204610BD08B50B0604D501F07F01FFF78E
:10A9880080FB01E0FFF79AFB002008BD0369002265
:10A9980061F30A1219680A431A60704703695A6812
:10A9A80003206FF341025A60FFF73CBA03695A6803
:10A9B800032042F002025A60FFF734BA11F0800F08
:10A9C8004FF0280306D001F07F0103FB010101F5D8
:10A9D8008C7103E003FB010101F55C71FFF775BEA3
:10A9E80011F0800F4FF0280306D001F07F0103FB20
:10A9F800010101F58C7103E003FB010101F55C71B4
:10AA0800FFF790BE2DE9F74F0446FFF78BFB0028B0
:10AA180000F03F822046FFF792FB0546002800F031
:10AA28003882C0F3074000F00800C0B2002861D0A7
:10AA38002046FFF7C5FDA146824627464FF000088D
:10AA4800DFF86CB32E4650E01AF0010F46D05FFADB
:10AA580088F2114620460092FFF7B8FD10F0010F6A
:10AA68000546009A20D07B6D01259D60E178A942BA
:10AA780007D11B69D9F87813C3F31203CB1AC9F8A5
:10AA88008833DBF8003020461B6811469847E37886
:10AA9800012B09D1B8F1000F06D194F81131052B1B
:10AAA80002D12046FFF7A0FD05F00203DBB213B187
:10AAB8007B6D02259D6005F00403DBB213B17B6D4D
:10AAC80004259D6005F00805EDB23DB1DBF80030C6
:10AAD80020469B6898477B6D0820986008F101081C
:10AAE8004FEA5A0A043709F12809BAF1000FABD125
:10AAF80035460120C5F3074303F00403DBB2002BFE
:10AB080000F0AF802046FFF769FD264683464FF0E8
:10AB1800000801959FE01BF0010F00F09780236962
:10AB28005FFA88F919695D6B04EB890225FA09F562
:10AB38009269ED019268EDB20D431540EA071CD504
:10AB48005A6B012000FA08F122EA01025A63B3693C
:10AB5800974A9860136805465B68204649469847B7
:10AB6800E378AB4209D1B8F1000F06D194F811315E
:10AB7800042B02D12046FFF737FD05F00403DBB2B2
:10AB880013B1B36904259D6005F00803DBB213B166
:10AB9800B36908259D6005F01003DBB213B1B369F2
:10ABA80010259D6005F02003DBB213B1B3692025A1
:10ABB8009D6005F04003DBB213B1B36940259D6089
:10ABC80005F00203DBB213B1B36902259D6025F0DD
:10ABD8007F0515F0FF0F39D0282505FB084505F539
:10ABE8008C75C246AB696A69C3EB020CAB689C45BD
:10ABF80028BF9C460CF1030CB3694FEA9C0C9B6977
:10AC08006746A04614E0AA68E9681C1B944228BF5E
:10AC18001446A3B240464A46FFF72EF9EB681B19C3
:10AC2800EB60AB69E71C1C19AC61B3699B69BF0891
:10AC38009BB2BB4205D9AC696B699C4201D2002B1F
:10AC4800E1D1B369802544469D60D04608F10108EA
:10AC58004FEA5B0B0436BBF1000F7FF45CAF019D3C
:10AC6800012005F00203DBB213B1E36802225A6146
:10AC7800C5F3076303F08003DBB2CBB1A37A43B11A
:10AC8800D4F80C31D4F80C216FF341036FF30003AF
:10AC9800136023695A6822F001025A60444B1B680A
:10ACA80020469B699847E3684FF000425A610120AB
:10ACB800C5F3072303F00803DBB2F3B13C4B1B6871
:10ACC80020465B6998472369E2689B684FF40061F6
:10ACD8005161A27A82B1DB070ED5D4F80C311A681B
:10ACE80042F001021A601A6842F003021A60314BFE
:10ACF8001A6942F006021A61012005F00803DBB266
:10AD080043B12B4B1B682046DB689847E368082251
:10AD18005A61012005F01003DBB2002B33D0E36841
:10AD28009A6922F010029A611F6A282607F00F0319
:10AD380006FB0346C7F34343022B06F55C7602D0B5
:10AD4800062B1AD10EE047F6F0733B40ABB1C7F3C0
:10AD58000A172046F1683A46FFF7A2F8F368DB19AC
:10AD6800F36007E004F5B96120460822FFF798F878
:10AD7800C7F30A17B369DF19B761E3689A6942F044
:10AD880010029A610120C5F3072303F01003DBB218
:10AD9800002B39D023695A68002622F001025A6034
:10ADA80031462046FFF76DF923463246FF2108E079
:10ADB8009402002000ED00E058698160186D0132AE
:10ADC8008160607804338242F6D3236901274FF00B
:10ADD800FF3267F30F069A6167F31F460F22DE61A1
:10ADE8005A612F221A611A686FF30A121A602046F4
:10ADF800FFF7FAFBE3684FF480525A61264B1B6851
:10AE080020461B6998473846C5F3072303F02003FB
:10AE1800DBB2EBB12046FFF74FFAE3682046DE6865
:10AE2800FFF73CFA032806D10023A3704FF4007300
:10AE3800A380092304E00123A3704023A3800523F2
:10AE480063F38D26E3684FF40052DE6001205A61F7
:10AE5800C5F3074303F01003DBB24BB10E4B1B687D
:10AE68002046DB699847E3684FF480125A61012055
:10AE7800C5F3074505F02005EDB255B1064B1B6833
:10AE880020461B6A9847E3684FF400125A61012074
:10AE9800FFE7BDE8FE8F00BF9402002043230B802C
:10AEA800004870470402002038B51F4B1A68511C2F
:10AEB800052A196035D11979002201291A6030D084
:10AEC8009968B1F5006F08BF9A60174B9968DC68FC
:10AED800A1421A4602D100221A7122E086BFC1F5AA
:10AEE80000631361C1EB0404D0F8EC3598BF14611A
:10AEF8001569B3F839300C4C9D428AB204D95918F7
:10AF0800ED1AA160256104E06918A1600021ABB2C7
:10AF18002161054901240C7104498A188121FFF730
:10AF2800D4FC002038BD00BF8C0D0020C72D0020A8
:10AF380038B528230A4D03FB01010A4BB1F88813E1
:10AF48001B69044628469847D4F8EC352046B3F8E0
:10AF5800403001212A46FFF79DFC002038BD00BF84
:10AF68007F2D00208002002070B50B7813F060055B
:10AF780006460C4625D0202D1FD1CD88B5B113F03B
:10AF8800800F487808D0214B21499B682A4698476A
:10AF9800E2881F49304625E01E4B1D4958641E4B68
:10AFA80030465D612A4600F022FB1DE0174B4878C9
:10AFB8009B6829462A46984725E000F077FB02253A
:10AFC80021E04B780A2B11D00B2B14D0062B1AD169
:10AFD8004B881B0A212B03D1CA883A2A28BF3A2258
:10AFE8000E49304600F0EAFA00250CE00C4901222F
:10AFF80000F0E4FA07E08B781BB9074A1D46936115
:10B0080001E000F053FB284670BD00BF800200201D
:10B01800BF2D0020040200208C0D00201602002005
:10B02800A40D002010B581210446FFF71AFC012168
:10B038002046FFF716FC82212046FFF712FC024B40
:10B048005B689847002010BD8002002038B5D0F812
:10B05800EC350446B3F8392081210223FFF7E0FBE1
:10B06800D4F8EC350121B3F8402020460223FFF73D
:10B07800D7FB8221082203232046FFF7D1FB094B87
:10B08800022200251A715D71074B1B689847D4F896
:10B09800EC35064AB3F8403020460121FFF7FAFBA9
:10B0A800284638BDC4020020800200207F2D0020E1
:10B0B80010B5074C606CFF2807D0064B064A9B6802
:10B0C800064952699847FF236364002010BD00BFFA
:10B0D80004020020800200208C0D0020BF2D0020DB
:10B0E80038B510490B79012B19D10C690CB90C71C1
:10B0F80015E0D0F8EC358D68B3F839309C42AAB227
:10B1080003D95D198D60E41A03E0A3B22C198C6091
:10B1180000240C61044952188121FFF7D6FB002056
:10B1280038BD00BF8C0D0020C72D002000207047BF
:10B13800002070470023F0B5084A094E1D4609E073
:10B148001468C75C375501340133B4F5006F1460D7
:10B1580008BF15608B42F3D10020F0BD980D002088
:10B16800C72D0020104B114AD3F800C000232DE949
:10B17800F0410F4F16461D460DE0146810F8038085
:10B1880007F804800134802C08BF2C46146034680A
:10B19800644505D001338B42EFD10020BDE8F08132
:10B1A8000220BDE8F08100BF483600205C36002050
:10B1B800C835002021280FD1084B1A680A701A6870
:10B1C800120A4A705A888A70DA78CA701A790A712B
:10B1D8005A794A719B798B71002070477802002058
:10B1E80007B502AB012103F8010D1846FFF7A2FFCE
:10B1F8000EBD002100E00131435C002BFBD199E733
:10B2080098E70B4B0B491A68096891420BD00A4919
:10B218008A5C02701A680132802A1A6005D10022FD
:10B228001A6001207047002070470120704700BF56
:10B23800483600205C360020C8350020204B1A68AC
:10B24800204B1B689A42F0B509D135E00133802BB9
:10B2580008BF00239A4203D11A4B1A602CE01A4CFB
:10B26800E15C0029F2D00A29F0D00D29EED0154C66
:10B278001549134D23600E460023CF182268BA5C87
:10B28800C254226801339F18802F08BF53422F6889
:10B298009A18974210D0B25C1AB10A2A01D00D2A26
:10B2A800EBD10022C254074A116859187F2911604E
:10B2B80003D98039116000E000231846F0BD00BFB3
:10B2C8005C36002048360020C8350020704700BF93
:10B2D800D0F8E43510B51B6904469847032384F871
:10B2E8001231002010BD08B5042380F81231D0F8BF
:10B2F800E435DB689847002008BD08B5D0F8E0358C
:10B30800DB6903B19847002008BD08B5D0F8E035DF
:10B318001B6A9847002008BD08B5D0F8E0355B6A7D
:10B328009847002008BD002110B5402204460B466E
:10B33800FFF776FA8021402200232046FFF770FAB3
:10B34800012384F81231D4F8E435A0785B68984773
:10B35800002010BD13B56946044600F085F99DF834
:10B36800001001F01F03012B07D0022B0AD073B97C
:10B378002046694600F026FA0FE02046694600F0AC
:10B3880007FA0AE02046694600F0A2F905E021F034
:10B398007F01C9B22046FFF7B1FA00201CBD38B5BD
:10B3A800044600293DD190F81131022B42D1D0F842
:10B3B8003421D0F820319A4211D9C178D21A012902
:10B3C800C0F8342104D1D0F82411CB18C0F82431A6
:10B3D80092B22046D4F8241100F000F92AE0D0F8FF
:10B3E8003821B2FBF3F503FB152565B99A420AD358
:10B3F800D0F83C319A4206D229462A4600F0EEF8A7
:10B40800C4F83C5116E0D4F8E035DB682BB194F869
:10B418001221032A01D120469847204600F00FF94F
:10B4280008E0D0F8E0355B6923B190F81221032ACF
:10B4380000D19847002038BD10B5044659BB90F894
:10B448001131032B30D1D0F88C23D0F878339A42BD
:10B4580014D9C178D21A0129C0F88C2304D1D0F8A4
:10B468007C13C918C0F87C139A4228BF1A4692B2B6
:10B478002046D4F87C1300F0CAF815E0D0F8E0357F
:10B488001B6923B190F81221032A00D1984720465E
:10B4980000F0C6F808E0D0F8E0359B6923B190F8D1
:10B4A8001221032A00D19847002010BD2DE9F04150
:10B4B800069F0446164698460D46FEF741FC204670
:10B4C8002946C4F8E085C4F8E475C4F8E865FFF7D0
:10B4D80061F9D4F8E4351B6898472046BDE8F04187
:10B4E800FEF782BC00207047D0F8E03510B504465E
:10B4F8001B689847D4F8E4359B689847002010BD2E
:10B5080008B5D0F8E0355B689847002008BD000012
:10B5180012230B8000487047C402002004230B80CC
:10B5280000487047D602002010B5044C04480A466B
:10B53800214600F075FA204610BD00BF6036002095
:10B5480081B605080A4608B50248034900F068FABA
:10B55800014808BD94B60508603600200A4608B5BB
:10B568000248034900F05CFA014808BDA2B6050884
:10B578006036002008B50A4608B9044800E00448C7
:10B58800044900F04DFA034808BD00BFADB60508F0
:10B59800BAB605086036002008B50A4608B9044856
:10B5A80000E00448044900F03BFA034808BD00BF26
:10B5B800C7B60508E8B605086036002010B513467A
:10B5C8000C46C0F83821C0F83421022280F8112135
:10B5D80000212246FFF779F9002010BD10B50C466E
:10B5E800134600212246FFF770F9002010BD10B560
:10B5F80013460C46C0F89023C0F88C23032280F829
:10B60800112100212246FFF745F9002010BD10B591
:10B618000C46134600212246FFF73CF9002010BDD6
:10B628000021042310B50A46044680F811310B4660
:10B63800FFF74BF92046FEF7D7FF002010BD002189
:10B64800052310B50A46044680F811310B46FFF76A
:10B6580021F92046FEF7C8FF002010BD282303FB70
:10B668000100B0F88803704790F8C8350B7090F85F
:10B67800C9354B7090F8CB2590F8CA3503EB0223F7
:10B688004B8090F8CD2590F8CC3503EB02238B80C6
:10B6980090F8CF2590F8CE3503EB02239BB2CB80F0
:10B6A800C0F83C31012380F81131704710B591F989
:10B6B8000030002B044601DBCB880BB9802100E069
:10B6C8000021FFF71BF92046BDE81040FEF78CBFAC
:10B6D80038B50D4604466B780979012B10D027D36D
:10B6E800032B51D190F81231022B28D0032B47D1CC
:10B6F8006B889BB991B1802910D0FFF7FFF80DE056
:10B7080090F81231022B1AD0032B39D16B88002BF9
:10B718003AD149B1802907D0FFF70EF9D4F8E035BE
:10B7280020469B68294698472046FFF779FF2BE07B
:10B7380090F81231022B02D0032B21D106E019B365
:10B74800802921D02046FFF7D9F81DE011F0800F9D
:10B758004FF0280306D001F07F0103FB010393F8A3
:10B768001A2103E003FB010191F87223074B02B190
:10B7780001221A60204605490222FFF71FFF03E055
:10B7880020462946FFF792FF002038BDA80D00206B
:10B7980038B590F81231032B04460D460CD10B79BD
:10B7A800012B09D8D0F8E0359B689847EB883BB95E
:10B7B8002046FFF735FF03E020462946FFF776FFCE
:10B7C800002038BD73B54B7804460D46092B00F2AE
:10B7D8001C81DFE813F0D10008011A01E4001A0106
:10B7E80072000A001A01C00092004B881A0A013A36
:10B7F800062A00F20A81DFE812F007001A00270083
:10B808000801080108010801D4F8E835A0781B6888
:10B818000DF106019847EB88402B014603D094F8B8
:10B828001231012B3AD10823ADF8063036E0D4F8AE
:10B83800E035A0789B6A0DF1060198470223437012
:10B848000146C4F8EC0529E0DBB2052B00F2DD80E7
:10B85800DFE803F003080D12171CD4F8E835A078C8
:10B868005B6817E0D4F8E835A0789B6812E0D4F854
:10B87800E835A078DB680DE0D4F8E835A0781B69D6
:10B8880008E0D4F8E835A0785B6903E0D4F8E83537
:10B89800A0789B690DF1060198470146BDF806306E
:10B8A800002B00F0B680EA88002A00F0B2809A42A5
:10B8B80028BF1A46ADF806205CE08B88002B40F0C4
:10B8C800A480CB88002B40F0A08094F812214B88EC
:10B8D800032A00F09A8003F07F05204684F813516C
:10B8E8002946FFF753F82046FFF79AFE0DB10223C9
:10B8F80000E0012384F812318BE08978464E012953
:10B90800317100F2828094F81231022B02D0032B9D
:10B918007BD108E0002962D00121032384F81011AB
:10B9280084F8123113E041B9022384F8123184F803
:10B9380010112046FFF7E4FD51E094F81011012999
:10B9480020464DD0FFF7DCFD317984F810112046F0
:10B95800FFF7CAFD43E0CA88012A56D194F812318C
:10B96800022B02D0032B50D102E020462B4913E0D2
:10B9780004F5887120460FE094F81231023B012B40
:10B9880043D8D4F814312449002B0CBF01230323D6
:10B9980041F80C3F20460122FFF710FE39E04B88A2
:10B9A800012B29D0022B34D18B8813F0FF0F30D113
:10B9B80021691B0A013B4A68042B0FD8DFE803F012
:10B9C800030507090B00012306E0022304E0032313
:10B9D80002E0042300E0052363F306124A602046D0
:10B9E800FFF71EFE15E094F81231023B012B0CD82C
:10B9F8004B88012B0DD10023C4F81431D4F8E0355D
:10BA080020469B6829469847E9E720462946FFF7DC
:10BA18004DFE00207CBD00BFA80D0020B00D002009
:10BA280030B5C8B10023DDB20133C41814F8014C95
:10BA3800002CF8D16B1C5B0013800B7003234B7038
:10BA4800022305E0CA545A1CD2B202338C54DBB22A
:10BA580010F8012B002AF5D130BD00BF70477047A0
:10BA6800704770477047704770470000000000003B
:10BA780008B5FCF701FA094B5A78187002435A7056
:10BA88001AB19A7801329A7030B99B78034A012B1F
:10BA980002D900235370937008BD00BFB80D002071
:10BAA8002DE9F84F3F4B1B78012B2DED028B09D068
:10BAB80002D3022B0FD108E03B4B1A68802392FB7C
:10BAC800F3F206E0384B1A6803E0374B1B68032291
:10BAD8005A43364B5A61364B1A8892B2002AFBD029
:10BAE800334B00221A80FDF75DFD10EE105AFDF76A
:10BAF8005FFD284610EE104A06F0BAFE8046204642
:10BB0800894606F0B5FE41EC100B41EC180B08F025
:10BB1800D3FF57EC106BB0EE480AF0EE680A09F054
:10BB2800CBF832463B46404649465BEC10AB06F044
:10BB3800F3FE07F0D3F99FED1F8A07EE100ADFED39
:10BB48001E7A57EE087A194C52465B46C4ED007AC5
:10BB58004046494606F0E0FE07F0C0F907EE900AB5
:10BB680027EE888A84ED018AFDF734FD84ED020A08
:10BB7800FDF736FD84ED030AFCF78CF80F4B62697C
:10BB88001B68D31A0E4A07EE100A1268F8EEC77A35
:10BB980093FBF2F3C4ED047A2383BDEC028BBDE87A
:10BBA800F88F00BF1C0E0020E82C00209C380020D5
:10BBB800680D00200000F04200008C42E4260020BE
:10BBC8006826002007B50420012105F09FFA4FF4EC
:10BBD8006043009301238DF8043002238DF805306B
:10BBE8000448002369468DF806308DF8073004F0C4
:10BBF800E5FE0EBD00080240084B1A684FF47A7340
:10BC0800B2FBF3F2064B013A5A60064AF02182F879
:10BC1800231000229A6007221A607047E40100206E
:10BC280010E000E000ED00E0034B5A6812B15A68DA
:10BC3800013A5A60704700BFB80D0020024B5860A7
:10BC48005A68002AFCD17047B80D002030B585B07D
:10BC580004460D4601A867490A220BF025FC664BED
:10BC68001B78032B10D8DFE803F00205080B01A8A6
:10BC7800624907E001A8624904E001A8614901E0BE
:10BC8800614901A80BF0FAFC04AA131913F80C3C3B
:10BC98005D19EDB22F2D01D80A3502E0392D01D9F1
:10BCA8000A3DEDB204AB1C194FF6FF7004F80C5CAA
:10BCB800FAF76CFA0020FAF76BFB0DF103050F2475
:10BCC800204623345A21002315F8012FA4B2FAF78D
:10BCD80079FBB4F5A57FF3D164205A212C220023E7
:10BCE800FAF770FB0023CD205A212C22FAF76AFBC1
:10BCF8000020FAF74BFA404B1B78032B78D8DFE883
:10BD080003F00233616C01A93C480BF0B7FC0A222E
:10BD180000213A480CF0DAFD3C4A3D4B1278186095
:10BD2800012A0BD002D3022A1AD10EE0B0F5FA5F2D
:10BD3800BCBF4FF4FA521A60364A0CE0364A9042B9
:10BD480001DC01321A60354A05E0354A904201DCCF
:10BD580001321A60334A1B689342C4BF2C4B1A60E5
:10BD6800314B1A68314B2BE001A925480BF086FCB2
:10BD78000A22002122480CF0A9FD244A2C4B1278F3
:10BD88001860012A0BD002D3022A31D10EE0B0F597
:10BD9800FA5FBCBF4FF4FA521A601E4A0CE01E4A02
:10BDA800904201DC01321A601C4A05E01C4A9042AC
:10BDB80001DC01321A601B4A1B68934218DD1C4BD8
:10BDC8001A6015E001A90F480BF058FC0D48002136
:10BDD8000A220CF07BFD174B09E001A90A480BF079
:10BDE8004DFC094800210A220CF070FD124B186026
:10BDF80005B030BD09B70508E3260020B4260020A9
:10BE0800D8260020EE2C0020A02600201C0E0020A2
:10BE1800F026002050DA11001FA1070080D1F00899
:10BE28005FE316008074D21AE4260020E82C002074
:10BE3800082D0020E42C00209C26002010B50D4B76
:10BE48000D4C1A680D4821460BF0F0FB0C4B0D48C1
:10BE58001A6821460BF0EAFB0B4B0C481A6821467E
:10BE68000BF0E4FB0A4B0B481A682146BDE810406A
:10BE78000BF0DCBBF0260020CFAC0508B426002070
:10BE8800082D0020D8260020E42C0020EE2C0020CD
:10BE98009C260020A02600209FED010A704700BFC5
:10BEA800000000009FED010A704700BF000000007D
:10BEB8009FED010A704700BF0000000018B101287B
:10BEC80001D1034B00E0034B1868FDF7F7BC00BF36
:10BED800D4260020E426002010B9034B18687047C8
:10BEE800024B1868704700BFF0260020E4260020A7
:10BEF80010B9034B18687047024B1868704700BFA9
:10BF0800082D0020D426002008B54FF49570FBF7C3
:10BF1800D5FE40F26523C31A584240EB030008BD22
:10BF280008B5C620FBF7CAFE40F28D13C21A50426C
:10BF380040EB020008BD4FF4957040F26521FBF715
:10BF4800AFBEC62040F28D11FBF7AABEDCE760EE5B
:10BF5800A00AB7EE007AF0EE606A70EE077A40EE5B
:10BF6800006A47EEA70A36EEC77A08B5C7EE200A78
:10BF780010EE900A06F07CFC0022084B06F0CCFC80
:10BF88000022074B06F016FB06F0A8FF07EE900A02
:10BF9800FDEEE77A17EE900A9F3008BD0000594081
:10BFA8000000E03F38B52DED028BF7EE008AB0EEC9
:10BFB800608A70EE288A10EE900A28EE088A06F049
:10BFC80057FC08EEA88A00220F4B06F0A5FC044691
:10BFD80018EE100A0D4606F04BFC02460B462046AA
:10BFE800294606F0C3FD0022084B06F0E3FA06F0E6
:10BFF80075FF07EE900AFDEEE77A17EE900A7730A4
:10C00800BDEC028B38BD00BF000069400000E03F76
:10C018002DE9F04F884F2DED068B97E80F0091B072
:10C028000CAC103784E80F000FCF05AE0FC697E8A9
:10C0380007004FF6FF7386E807009F2077216422E8
:10C04800F7F76DFDA020772164224FF6FF73F7F70D
:10C0580066FD9E20772164224FF6FF73F7F75FFD98
:10C068009F20762164224FF6FF73F7F758FD4FF6AD
:10C07800FF73782164229F20F7F751FD0020F9F71C
:10C0880062F99F2077216522FAF7C2F80C349F20C5
:10C0980077216422FAF7BCF80DF12C0A0394F7EE25
:10C0A800009A4FF00F0B00E04D460AF1040AF7EE34
:10C0B800008A9AED009A0024B0EE68AA01E0B8461A
:10C0C800354618EE900A06F0D3FB59A3D3E90023AE
:10C0D80006F022FC06F002FF08EE900A38EEE98A24
:10C0E800B0EE490AF0EE480AFFF731FFB0EE490A10
:10C0F800F0EE480A0646FFF755FFB2B2074683B28C
:10C108002CB9104619460F22F9F7DCF906E0A8B257
:10C118001FFA88F1CDF800B0F9F7C4FF0134B4F57F
:10C12800967FCCD13D46F7EE008A002401E04546D3
:10C138004E4618EE900A06F09BFB3DA3D3E9002378
:10C1480006F0EAFB06F0CAFE08EE900A39EEE88A25
:10C15800B0EE490AF0EE480AFFF7F9FEB0EE490AD8
:10C16800F0EE480A8146FFF71DFF1FFA89F2804664
:10C1780083B22CB9104619460F22F9F7A3F905E046
:10C18800B0B2A9B2CDF800B0F9F78CFF0134B4F51C
:10C19800967FCCD1039B9A4586D104AD0DF12C0B2B
:10C1A8004FF0000A01E0B846B146043595ED009A13
:10C1B800F7EE008A002401E0B846B14618EE900A6E
:10C1C80006F056FB1AA3D3E9002306F0A5FB06F0F8
:10C1D80085FE08EE900A38EECA8AF0EE490AB0EEFB
:10C1E800480AFFF7B4FEB0EE480AF0EE490A0646E0
:10C1F800FFF7D8FEB2B2074683B22CB910461946EB
:10C208002246F9F75FF907E01FFA89F01FFA88F16B
:10C21800CDF800A0F9F746FF0134B4F5C87FCBD1BB
:10C228005D45C0D111B0BDEC068BBDE8F08F00BFF5
:10C23800295C8FC2F528F03F6CB10408121A06EE8B
:10C24800902A081AB8EEE67A06EE900AF8EEE67A30
:10C2580008B5C7EE277A17EE900A06F009FB002208
:10C26800044B06F059FB0022034B06F0A3F906F035
:10C27800EDFD08BD000074400000E03F8A1A06EE9C
:10C28800902A081AB8EEE67A06EE900AF8EEE67AF0
:10C2980008B5C7EE277A17EE900A06F0E9FA0022E9
:10C2A800044B06F039FB0022034B06F083F906F035
:10C2B800CDFD08BD000069400000E03F70B50646AE
:10C2C8000D460024610704D5A0B231462A46F9F785
:10C2D800F9F80134B4F5A07FF4D170BD70B5064605
:10C2E8000D460024600704D5A1B230462A46F9F766
:10C2F800E9F80134C82CF5D170BD234B1B78012B0C
:10C3080003D011D3022B3DD123E0204B1A68204BD8
:10C318001A60204B1A68204B1A60204B1A68204B71
:10C328001A60204B1A6811E0184B1A68184BD20192
:10C338001A60184B1A68184BD2011A60174B1A6802
:10C34800174BD2011A60174B1A68D201164B1A60A4
:10C3580070470E4B0E4A1968032391FBF3F11160E5
:10C368000C4A11680C4A91FBF3F111600B4A1168F1
:10C378000B4A91FBF3F111600A4A126892FBF3F33E
:10C38800094A1360704700BF1C0E0020F0260020E9
:10C39800E4260020082D0020D4260020E42C0020CC
:10C3A80068260020C0260020002D0020014B1868B8
:10C3B800FDF784BAE426002008B5FFF79EFFBDE824
:10C3C8000840F3E770B500210A222748274D284E78
:10C3D800284C0CF07BFA00210A22286026480CF031
:10C3E80075FA00210A22306024480CF06FFA002107
:10C3F8000A22206022480CF069FA224B3268186041
:10C408002B682149D31A06EE903A2368B8EEE67AEB
:10C4180006EE903AF8EEE67AC7EE277AFCEEE77A6F
:10C4280017EE903A9AB20B80531C07EE903AB8EE8A
:10C43800E77ADFED167A67EE277A154BFCEEE76AA6
:10C4480016EE901A8AB206EE902AB8EEE67A1980AD
:10C4580077EEC77AF5EEC07AF1EE10FA01DD013217
:10C468001A80BDE87040A7E7B4260020F026002017
:10C47800082D0020E42C0020D8260020EE2C0020D7
:10C48800A02600209C260020DC3A00200000803DE9
:10C49800703B00200022F0B51346202603254FF0FC
:10C4A8002C0C00E02646303EF6B217460132092E23
:10C4B80010F8014B0AD897FBF5F605FB16772FB94C
:10C4C800CE1801F803C07470023301E0CC54013374
:10C4D800092AE7D12022CA54CB1848225A707A2256
:10C4E8009A700022DA70F0BDF0B51F46144B1E7822
:10C4F800012E8DB005460C4620D0A6F1030CDCF1C8
:10C50800000646EB0C06CEB90E4908A80BF08EF8CB
:10C5180008A86946FFF7BEFF0B496A4604A80BF056
:10C5280085F8BDF84800F9F731FE3846F9F744FEBA
:10C538002846214604AA3346F9F762FF0DB0F0BD3C
:10C5480071260020CFAC05084CB4050810B50121B0
:10C558000446F8F7DDFF014B1C8110BDB80D002023
:10C5680008B50021C620FBF79BFB4FF4957000210E
:10C57800BDE80840FBF794BB014B9F221A81704726
:10C58800B80D002000200146C82240F23F13F8F7FA
:10C59800CFBF07B50DF10700FEF733FE9DF8070082
:10C5A8000EBD08B5FFF7F5FF0028FBD108BD30B573
:10C5B800044687B010EE100A0D4606F059F90246F7
:10C5C8000B4601A805490BF031F82046294601AA77
:10C5D8000023F9F715FF07B030BD00BF13B70508F2
:10C5E80008B5084803F04CFC0648022103F019FD81
:10C5F8000028F9D0034803F06FFC07EE900AB8EE64
:10C60800670A08BD0020014010B52DED028B9FED93
:10C61800098A1924FFF7E4FF013CE4B238EE008AE6
:10C62800002CF7D19FED040A28EE000ABDEC028B1E
:10C6380010BD00BF00000000ACC868392DE9F04FFC
:10C64800994B9A4C5D695E682DED068B93ED00AAB7
:10C65800C7B007461AEE100A93ED038AD3ED04AA71
:10C66800D3ED028A93ED069A06F002F941EC100B1D
:10C67800CDE9040108F004FC3A468D493BA88DED4C
:10C688000C0B0AF0D3FFA06806F0F2F802460B463E
:10C698002BA888490AF0CAFFE06806F0E9F80246C4
:10C6A8000B462FA884490AF0C1FF1AEE900A06F03B
:10C6B800DFF8CDE90A01DDE90A23804933A80AF049
:10C6C800B5FF284606F0D4F8CDE90601DDE90623D2
:10C6D8007B4937A80AF0AAFF18EE900A06F0C8F8B6
:10C6E8008046894642464B46764913A80AF09EFF83
:10C6F80018EE100A06F0BCF882468B46524672497C
:10C708005B4617A80AF092FFDDE904236F491BA8CE
:10C718000AF08CFF304606F0ABF85BA3D3E90023A0
:10C72800CDE9080106F0F8F802460B461FA868494B
:10C738000AF07CFF49EC118B4BEC10AB08F018FBAE
:10C7480051A3D3E9002351EC100B06F0E5F802469B
:10C758000B4627A85F490AF069FF19EE100A06F090
:10C7680087F80B4602465C4923A80AF05FFFD4ED20
:10C77800047AFDEEE77A594917EE902A0FA80AF0D5
:10C7880055FF0022564BDDE90C0106F0C5F806F00E
:10C79800A5FB06F06DF802460B4643A851490AF07E
:10C7A80045FFB5EEC08AF1EE10FADFED4F9A37D5A6
:10C7B800384606F04BF836A3D3E9002306F0ACF868
:10C7C800F1EE487A044617EE900A0D4606F050F846
:10C7D80002460B462046294606F09EF802460B46BE
:10C7E8002DA1D1E9000106F0C1F906F077FB9FED14
:10C7F8003F7A07EE900AF4EEC77AF1EE10FAC6BF58
:10C80800C7EEA97A3A4C3B4CF4EEE97AF1EE10FA0D
:10C8180038DD9FED357A384D384CC7EE877A78E0A9
:10C828001FA3D3E900235046594606F075F804467D
:10C8380038460D4606F00AF815A3D3E9002306F09A
:10C848006BF802460B462046294606F08FF906F09B
:10C8580045FB07EE900AB7EE007AF4EEC77AF1EEE0
:10C8680010FA46BF67EEA97A254C264CF4EEE97A11
:10C87800F1EE10FA4CDD9FED1C7A234D234CC7EEE8
:10C88800877A46E01C4D44E06666666666A64C40BC
:10C898001F85EB51B81E1940000000A2941A6D4282
:10C8A8000000000080842E418C3A00209C38002033
:10C8B80035B705083FB705084AB7050855B705084D
:10C8C8005FB7050869B7050874B705087FB7050895
:10C8D8008AB7050895B70508A0B70508ACB70508D5
:10C8E800000034C0B9B7050800007A440024744930
:10C8F80024B7050821B70508C5B605082DB70508EA
:10C908002AB7050827B7050830B7050832B705085C
:10C918008B4D17EE900A05F0ABFF2A46CDE90001D2
:10C92800884902943FA80AF081FE874B874D186812
:10C93800874B19688F42CCBF002301238742D8BF99
:10C948000023EB60834B1B780D2B2ED13A46FFF763
:10C9580075FC814B0646186805F08AFF00227F4B5C
:10C9680005F0DAFF02460B4600207D4905F020FE5F
:10C9780006F06CFA4FF6E073009304460023052096
:10C98800DC213A46FFF7B0FDEB6853B1754B1888C8
:10C99800754B4FF4FC6519880095B2B2A3B2F9F74C
:10C9A80081FB704B1E60704B1C606A4B1B78082B18
:10C9B80040F0AE800220F9F7EBFC4FF6FF70F9F774
:10C9C800FBFB1F20F9F7E2FB19210023674A2D2002
:10C9D800F9F716FD4FF6FF70F9F7EEFB002000247B
:10C9E800F9F7D4FB0F20B4213A464FF6FF730094B1
:10C9F800FFF77AFD0F206E2123462BAAF9F700FDD9
:10CA0800B0206E2123462FAAF9F7FAFC0F2038210F
:10CA180023461BAAF9F7F4FCB020382123461FAAA5
:10CA2800F9F7EEFC0F205C21234633AAF9F7E8FC5E
:10CA38002346B0205C2137AAF9F7E2FC0F204A21EF
:10CA4800234613AAF9F7DCFCB0204A21234617AA8B
:10CA5800F9F7D6FC0F209B21234623AAF9F7D0FC2F
:10CA68000F20842123463FAAF9F7CAFCB02084216D
:10CA7800234627AAF9F7C4FCB0209B2143AA2346E2
:10CA8800F9F7BEFC3A4B1B68B3F57A7FCCBF4FF47D
:10CA9800FC604FF47840F9F78FFB0023A020B42105
:10CAA8000FAAF9F7ADFC334B1C78012C0CD002D33C
:10CAB800022C1DD111E04FF6E070F9F77DFB4FF421
:10CAC8008C7002212C4A10E04FF4FC60F9F774FBDB
:10CAD8004FF48C700221294A07E04FF6E070F9F70D
:10CAE8006BFB274A4FF48C7021460023F9F788FC2A
:10CAF8000020F9F761FB4FF4FC60F9F747FBFFF7FB
:10CB080083FD0F20DC21FFF752FD1F20F9F754FBAE
:10CB1800104B1B789A1FD2B2012A02D90B2B40F076
:10CB28005C82184B1B78023B052B00F25682DFE82B
:10CB380013F02D007D00EE004701EF01640100BFF6
:10CB480030B70508C7B70508F0260020B80D002043
:10CB5800082D002071260020C03600200000044067
:10CB680000003940D83800207C3B0020D4B70508A5
:10CB7800181B00201C0E00202EB6050833B6050829
:10CB880037B60508FC2C00200000C8425FED027A89
:10CB98002AEE27AA1AEE100A05F06AFE9DED080B88
:10CBA8008046894607F088FF404653EC102B4946DB
:10CBB80005F0B2FED2A3D3E9002305F0FBFC06F092
:10CBC80045F99DED080B044608F076F8404653EC0D
:10CBD800102B494605F0A0FE02460B46CAA1D1E932
:10CBE800000105F0E5FC06F031F94FF6E07300931B
:10CBF800054600230520DC213A46FFF775FCB44BB7
:10CC0800DB6853B1B34B1888B34B4FF47846198897
:10CC18000096A2B2ABB2F9F745FAAE4B1C60AE4B28
:10CC28004FF6E0701D60F9F7B1FAD6E1AB4B186822
:10CC3800AB4B3A461968FFF701FBAA4B1B784FF438
:10CC4800FA7292FBF3F307EE903AB8EEE79ADFED4B
:10CC5800A67AF4EE498AF1EE10FAC8BFF0EE498AD6
:10CC6800F5EE408AF1EE10FA48BFF0EE678AF4EE6E
:10CC7800C98AF1EE10FA044620D8F4EEE78AF1EEFC
:10CC880010FA1BDBFDEEC97AFDEEE88A17EE901A62
:10CC980018EE902A0020FFF7F1FA8D4BDB68054665
:10CCA80053B18C4B18888C4B4FF6FF761988009639
:10CCB800A2B2ABB2F9F7F6F9874B1D60B4EE498A18
:10CCC800F1EE10FAC8BFB0EE498AF1EE497AB4EE37
:10CCD800678AF1EE10FA48BFB0EE678AB4EEC98AE7
:10CCE800F1EE10FA00F27981B4EEE78AF1EE10FA6B
:10CCF800C0F27381FDEEE77ABDEEC99ABDEEC88A2F
:10CD080017EE900A19EE101A18EE102AAEE0734BBF
:10CD18001868734B3A461968FFF790FAF5EEC0AAFF
:10CD2800F1EE10FA044627DDDDE90A015AA3D3E93A
:10CD3800002306F063F8F8B159A3D3E90023DDE92D
:10CD48000A0105F0E9FD0B4602466849002005F096
:10CD58002FFC06F07BF85E4BDB68054653B15D4B54
:10CD680018885D4B4FF6FF7619880096A2B2ABB2D1
:10CD7800F9F798F9584B1D60DDE906014AA3D3E994
:10CD8800002306F059F8002800F02781DDE90601A4
:10CD980041A3D3E9002306F031F8002800F01D81F3
:10CDA80043A3D3E90023DDE9060105F0B5FD0246FA
:10CDB8000B4600204E4905F0FBFB06F047F857E00C
:10CDC800464B1868464B3A461968FFF737FA3AA3B4
:10CDD800D3E900230446DDE9040106F02DF850B13B
:10CDE8009DED040B08F04CF8002251EC100B414B60
:10CDF80005F092FDDCE0C825DDE031A3D3E900238E
:10CE0800DDE9080105F088FD2FA3D3E9002305F02B
:10CE1800ADFE06F063F8314B08EE100A1868304B87
:10CE28003A461968FFF70AFADFED337A4AEE677A6D
:10CE3800274BFDEEE77ADB6817EE905A044625EAA1
:10CE4800E57553B1234B1888234B4FF6FF761988A5
:10CE58000096A2B2ABB2F9F725F9BDEEC88A1E4B0F
:10CE680018EE102A1D606FF0B300B421FFF706FA20
:10CE7800174BDB68054653B1164B18881F4B4FF408
:10CE8800FC6619880096A2B2ABB2F9F70BF91B4BF6
:10CE9800A0E000BFAFF300809A9999999999B93F9A
:10CEA8000000000000409F409A9999999999B9BF4C
:10CEB8000000000000408F4089B5F81400E3693F86
:10CEC80000000000008076401F85EB51B81E194015
:10CED800B80D0020D83800207C3B0020F026002028
:10CEE800082D00201C0300200000000000006940FD
:10CEF80000005940000054C000004843C8360020D4
:10CF08000000000000E063400000000000C05D4039
:10CF18003B4B187805F09AFC02460B46002039492D
:10CF280005F024FE05F0DAFF08EE100A05F0A0FC73
:10CF380041EC100B07F0A4FFB4EE489AF1EE10FA9A
:10CF4800C8BFB0EE489AB4EEC89AF1EE10FA5BEC9E
:10CF580010AB42D82C4B18682C4B3A461968FFF78F
:10CF68006DF9044619EE100A05F082FC41EC100B2D
:10CF780007F086FF5946504659EC108B05F0AEFF76
:10CF88009FED237A07EE900AC7EE277A17EE900AEC
:10CF980005F06EFC42464B4605F0BEFC02460B46C9
:10CFA80000201C4905F004FB00221B4B05F002FB86
:10CFB80005F04CFF0546194BDB6853B1184B188830
:10CFC800184B4FF6FF7619880096A2B2ABB2F9F764
:10CFD80069F8144B1D60124B1C60134B1B78022B15
:10CFE80009D043B14FF6FF7300930520DC213A4680
:10CFF8000023FFF779FA47B0BDEC068BBDE8F08F48
:10D008001C03002000005940F0260020082D0020B5
:10D0180000004843000069400000E03FB80D0020D0
:10D02800D83800207C3B0020FC2C002010B54FF4A1
:10D03800C770FAF743FEDB2805D14FF4C870FAF73A
:10D048003DFE84B219E041F2E104214644F20100B8
:10D05800FAF726FE44F20100FAF730FEA04214BFA8
:10D0680080244FF4007421B24FF4C870FAF718FE08
:10D078004FF4C770DB21FAF713FE204610BD024BB0
:10D0880000221A60704700BFE436002070EEA10A43
:10D0980088B030EE010A08B0704770EEE10A88B037
:10D0A80030EE410A08B07047F0EE407A20EEA10A4F
:10D0B80060EE810A47EEA10A88B017EE810A08B02F
:10D0C8007047D0B561EEA17A41EE017A2DED048B5F
:10D0D80017EE900A88B0B0EE409AF0EE609AF0EE43
:10D0E800418AB0EE618A05F0C3FB002200230646A0
:10D0F8000F4605F079FEE8B969EE887A49EE287A94
:10D1080029EE088A17EE900A05F0B2FB32463B4634
:10D1180005F02CFD19EEA88A05F0E0FE044618EE8D
:10D12800100A05F0A5FB32463B4605F01FFD05F049
:10D13800D5FE01E00448044600EE900A00EE104ACD
:10D1480008B0BDEC048BD0BD0050C347F0B58E4B82
:10D158002DED068B93ED001AD3ED011A8FB0F0EE8A
:10D16800408AB0EE608A8DED060ACDED070A30EEF2
:10D17800410A70EEE10A38EE811A78EE211A8DED37
:10D188000C1ACDED0D1A8DED0A0ACDED0B0AFFF73D
:10D1980098FF8DED040ACDED050A04AA92E8030074
:10D1A80008AB83E80300DDED099A9DED08AA69EE56
:10D1B800A97A4AEE0A7A17EE900A05F059FB41EC73
:10D1C800100B07F0E3FE51EC100B05F087FE09EE9B
:10D1D800100A19EE900A05F04BFB04461AEE100AE5
:10D1E8000D4605F045FB45EC104B41EC110B07F0E3
:10D1F800BFFD51EC100B05F071FE68EE087A48EEA1
:10D20800A87AB1EE48AAC8EEA79A604B604D5A6951
:10D218001B8B6860EA612B8404468AEE27AA85ED99
:10D22800009A19EE100AC5ED028A85ED038AC5ED4C
:10D23800049A85ED05AA05F01BFB4DA3D3E900234D
:10D2480005F0FAFDDFED537A002818BFB0EE679AB3
:10D25800B7EE007A79EE077A37EE497A4E4BC7EE89
:10D26800877A1B78033BC5ED067A042B71D8DFE873
:10D2780003F0032738664F0018EE100A05F0F8FA95
:10D28800044618EE900A0D4605F0F2FA06460F46D7
:10D2980047EC116B45EC104B07F06AFD36A3D3E958
:10D2A800002351EC100BCDE9004505F035FB324663
:10D2B800CDE902013B46394939480AF0B7F948E057
:10D2C80019EE900A05F0D4FA04461AEE100A0D4633
:10D2D80005F0CEFA2246CDE900012B463048314907
:10D2E8002AE019EE100A05F0C3FA41EC100B07F01A
:10D2F800C7FD00222C4B51EC100B05F00DFB05F07F
:10D30800EDFD05F0B5FA02460B46254827491EE013
:10D3180019EE100A05F0ACFA064620460F4605F04D
:10D32800A7FA17A3D3E9002305F0F6FACDE900011F
:10D338001B481F4932463B460AF078F909E017EEC8
:10D34800900A05F095FA02460B46154819490AF065
:10D358006DF9134C00230220CA212246F9F750F830
:10D36800002323700FB0BDEC068BF0BDAFF3008037
:10D37800AE47E17A14AEEF3F6666666666A64C4035
:10D38800F6285C8FC2A54C400C3700209C38002042
:10D398008C3A0020A4707D3FFC2C0020F3B70508D0
:10D3A800A03600200DB80508000034C01DB80508D7
:10D3B8002FB805084BB8050800B560EEA07A40EE16
:10D3C800007A2DED028B17EE900A87B0B0EE408AF6
:10D3D800F0EE608A8DED020ACDED030A05F048FAF9
:10D3E80041EC100B07F0D2FD51EC100B05F076FD67
:10D3F800DFED117A07EE100A78EEA78A38EE078A71
:10D4080068EEA87A48EE087AC7EE277A17EE900AEF
:10D4180005F02EFA41EC100B07F0B8FD51EC100B9B
:10D4280005F05CFD00EE900A20EE880A60EEA80A7E
:10D4380007B0BDEC028B00BD00000000F0B52DED7B
:10D44800028BDFED3A1A3A4B8DB030EEA17AF0EE4E
:10D45800407AB7EE001A8DED020A83ED001A30EE1D
:10D46800010AC3ED011A31EE671A71EEE01ACDED2B
:10D47800030AF0EE470A8DED077A8DED081ACDED17
:10D48800091A8DED060AFFF71CFE8DED000ACDED99
:10D49800010A9DE8030004AB83E803009DED058ABB
:10D4A800DDED048A68EE087A48EEA87A17EE900A4D
:10D4B80005F0DEF941EC100B07F068FD18EE100AD4
:10D4C80057EC106B05F0D4F9044618EE900A0D4697
:10D4D80005F0CEF945EC104B41EC110B07F048FC78
:10D4E8003946304655EC104B05F0F8FC05F0C0F90C
:10D4F80041EC100B07F03EFC002251EC100B0D4BD9
:10D5080005F00AFA05F0EAFC29460646204605F029
:10D51800E5FC00EE900AF6EE007A60EEA70A00EE4F
:10D52800106A0DB0BDEC028BF0BD00BF000000001A
:10D53800E43A00200000E03FF0EE407A86B020EEAA
:10D54800200A67EE810A06B070472DE9F04F2DEDED
:10D55800028B85B0FCF726F810EE105AFCF728F875
:10D56800284610EE104A05F083F980462046894681
:10D5780005F07EF941EC100B41EC180B07F09CFA12
:10D5880057EC106BB0EE480AF0EE680A07F094FB0F
:10D5980032463B46404649465BEC10AB05F0BCF9C9
:10D5A80005F09CFC9FED138A07EE100ADFED127A56
:10D5B80057EE087A114C5B46C4ED007A5246404655
:10D5C800494605F0A9F905F089FC07EE900A27EE0F
:10D5D800888A04AB84ED018A94E8030003E9030018
:10D5E800DDED030A9DED020A05B0BDEC028BBDE836
:10D5F800F08F00BF0000F04200008C42743B002016
:10D6080030B53F4B2DED088BD3ED008AD3ED019A51
:10D618003C4BD3ED00AAD3ED01BA3B4B93ED008A06
:10D6280093ED019A394B93ED00AA93ED01BA38EEC8
:10D63800EA0A79EEEB0A38EE4A1A79EE4B1A93B0F9
:10D648008DED0A0ACDED0B0A8DED0C1ACDED0D1AF4
:10D65800FFF72AFD8DED000ACDED010A9DE80300D4
:10D668003AEE6A0A7BEE6B0A04AB38EE681A79EE7A
:10D67800691A83E803008DED081ACDED091A8DEDBE
:10D688000E0ACDED0F0AFFF70FFD8DED000ACDED67
:10D69800010A9DE8030006AB83E803009DED040A38
:10D6A800DDED050A9DED061ADDED071AFFF709FD08
:10D6B8008DED000ACDED010A9DE8030002AD85E875
:10D6C8000300134B9DED021A93ED000AD3ED010AF6
:10D6D800DDED031AFFF7E8FC8DED000ACDED010A38
:10D6E8009DE8030012AB03E903006C46DDED110A67
:10D6F80085E803009DED100A13B0BDEC088B30BD22
:10D7080098360020F8360020683B0020F83A0020C0
:10D71800C0380020F7EE007A77EEC07A20EE022AB1
:10D7280020EE210A07EEA00AF0EE420A47EE810A2F
:10D7380088B008B070472DE9F0432DED028B924B6D
:10D748001B78012B89B08146884646D14FEAC0092B
:10D7580001291FFA89F92BD809F58065A8B2FAF7CB
:10D76800F1FA8A4C0435A8B284ED000AFAF7EAFA0D
:10D7780009F58645A8B284ED010AFAF7E3FA844C64
:10D78800043584ED000AA8B2FAF7DCFAA9F5FC40E2
:10D7980084ED010A80B2FAF7D5FA7E4CA9F5FA4071
:10D7A800FC3884ED000A80B2FAF7CCFA84ED010A5D
:10D7B80008F1FF385FFA88F8B8F1010F00F2DF804E
:10D7C800A9F57C5080B2FAF7BDFA734CA9F57A59DD
:10D7D80084ED000AA9F17C09CBE0022B40F0CF8050
:10D7E8006E4B6F4A1B68012992ED007A00F2AC80FB
:10D7F80007EE900AF8EE676A07EE903A46EE877AE7
:10D80800BDEEE77A17EE104AA4B207EE104A04F10B
:10D818008005ED00B8EE478AADB2284637EEC88AD3
:10D82800FAF790FA0435A8B204F50665EE008DED16
:10D83800020AFAF787FAB6B230468DED030AFAF70C
:10D8480081FA043604F58257B0B28DED040AFE0061
:10D85800FAF778FAB6B230468DED050AFAF772FA99
:10D868000436B0B281348DED060AE400FAF76AFA9C
:10D87800A4B220468DED070AFAF764FA434E043441
:10D88800A0B286ED000AFAF75DFA6C1CE400A4B2B7
:10D89800204686ED010AFAF755FA3D4D0434A0B248
:10D8A80085ED000AFAF74EFA7C1CE400A4B2204683
:10D8B80085ED010AFAF746FA364F0434A0B287ED2F
:10D8C800000AFAF73FFAD6ED001A96ED012ADDEDC7
:10D8D800020AF0EE408A87ED010A9DED031AB0EEC8
:10D8E800480AFFF717FF8DED000ACDED010A9DE804
:10D8F8000300D5ED001A95ED012AB0EE480ADDEDDA
:10D90800040A86E803009DED051AFFF703FF8DED75
:10D91800000ACDED010A9DE80300D7ED001A85E85D
:10D928000300B0EE480ADDED060A9DED071AB0EED9
:10D93800682AFFF7EFFE8DED000ACDED010A9DE89C
:10D94800030087E803006C4608F1FF385FFA88F89F
:10D95800B8F1010F13D809F5C1594FEAC9091FFADF
:10D9680089F94846FAF7EEF90B4C84ED000A09F1FB
:10D9780004091FFA89F0FAF7E5F984ED010A09B0FC
:10D98800BDEC028BBDE8F083C9010020683B002094
:10D99800F8360020F83A0020983600206C2600203F
:10D9A800AC2600202DE9F04F6E4B2DED048B1C7832
:10D9B800012CC7B0054605D006D3022C0CBF302475
:10D9C800002402E0002400E010244FF47670FAF7F7
:10D9D80075F907464FF47570FAF770F980464FF4F9
:10D9E8007470FAF793F9032DC0B21D9040F094803B
:10D9F8005D4A5E4924A809F019FEC1B224A8FDF7C2
:10DA0800FFFB3B4642465A4924A809F00FFEC1B223
:10DA180024A8FDF7F5FB574A544924A809F006FE47
:10DA2800C1B224A8FDF7ECFB04F1C800FAF76EF9BF
:10DA3800064604F1CC00FAF769F9054604F1D0006E
:10DA4800FAF764F9074604F1D400FAF75FF9AB1B5B
:10DA580006EE903AB8EEE67A06EE907AF8EEE67AB6
:10DA68002B46C7EE277A324601904349009724A8EF
:10DA7800FDEEE77ACDED027A09F0D8FDC1B224A80F
:10DA8800FDF7BEFB3D4A394924A809F0CFFDC1B2D4
:10DA980024A8FDF7B5FBE820FAF738F90546EC208D
:10DAA800FAF734F90446F020FAF730F90646F4207C
:10DAB800FAF72CF9631B07EE903A06EE906AB8EE77
:10DAC800E77AF8EEE67A2A46C7EE277A01902A49DD
:10DAD8000096234624A8FDEEE77ACDED027A09F0F8
:10DAE800A5FDC1B224A8FDF78BFB1D9A022A06D119
:10DAF800234924A809F0C2FD24A8142109E01D9B8C
:10DB0800012B40F089821F4924A809F0B7FD24A8F9
:10DB18001021FDF775FB7FE21D9A012A40F00E8166
:10DB280004F1C800FAF7F2F81B9004F1CC00FAF7F8
:10DB3800EDF8074604F1D000FAF7E8F81B9B1C90B3
:10DB4800FF1A06EE907AB8EEE67A06EE900AF8EE3C
:10DB5800E67A0024C7EE277AFDEEE77ACDED1F7A44
:10DB6800E7E000BF1C0E00205BB8050856B80508A2
:10DB780065B8050872B8050878B80508C2B8050878
:10DB8800C8B80508DDB805081C9B1B9A204601216A
:10DB980003FB042AFFF7CFFD914B924A18681768D8
:10DBA800D3ED018A92ED019A8F4B904AD3F80090F9
:10DBB800D3ED019A1368012D209392ED018A7ED14D
:10DBC800F5EEC08AF1EE10FA54BF4FF0000C4FF09A
:10DBD800010CB5EEC09ABCF1000F0CBF4FF02B083A
:10DBE8004FF02D08F1EE10FA54BF4FF0000E4FF031
:10DBF800010EF5EEC09ABEF1000F0CBF2B262D26A4
:10DC0800F1EE10FA54BF00210121B5EEC08A0029B7
:10DC18000CBF4FF02B0B4FF02D0BF1EE10FA54BF49
:10DC280000220122002A0CBF2B232D231E93BCF1B6
:10DC3800000F01D0F1EE688ABEF1000F01D0B1EEFD
:10DC4800499A09B1F1EE699A0AB1B1EE488A04F02D
:10DC58000FFECDE9000118EE900ACDF8088004F017
:10DC680007FECDE90401384604F002FECDE90601BD
:10DC780019EE100A089604F0FBFDCDE90A014846A2
:10DC880004F0F6FDCDE90C0119EE900ACDF838B094
:10DC980004F0EEFDCDE91001209804F0E9FD1E9A8C
:10DCA800CDE9120118EE100A149204F0E1FD524673
:10DCB800CDE9160124A84E4909F0B8FC2FE0022D41
:10DCC8002ED1FFF79DFC8DED220ACDED230A22AB64
:10DCD80093E8030046AB03E90300DDED457AF5EE72
:10DCE800C07AF1EE10FA449805D5F1EE677A17EE8E
:10DCF800906A2D2702E017EE906A2B2704F0B8FDF2
:10DD080002460B463046CDE90023029704F0B0FDE9
:10DD18005246CDE9040124A8364909F087FCC6B269
:10DD280024A83146FDF76CFA0120FDF787FF01347E
:10DD3800A4B21F9BA342BFF627AF6AE11D9A022A2D
:10DD480040F06781E820F9F7E1FF1B90EC20F9F734
:10DD5800DDFF0646F020F9F7D9FF1B9B1C9006EE65
:10DD6800900AF61AB8EEE68A06EE906AF8EEE67AB7
:10DD780004F1C800C7EE887AFDEEE77ACDED1E7A89
:10DD8800F9F7C4FF064604F1CC00F9F7BFFF0746D0
:10DD980004F1D000F9F7BAFFBF1B07EE100A06EE30
:10DDA800907AF8EEC77AB8EEE67A1B9A1F9087EE5B
:10DDB800277A931B012D06EE903ABDEEC77A88EEBE
:10DDC800278A0D4B8DED207AB8EEE67A87EE277A12
:10DDD80083ED007A094B83ED008A40F0D0808FE014
:10DDE800683B0020F8360020F83A002098360020DA
:10DDF800EEB8050829B905086C260020AC260020D5
:10DE08001F9A002102FB046220462192FFF793FC2F
:10DE180095ED018AD8ED018AB5EEC08AF1EE10FAC7
:10DE280054BF4FF0000C4FF0010CF5EEC08A9AED8C
:10DE3800019ABCF1000F0CBF2B272D27F1EE10FA29
:10DE480054BF4FF0000E4FF0010EB5EEC09ABEF170
:10DE5800000F0CBF4FF02B0B4FF02D0BF1EE10FA0B
:10DE680054BF002101212868D8F80090DAF8003062
:10DE780000290CBF2B222D22BCF1000F01D0B1EEDE
:10DE8800488ABEF1000F01D0F1EE688A09B1B1EEFF
:10DE9800499A19921A9304F0EBFCCDE9000118EEA7
:10DEA800100A029704F0E4FCCDE90401484604F0A6
:10DEB800DFFCCDE9060118EE900ACDF820B004F099
:10DEC800D7FC1A9BCDE90A01184604F0D1FC199A2F
:10DED800CDE90C0119EE100A0E9204F0C9FC219A42
:10DEE800CDE910014F4924A809F0A0FBC1B224A82C
:10DEF800FDF786F901340120FDF7A0FEA4B205E084
:10DF0800494DDFF83481DFF834A10024209BA34277
:10DF1800BFF676AF0024454D2DE01C9B1B9A20468A
:10DF2800022103FB0426FFF706FC95ED018AB5EEF6
:10DF3800C08AF1EE10FA286803D5B1EE488A2D2779
:10DF480000E02B2704F094FCCDE9000118EE100A3C
:10DF5800029704F08DFC3246CDE90401344924A827
:10DF680009F064FBC1B224A8FDF74AF90120FDF7C6
:10DF780065FE0134A4B21E9BA342CEDA49E0022D0D
:10DF880047D142E01C9B1B9A0121204603FB042534
:10DF9800FFF7D1FBFFF734FB8DED220ACDED230A05
:10DFA80022AB93E8030046AB03E90300DDED457AB5
:10DFB800F5EEC07AF1EE10FA449806D5F1EE677ADC
:10DFC80017EE908A4FF02D0903E017EE908A4FF074
:10DFD8002B0904F04DFC06460F464046CDE9006784
:10DFE800CDF8089004F044FC2A46CDE90401104914
:10DFF80024A809F01BFBC1B224A8FDF701F90134DC
:10E008000120FDF71BFEA4B200E000241E9BA342E2
:10E01800B8DA084B1D9A1A7047B0BDEC048BBDE8FE
:10E02800F08F00BF3DB90508683B002098360020F6
:10E038006BB90508C9010020F8360020F83A00201D
:10E04800F0B52DED028B04468FB0002800F0418119
:10E05800AB4B18890419A4B222B2002A05DB40F29E
:10E068003F139A42C8BF1C4600E00024F7F73EFA67
:10E07800A0B24EF29C71F7F74BFAA14B1C81A14B51
:10E08800586804F0F5FB96A3D3E9002304F044FC98
:10E0980004F024FF9C4B18609C4B1B780A2B054608
:10E0A8003DD123B206EE903AF8EEE67A17EE900AE2
:10E0B80004F0DEFB964B064618680F4604F0C6FBD4
:10E0C80002460B4688A1D1E9000104F04FFD024643
:10E0D8000B463046394604F01FFC064628460F46D4
:10E0E80004F0C6FB02460B463046394604F014FCE1
:10E0F8000022884B04F03AFD04F0F0FE04F0B8FB6F
:10E1080002460B4604A8844909F090FA0020F8F763
:10E118003FF90520D72104AA0023F8F771F97B4BB2
:10E128001B780D2B7D4B188824B200FB04F067D1B7
:10E1380004F08CFB6EA3D3E9002304F017FD04F070
:10E14800CDFE774B1B6806EE903A07EE900AB8EEC4
:10E15800E67A744B27EE877AFCEEE77ABDEEC77A4B
:10E1680017EE900A17EE104A1B68012180B2E418D6
:10E17800FFF7E1FA6C4BD3ED017A6C4B93ED018A12
:10E188006B4B93ED017A38EE678A77EE677A88EE03
:10E19800278A18EE100A04F06BFB57A3D3E9002373
:10E1A80004F036FEDFED637A002818BFB0EE678A08
:10E1B80018EE100A04F05CFB41EC100B06F060FE50
:10E1C800002251EC100B5C4B04F0A6FB04F086FE19
:10E1D80004F04EFB02460B4606A8584909F026FAF9
:10E1E8009620DC2106AA0023F8F70AF94FF6FF73F8
:10E1F80000930520DC2122460023FEF775F968E02C
:10E2080004F024FB3AA3D3E9002304F0AFFC04F0A4
:10E2180065FE434B1B6806EE903A08EE100AF8EECE
:10E22800E67ABCEEC87A68EE277A17EE105AFDEE49
:10E23800E77A3C4B17EE906A1B68ADB2284601217D
:10E24800F618FFF778FAFFF7DBF98DED020ACDED46
:10E25800030A02AC94E803000AAB83E80300681CD5
:10E2680080B20121FFF767FAFFF7CAF98DED020ABC
:10E27800CDED030A94E803000EAB06EE905A03E9CD
:10E288000300B8EEE60ADDED0A0A38EE400A9DED15
:10E298000B1ADDED0C1A9DED0D2AFFF73BFA8DEDFB
:10E2A800020ACDED030A94E8030008AB83E80300F3
:10E2B8004FF6FF73009305200023DC213246FEF75A
:10E2C80013F91F4B9DED080A1878DDED090AFEF7D2
:10E2D8003DFF0FB0BDEC028BF0BD00BFAFF3008077
:10E2E8007B14AE47E17A843F000000A0D954BD41B9
:10E2F8000000000000F07340FCA9F1D24D62503FCD
:10E30800B80D00201C0300205C3B00207126002073
:10E31800082D00200000F43F7EB90508DC3A0020F3
:10E32800E42C0020F0260020F83600209836002043
:10E33800F83A00206F12833A0000344087B9050884
:10E34800FC2C00202DE9F843461F8846B6B200256C
:10E358000D4F12E008EB040189B23046F7F77AF85E
:10E3680029F814000A200134FAF7A8FE062CF1D186
:10E3780016350136F22DB6B204D06FF0040407EB5F
:10E388000509E7E7BDE8F883183B00202DE9F04FC1
:10E3980085B00B1A0193431E9BB20293431C441F82
:10E3A80000F1060901F1FF3A01F1010B9BB20F469A
:10E3B8001646A4B21FFA89F91FFA8AFA1FFA8BFBCC
:10E3C80003938046204651463246F7F77BF82046AD
:10E3D80039463246F7F776F8204659463246F7F777
:10E3E80071F8019B0298E518ADB229463246F7F755
:10E3F80069F8404629463246F7F764F8013403982D
:10E4080029463246F7F75EF8A4B20A20FAF756FE14
:10E418004C45D7D105B0BDE8F08F2DE9F843461F2C
:10E428008846B6B200250E4F12E008EB040139F811
:10E43800142089B23046F7F745F801340A20FAF774
:10E448003DFE062CF1D116350136F22DB6B204D0B8
:10E458006FF0040407EB0509E7E7BDE8F88300BFA0
:10E46800183B00202DE9F0432DED068B70EE007A65
:10E478008DB017EE900AB0EE408A10EE904A20EE6A
:10E48800009A04F0F5F9064620460F4604F0F0F924
:10E49800F7EE008A41EC100B41EC1A0B06F00CFB6E
:10E4A80079EE287A55EC104B17EE900A04F0E0F953
:10E4B8002246804689462B463046394604F02CFAD7
:10E4C80002460B464046494604F072F804F006FD41
:10E4D800B0EE4A0AF0EE6A0A09EE900A38EEC99AD6
:10E4E800DFED377A89EE299A29EE279A06F0E4FBC0
:10E4F800304653EC102B394604F00EFA044619EE58
:10E50800900A0D4604F0B4F902460B462046294607
:10E5180004F02CFB00222B4B04F0FEF904F0DEFC87
:10E52800B4EE688ADFED287A284BF1EE10FA04463B
:10E5380019EE100A08BFB0EE678A1D6804F098F952
:10E5480002460B4603A8224909F070F8204604F059
:10E558008FF902460B4606A81E4909F067F878EEBF
:10E56800287A38EEC88A87EE888A18EE100A04F0EE
:10E578007FF902460B4609A8174909F057F8052004
:10E58800014603AA0023F7F73BFF0520142106AA3A
:10E598000023F7F735FFC820052109AA0023F7F75C
:10E5A8002FFF4FF6E07300930520DC212A46002355
:10E5B800FDF79AFF0DB0BDEC068BBDE8F08300BFF8
:10E5C8000000484200004940A4707D3FB838002050
:10E5D80090B9050898B90508A0B905082DE9F04FC4
:10E5E800494B2DED048B1D78022D85B080467BD1DB
:10E5F800464E348A01212046FFF79DF8FFF700F8C0
:10E608008DED000ACDED010A9DE8030004AB03E996
:10E61800030028469DED020ADDED030AFEF796FD8C
:10E628003B4B1A683B4B1B6802FB04343A4B1C609B
:10E638003A4BDFED3B7A93ED008A68EE277A5F6804
:10E6480017EE900A04F014F9824638468B4604F017
:10E658000FF941EC100B41EC190B06F02DFA50465E
:10E6680053EC102B594604F057F923A3D3E90023A0
:10E6780003F0A0FF04F012FCB0EE490AF0EE690ABC
:10E68800054684B206F018FB504653EC102B594649
:10E6980004F042F90B46024619A1D1E9000103F042
:10E6A80087FF04F0FBFBB37C81461FFA80FA1BB995
:10E6B800B08AF18AFFF7B1FE002320465146B374B1
:10E6C800FFF740FE204651461F22FFF75FFEB0EEDF
:10E6D800480A00EE907AFFF7C5FE338AB58298445F
:10E6E800A6F81080A6F8169005B0BDEC048BBDE81E
:10E6F800F08F00BFAFF300800000000000E063402F
:10E708000000000000C05D40FC2C0020B80D002077
:10E71800E42C0020F0260020B83800208C3A002095
:10E728000000C842124B1B78022B10B50CD1114BBC
:10E738001B78022B08D1104C2078C0B140B2FFF7EB
:10E748004DFF0023237010BD0C4C237E23B99F205E
:10E75800F6F7A6FE01232376064B1B78022B06D17B
:10E76800054C94F90000FFF76BFC0023237010BDE3
:10E77800FC2C0020E4380020251B0020B80D0020C8
:10E78800034B00201860034B1870FDF797BB00BFC0
:10E79800E4360020E4380020034B00201860034BC7
:10E7A80002221A70FDF78ABBE4360020E438002004
:10E7B80037B500242546A0B2282132230246013469
:10E7C8000095F7F76FFCB4F5A07FF4D13EBD2DE9B5
:10E7D800F04F2DED088B022897B080468DED070A83
:10E7E800B34B05D0032805D0012805D10C2202E03F
:10E7F800092200E00B221A701878F2F70FFA0421A8
:10E8080003914FF00009F3EE0EAA9FEDAABADFEDCF
:10E81800AABA7DE1A94B1A68A94B1B6802FB093308
:10E8280007EE103A01211FFA89F0B8EEC78AFEF701
:10E8380082FFFEF7E5FE8DED080ACDED090A08AD69
:10E8480095E803000AAB83E803009E4B1A6802EBC5
:10E85800C9030EAF19689C4B1960039952181268C6
:10E868005A60FEF7CDFE8DED080ACDED090A95E850
:10E8780003000CAB83E80300DDED0A9A9DED0BAABB
:10E88800DDED0C8A9DED0D9AB0EE690AF0EE4A0AAC
:10E89800B0EE681AF0EE491AFEF706FC8DED080A8C
:10E8A800CDED090A95E80300B0EE691AF0EE4A1AB0
:10E8B80087E80300B0EE680AF0EE490AFEF701FCAB
:10E8C8008DED080ACDED090A95E8030010AB83E841
:10E8D80003009DED0E0ADDED0F0AFEF76DFD8DEDCF
:10E8E800080ACDED090A95E8030016AA02E9030013
:10E8F8009DED100ADDED110A149EFEF75DFD8DED0C
:10E90800080ACDED090A95E8030087E80300DDED64
:10E918000F0AF5EEC00AF1EE10FA48BFF1EE600AF0
:10E928009DED0E0ACDED0F0AFEF788FD8DED080A64
:10E93800CDED090A08AA92E8030012AB83E80300A8
:10E948000798129D03F094FF5D4B139FD3F800B016
:10E958005E4BBDEEC87AD3F800A0CDE9040117EEEE
:10E96800102A58465146FDF769FC07EE10AAF8EE42
:10E97800C77A07EE10BAB4EEE78AF8EEC77AF1EE76
:10E9880010FAB4EEE78A8CBF00220122504B0690A1
:10E99800F1EE10FAD4BF002202F00102B8F1020F22
:10E9A800DA6012D0B8F1030F3ED0B8F1010F68D188
:10E9B800304603F05DFF36A3D3E9002303F0ACFF34
:10E9C8000022444B03F0F6FD2AE0284603F050FFEE
:10E9D800DDE9042304460D462FA1D1E9000104F026
:10E9E800C5F802460B462046294603F095FF2CA39E
:10E9F800D3E9002303F090FF04F070FA07EE900AC1
:10EA0800C7EEAA7A17EE900A03F032FF41EC100B1A
:10EA180006F036FA002251EC100B2F4B03F07CFF66
:10EA280004F014FA04462CE018EE100A03F020FF54
:10EA3800044638460D4603F01BFF17A3D3E900230D
:10EA480003F06AFFDDE9042304F090F804F046FAC5
:10EA580003F00EFF14A3D3E9002303F05DFF024681
:10EA68000B462046294604F081F804F037FA07EEF1
:10EA7800900AB0EE6B7A07EE8B7AFDEEC77A17EE46
:10EA8800904A002C2ADBC72CA8BFC72427E000BF68
:10EA98008716D9CEF753F5BF8FC2F5285CAF434030
:10EAA800000000000090704000000080DBC4864138
:10EAB800FC2C00200000C8C30000C843E42C002040
:10EAC800F0260020D036002098360020082D00209F
:10EAD800B80D002000006940000049C00024114B17
:10EAE800DB685BB1104B1888104B1988069B4FF6F2
:10EAF800FF759AB2A3B20095F7F7D4FA0B4B039AB5
:10EB08001C600699084B0832196009F10109039243
:10EB1800074B1B884B45BFF67DAE17B0BDEC088B85
:10EB2800BDE8F08FB80D0020D83800207C3B0020CD
:10EB3800DC3A00202DE9F0432E4B85B01878F2F727
:10EB48006DF82D4B0B221A702C4B1C78012C05D01C
:10EB580006D3022C0CBF3024002402E0002400E07D
:10EB68001024274B1B78012B07D104F1C800F9F7B3
:10EB7800CDF8064604F1D00004E0E820F9F7C6F81D
:10EB88000646F020F9F7C2F800240746DFF880901F
:10EB98001C4DDFF8808020E007FB0463204601213C
:10EBA8006B61A8F82040FEF7C6FDFEF729FD8DED44
:10EBB800000ACDED010A9DE8030004AB03E9030058
:10EBC8000C4B9DED020A1878DDED030AFEF7BEFA3C
:10EBD8006869FDF733FD0134A4B2B9F80030A342E7
:10EBE800DADA094B02221A70084B00221A7605B0AD
:10EBF800BDE8F083FC2C0020712600201C0E0020AC
:10EC0800C90100209C380020E4380020B80D0020FD
:10EC1800DC3A00208C3A00201FB5044600214FF052
:10EC2800804002F0D4FE2E4B18682E4B1B6800FB68
:10EC380004302D4B1B68984209DB2C4B1B6898420B
:10EC480005DCFAF73BFE2A4B1868FCF7F7FFFCF7E0
:10EC580027FF284A284B1168526819605A60214BCF
:10EC68001A68214B1B68D31A06EE903A1C4B1B6896
:10EC7800B8EEE67A06EE903AF8EEE67A0021C7EEAC
:10EC8800277AFCEEE77A17EE904AA0B2FEF753FD1A
:10EC9800FEF7B6FC8DED000ACDED010A9DE80300F4
:10ECA80004AB03E90300154B9DED020A1878DDED6E
:10ECB800030AFEF74BFA124B1868124B1B6824B272
:10ECC80000FB0430FDF7BAFC0F4B00224FF08040E8
:10ECD80001211A7004B0BDE8104002F078BE00BFF0
:10ECE80068260020D8360020E4260020D4260020FC
:10ECF8009C2600209C38002098360020FC2C002000
:10ED0800E42C0020F02600209526002008B5FFF707
:10ED180083FF0A4B1A680A4B1B689A420CDD4FF0B6
:10ED28008040002102F053FE064B02221A70064A68
:10ED380000231370054A137608BD00BFD83600209B
:10ED4800D4260020E438002095260020B80D0020A5
:10ED580010B500214FF0804002F039FE0A4B002424
:10ED68001C700A4B20461C70F7F73CFA084B1868D1
:10ED7800FAF7A4FD074B084801221A70074B1C70CC
:10ED8800BDE81040F2F7DBBF95260020E8360020EA
:10ED9800E4260020FC2C0020A0180020712600206A
:10EDA80007EE100A034BF8EE477A0022C3ED007A0B
:10EDB8005A6070470C37002007EE100A034BF8EE34
:10EDC800477A0022C3ED007A5A607047C0380020A5
:10EDD8000F4B10491A68104B1B68D31A06EE903A6D
:10EDE8000E4B1B68B8EEE67A06EE903AF8EEE67A35
:10EDF800C7EE277AFCEEE77A17EE903A9AB20B80C4
:10EE0800074B188890422CBF00200120704700BF94
:10EE1800082D0020DC3A0020F0260020E42C0020F9
:10EE2800E826002013B502AB011D23ED010A054AAF
:10EE380089B213F8014B1454013080B28842F8D1DA
:10EE48001CBD00BF1A3800202DE9F8431F4F0740AA
:10EE5800002F04460D4603DA013F67F00F0701371C
:10EE6800BFB2DFF874804FEAC7091FFA89F948462C
:10EE780098ED000A09F10409FFF7D4FF1FFA89F099
:10EE880098ED010AFFF7CEFF114B10261B8894FB63
:10EE9800F6F6F6019C42B6B20CD1701980B20D4953
:10EEA8008022FAF7ABF900B1FEE721B24FF47F7088
:10EEB800F8F7F6FE0F2F07D17519A8B20549802279
:10EEC800FAF79CF900B1FEE7BDE8F8830F0000806F
:10EED800DC3A00201A3800209C3800202DE9F04345
:10EEE800744B2DED028B1888FF2898BF4FF4807063
:10EEF80093B0C00008F028F86F4B0546186028B991
:10EF08000520B4216D4A2B46F7F77AFA0024694F99
:10EF18006B4E4FF000086AE0FCF7C2FD20464FF444
:10EF28004141FFF791FF674B1A685B683260002127
:10EF380073602046FEF7FFFBFEF762FB8DED020AC9
:10EF4800CDED030A0DF1080999E803000AAB83E83F
:10EF580003005D4B9DED0A1A93ED007AD3ED017A1B
:10EF6800DDED0B1A31EE470A71EEE70A31EE071AAA
:10EF780071EEA71A8DED0E0ACDED0F0A8DED101A60
:10EF8800CDED111AFEF79DF88DED020ACDED030ABD
:10EF980099E803000CAB83E80300FF2C4FEAC40395
:10EFA8002B4404D9C3F80080C3F8048003E00C9A0A
:10EFB8001A600D9A5A603B8840F23F10604390FBFC
:10EFC800F3F080B24FF4FC63024628210093322309
:10EFD800F7F768F83D4B18683D4B1B68C018FAF7FF
:10EFE8006DFC3C4B1868FCF729FE0134A4B23B8841
:10EFF800A34291DA012213464FF4807105A805F067
:10F008004DF8354EDFF8F880294605A805F028FBAD
:10F0180008233370314B01241C700020F6F7B0FB35
:10F028002F48F2F78CFE3078F1F7F8FD2D4B9FED65
:10F038002E8ADFED2E8A1C700024D5ED007AB0EE02
:10F04800687A07EEC87A2046FCEEC77A17EE906A0F
:10F0580003F0FCFB264B002203F05EFC03F01EFFCE
:10F06800B6B2A3B2C72E28BFC72687B253B1214B69
:10F07800B8F8000019884FF6FF7300933A463346F4
:10F08800F7F710F81B4BC8F8007001340835B4F5D1
:10F09800807F1E60D1D1184B1868FAF70FFC114B0E
:10F0A80002221A70154B00221A7613B0BDEC028B9F
:10F0B800BDE8F083DC3A0020D036002049B10508CD
:10F0C800983600209C3800200C370020D8360020C5
:10F0D800682600209C260020FC2C00207B0D0020A8
:10F0E800FC170020E4380020000016430000C84246
:10F0F8000000F43F7C3B0020E4260020B80D0020EF
:10F10800D8380020F0B5294B294F2A4D2A4E012224
:10F1180085B01A7000243AE0284B1A68336802FB5D
:10F1280004336B61264B1C84FCF7BAFC20464FF471
:10F138004141FFF789FE234B2A681A606A68204616
:10F148005A600021FEF7F7FAFEF75AFA8DED000A29
:10F15800CDED010A9DE8030004AB03E903001A4B57
:10F168009DED020A1878DDED030AFDF7EFFF6869E7
:10F17800FDF764FA154B1868154B1B68C018FAF7A9
:10F188009DFB144B1868FCF759FD0134A4B23B8869
:10F19800A342C1DA104B1868FAF790FB034B02221E
:10F1A8001A700E4B00221A7605B0F0BDE438002024
:10F1B800DC3A00209C380020F0260020E42C0020B7
:10F1C8008C3A002098360020FC2C0020D8360020ED
:10F1D800682600209C260020E4260020B80D002088
:10F1E80038B5FDF7E3F80F4B0F4C9F221A810F4BF0
:10F1F800012518782570F1F711FD0D4B00221A60D2
:10F208000C4B1B78072B04D00B2B07D0062B08D1EF
:10F2180002E0BDE8384075E7257038BDBDE83840E4
:10F2280088E438BDB80D0020E4380020FC2C00200C
:10F23800E4360020712600202DE9F7430025814699
:10F248002C46154E154FDFF85C801FE0FCF728FCB4
:10F2580049462046FFF7F8FDD8F800303868C0184E
:10F26800FAF72CFB0E4B1868FCF7E8FC308895FB86
:10F27800F0F080B24FF4FC63009328210246322359
:10F28800F6F710FF05F59E75013403353388A34260
:10F29800DCDABDE8FE8300BFDC3A0020D836002067
:10F2A8009C2600206826002010B5104C4FF475707D
:10F2B800B4F90010F8F7F4FC0D4B4FF47670B3F97D
:10F2C8000010F8F7EDFC40F2D230F8F7F7FCB02860
:10F2D80004D040F2D230B021F8F7E2FC2088FFF7E2
:10F2E8005FFD034B1888BDE8104065E5C4010020A8
:10F2F800C001002000210A2208B509F0E7FAD0F180
:10F30800010038BF002008BD73B5041D0E46A4B225
:10F318000C2200234FF6E075204601360095F6F7DB
:10F3280065FF00230C22B1B220460095F6F75EFF78
:10F338000D4B1B78012B16D10C4E0D4D30882988AA
:10F348000024043080B20C2223460094F6F74EFFC6
:10F358003088298800940430013180B289B20C22A7
:10F368002346F6F743FF7CBDBC3600200A37002051
:10F37800BC38002008B54FF6FF70F6F707FF0020ED
:10F38800F7F706F8E12023212C4A0023F7F738F88D
:10F39800E1204621294A0023F7F732F8E1206921C4
:10F3A800264A0023F7F72CF8E1208C21244A002371
:10F3B800F7F726F82348FFF79DFF20B12148224997
:10F3C800012208F033F94B2023211E4A0023F7F7C6
:10F3D80017F81E48FFF78EFF20B11C481A49012272
:10F3E80008F024F94B204621184A0023F7F708F8BB
:10F3F8001748FFF77FFF20B115481349012208F08D
:10F4080015F94B206921124A0023F6F7F9FF114834
:10F41800FFF770FF20B10F480B49012208F006F9E9
:10F428004B208C2100230B4AF6F7EAFF0A4B188879
:10F438000A4B1988BDE8084066E700BF59AF0508C0
:10F44800ACB90508B4260020CFAC0508D8260020A2
:10F45800EE2C0020A0260020F43A0020BC3A002020
:10F4680070B5044600200D461646F6F791FF0020B9
:10F47800F6F7A2FE4FF4FC60F6F788FE2046294610
:10F4880056BB1E4A3346F6F7BBFF1D48FFF732FF4F
:10F4980020B11B481B49012208F0C8F804F1700686
:10F4A800B6B230462946164A0023F6F7A9FF164891
:10F4B800FFF720FF20B114481249012208F0B6F8DE
:10F4C8003235ADB220462946104A0023F6F798FF98
:10F4D800304629460C4A07E00D4A0023F6F790FF0C
:10F4E80032350B4AA9B220460023F6F789FF094BAB
:10F4F8001888094B1988BDE8704005E7B1B90508B7
:10F50800603B0020F4B00508D03A0020B9B90508DE
:10F5180094B10508F43A0020BC3A002030B5144DE7
:10F528009DF80C402C70134D2880134D02FB0400ED
:10F538002980124D80B22880114D2980114D2A80D2
:10F54800114A1380114B1880114B1980114B124925
:10F55800E2B21A7000230B7010490A709DF810204F
:10F568000134013254430E4A14700E4A137030BDF0
:10F57800783C0020583B00209A380020F43A0020BC
:10F58800BC3A002018380020843B00200A370020AD
:10F59800BC380020BE3A0020E9360020F63A0020A8
:10F5A800C4360020BC36002038B5054600200C467D
:10F5B800F6F7EEFE0020F6F7FFFD4FF4FC60F6F7D5
:10F5C800E5FD0B48FFF796FE28B1094809490A4BA3
:10F5D800002208F02BF8284621460023044AF6F7B3
:10F5E8000FFF064B1888064B1988BDE838408BE694
:10F5F80000370020C5B505080000F03FF43A0020A8
:10F60800BC3A0020114B1B68002B70B505460C4610
:10F6180004DA5B420E480F492D2202E00C480D49DE
:10F62800202208F003F80020F6F7B2FE0020F6F7D3
:10F63800C3FD4FF4FC60F6F7A9FD054A28462146AC
:10F648000023BDE87040F6F7DBBE00BFF03A0020AB
:10F65800C8380020C1B905080F4B10B519684FF418
:10F66800E170F8F73AFB40F23D114FF4E070F8F71B
:10F6780017FB0020F6F78CFE0020F6F79DFD4FF4EF
:10F68800FC60F6F783FD054A192064210023BDE8D4
:10F698001040F6F7B5BE00BFF03A0020C9B905081A
:10F6A80008B54FF4E070F8F709FB40F23D139842B3
:10F6B80005D14FF4E170BDE80840F8F727BB0020FA
:10F6C80008BD38B5054600200C46F6F761FE002057
:10F6D800F6F772FD4FF4FC60F6F758FD0B48FFF79C
:10F6E80009FE28B109480A490A4B002207F09EFF83
:10F6F800284621460023054AF6F782FE064B18885D
:10F70800064B1988BDE83840FEE500BFDC3600200E
:10F71800C5B505080000F03FF43A0020BC3A0020C7
:10F7280038B5C501ADB20024601980B2F9F70EFBF7
:10F738000134C0B2FBF754FDA4B24FF47A70F9F764
:10F74800BDFC802CF0D138BD73B5104D00240E20BF
:10F75800FBF746FD002609E00DF10700FBF751FD18
:10F7680020B19DF80730AB550136F6B23306F3D514
:10F77800E00180B205498022F9F740FD00B1FEE7BB
:10F788000134A4B2B4F5007FE1D17CBD1A38002061
:10F7980007EE100AF8EE477A7FB517EE900A03F0E5
:10F7A80067F802460B4601A8054907F03FFF0A2003
:10F7B800962101AA0023F6F723FE07B000BD00BF7B
:10F7C800D0B905082DE9F34700240746B0F5024FE4
:10F7D80014BF4FF0910A4FF0690A25462E4EA046F5
:10F7E8000DE094FBF0F080B2462102465023CDF89C
:10F7F8000080F6F757FC04F59E7401350334308811
:10F80800A842EEDA0020F6F7D7FC4FF4FC60F6F7D2
:10F81800BDFC00258C2051463F220023F6F7D2FD7F
:10F828002C461D4EDFF87C80DFF87C9027E0F9F746
:10F83800D1FE88ED000AF9F7D3FE394688ED010AB2
:10F848002046FFF701FB154B1868D9F8003000FB7C
:10F858000430FAF733F8124B1868FCF7EFF93088E0
:10F8680095FBF0F080B24FF4FC630093462102460A
:10F878005023F6F717FC05F59E75013403353388D8
:10F88800A342D4DA8C2051463C22002302B0BDE8C2
:10F89800F047F6F797BD00BFDC3A00206826002045
:10F8A8009C2600209C380020E426002070B53A4BA6
:10F8B8003A4E3B4D01222DED048B1A70394B002432
:10F8C8001C609FED399A55E0F9F784FEF0EE408A06
:10F8D800F9F786FE20464FF44141B0EE408A85EDA7
:10F8E800010AC5ED008AFFF7AFFAA0B20021FDF7C3
:10F8F80022FF2E4BD3ED017A2D4B93ED017A38EE92
:10F90800678A77EE677A88EE278A18EE100A02F07F
:10F91800AFFF1FA3D3E9002303F07AFA002818BF2A
:10F92800B0EE498A18EE100A02F0A2FF41EC100B63
:10F9380005F0A6FA002251EC100B1E4B02F0ECFF6A
:10F9480003F0CCFA1C4B18601C4B18681C4B1B6846
:10F9580000FB04306861FCF771FE1A4B18681A4BFB
:10F968001B6800FB0430F9F7A9FF184B1868FCF76F
:10F9780065F901343388A342A6DA154B9F221A8110
:10F9880000221A76044B02221A70BDEC048B70BD5B
:10F99800FCA9F1D24D62503FE4380020DC3A002047
:10F9A8009C380020E43600206F12833AF836002095
:10F9B800F83A002000003440C0360020E42C002033
:10F9C800F026002068260020E42600209C2600203F
:10F9D800B80D0020AFF300800EB403B070470A28BA
:10F9E80010B5044602D10D20FFF7F9FF064A136847
:10F9F8001BB103F8014B136010BD044B1B680BB11E
:10FA08002046984710BD00BFD80D00207C3C002040
:10FA180010B5044601E0FFF7E2FF14F8010B0028D7
:10FA2800F9D110BD2DE9F04F044685B00D464FF0D1
:10FA38000A0A00E035462078002800F0C48025280E
:10FA480001D0013467E06078302803D1A078012321
:10FA5800033407E02D2802D00234002302E0A07806
:10FA6800022303344FF0000805E00AFB080814F8E5
:10FA7800010BA8F13008A0F13002D2B2092AF4D95A
:10FA88006C2801D04C2803D114F8010B43F004036F
:10FA9800002800F09880602886BFA0F12002D2B22A
:10FAA80002464F2A3DD006D8432A2DD0442A09D0F1
:10FAB800422A30D133E0552A04D0582A29D0532A73
:10FAC80029D101E00A272DE02E1D2F68002500E02E
:10FAD80001357A5D002AFBD104E02020FFF77FFF83
:10FAE8004D4601E0980704D4454505F10109F4D3D2
:10FAF8004D463846FFF78CFF03E02020FFF76FFFE5
:10FB080001354545F9D395E728782E1DFFF767FF9E
:10FB180090E7102706E0FFF762FF2E468AE70227E4
:10FB280000E008272E1D442A296804D1002902DA9A
:10FB3800494243F00803002200E02A46B1FBF7FEE1
:10FB480007FB1E11CDB2092D714607D9782814BFBD
:10FB58004FF0070C4FF0270C6544EDB230350DF827
:10FB68000250551CBEF1000F02D0102DE5D10F2216
:10FB7800190705D504A94D192D2105F8101C951C48
:10FB880013F0010F0CBF4FF0200B4FF0300B9B0709
:10FB98002F4604D508E05846FFF721FF4F46474552
:10FBA80007F10109F7D34F46013D1DF80500FFF79E
:10FBB80016FF002DF8D103E02020FFF710FF0137D2
:10FBC8004745F9D336E705B0BDE8F08F70B5064D67
:10FBD8000C462E68286001E0FFF701FF14F8010BBE
:10FBE8000028F9D12E6070BD7C3C00200FB407B509
:10FBF80004A951F8040B0191FFF714FFBDE80E406A
:10FC080004B070470EB417B505A9084C51F8043B69
:10FC1800206018460191FFF705FF22680023137042
:10FC28002360BDE81E4003B0704700BFD80D002018
:10FC38000EB433B505A9074C51F8043B256820607C
:10FC480018460191FFF7EEFE2560BDE83C4003B081
:10FC5800704700BF7C3C002070B51E4604461C4817
:10FC68001546FFF7C3FF022E1FD0042E25D0012E04
:10FC78002AD105E0A15D1748FFF7B8FF013600E07B
:10FC88000026AE42F6DB2020FFF7A9FE002609E099
:10FC9800A05DA0F12003DBB25E2B88BF2E20FFF70A
:10FCA8009EFE0136AE42F3DB0EE034F8021B0A4832
:10FCB800FFF79CFF013DF8D106E054F8041B074804
:10FCC800FFF794FF013DF8D10A20BDE8704086E6B1
:10FCD800D7B90508DEB90508E4B90508EAB9050881
:10FCE80008B501214FF4807001F07CFA4FF4807060
:10FCF8000021BDE8084001F075BA43680A6823F09E
:10FD0800407323F4807313430A7943EA0223436060
:10FD1800CA680B6930B51A4384688D68084B2A4352
:10FD2800234013434A7943EA420383600B7DC26A46
:10FD3800013B22F47002DBB242EA0353C36230BDD6
:10FD4800FDF7FFC000230360037143718360C36044
:10FD58000361012303757047074A084B516810B5C2
:10FD68000B4090E8120021438468C0682143014396
:10FD78000B43536010BD00BF00230140E030FCFF7F
:10FD88000023036043608360C3607047836811B1D8
:10FD980043F0010301E023F00103836070474368E7
:10FDA80023F4400323F400730B434360704741621C
:10FDB80082627047436823F01F030B434360704718
:10FDC800044B5A6810B142F4000201E022F4000228
:10FDD8005A60704700230140044B5A6810B142F43E
:10FDE800800201E022F480025A607047002301403B
:10FDF800092970B50CB20CD904EB44041E3CC66842
:10FE08000725A54026EA0505A34045EA0304C46082
:10FE18000AE0066904EB44040725A54026EA05051F
:10FE280013FA04F42C430461062A0CD80523013A7A
:10FE38005A43446B1F23934024EA0303914043EA47
:10FE48000102426370BD0C2A12B20CD802EB820286
:10FE5800233A046B1F23934024EA0303914043EAA7
:10FE68000102026370BD02EB8202413AC46A1F2399
:10FE7800934024EA0303914043EA0102C26270BD41
:10FE8800836843F08043836070478068C0F3805084
:10FE98007047836811B143F4806301E023F4806301
:10FEA80083607047836811B143F0020301E023F0D7
:10FEB8000203836070474368013923F4604343EACF
:10FEC800413343607047436811B143F4006301E074
:10FED80023F4006343607047C06C80B27047014BE5
:10FEE8001868704708230140836811B143F4807390
:10FEF80001E023F4807383607047836811B143F491
:10FF0800007301E023F4007383607047044B5A6860
:10FF180010B142F4005201E022F400525A607047D6
:10FF280000230140092970B50CB20CD904EB440434
:10FF38001E3CC6680725A54026EA0505A34045EAF4
:10FF48000304C4600AE0066904EB44040725A540DD
:10FF580026EA050513FA04F42C430461836BC3F302
:10FF68000154121B0232D2B202EB82021F249440C7
:10FF780023EA040391400B43836370BD836B01390B
:10FF880023F4401343EA01538363704782B000238C
:10FF980001930190019BCB180193019B1A6002B059
:10FFA8007047836823F470230B438360704783682A
:10FFB80023F440130B4383607047836843F4800342
:10FFC800836070478068C0F380507047436811B100
:10FFD80043F4806301E023F480634360704743681F
:10FFE80011B143F4805301E023F480534360704718
:08FFF80082B000230193019087
:020000040801F1
:10000000019B28335B180193019B186880B202B0F2
:1000100070470123C9B213FA01F143680AB11943C9
:1000200001E023EA010141607047036819420CBFF7
:10003000002001207047C943016070474368006891
:1000400010EA112007D00122C9B212FA01F11942B7
:100050000CBF0020012070476FEA1121016070473A
:10006000036823F00103036000230360436083609F
:10007000C3600361212343612C4B98421CD02C4B5D
:10008000984220D02B4B984225D02B4B98422AD017
:100090002A4B98422FD02A4B984233D0294B984272
:1000A00037D0294B984204D14FF03D5243F8AC2C45
:1000B0007047264B984203D13D2243F8082C7047E5
:1000C000234B984204D14FF4746243F8202C7047BC
:1000D000204B984204D14FF4741243F8382C7047E7
:1000E0001D4B984204D14FF0746243F8502C704776
:1000F0001A4B984203D11A4A43F8642C7047194BA3
:10010000984203D1184A43F87C2C7047174B984209
:1001100003D1174A43F8942C7047164B984204BFFA
:100120004FF03D5243F8AC2C704700BF10600240C6
:100130002860024040600240586002407060024007
:1001400088600240A0600240B86002401064024033
:1001500028640240406402405864024070640240D7
:100160003D00002088640240400F0020A06402404F
:1001700000003D20B86402400268134B10B51340E4
:10018000CC680A6822434C6922438C692243CC69BB
:1001900022430C6A22434C6A22438C6A22434C6BF2
:1001A00022438C6B22431343036042690C6BCB6A7E
:1001B00022F007022343134343610B6943604B68FA
:1001C00083608B68C36010BD3F801CF00023036018
:1001D00043608360C360036143618361C361036201
:1001E00043628362C362036343638363704703684C
:1001F00011B143F0010301E023F0010303607047F4
:10020000036811B143F4004301E023F400430360A9
:100210007047036811B143F0200301E023F020038D
:100220000360704741607047406880B27047036860
:1002300012B143F4002301E023F4002303600161C1
:100240007047036811B143F4802301E023F4802355
:10025000036070470AB101617047C1607047006870
:10026000C0F3C0407047006800F00100704740696B
:1002700000F0380070470A4A0A4B10B50A4CA042F9
:1002800088BF13468A004CBF5B681B6821F0F021D1
:1002900021F0821119420CBF0020012010BD00BFC7
:1002A00000640240006002400F64024010B5084B39
:1002B000084A094CA04288BF134611F0005F21F0A4
:1002C000F02121F0821114BFD960996010BD00BFE8
:1002D00000600240006402400F6402400B0607D534
:1002E000436912B143F0800301E023F080034361CE
:1002F000802909D001F01E01036812B11943016081
:10030000704723EA010101607047124B124A10B591
:10031000124CA0428CBF14461C4621F0F02323F05F
:10032000C3132BB1026802F01E0202EAD12202E0DE
:10033000426902F0800288004CBF6368236821F0A4
:10034000F02121F08210184002D0101C18BF0120AB
:1003500010BD00BF00600240006402400F64024014
:1003600010B5084B084A094CA04288BF134611F04B
:10037000005F21F0F02121F0821114BFD960996053
:1003800010BD00BF00600240006402400F640240E4
:10039000044B00221A605A609A60DA60024A5A617D
:1003A000704700BF003C0140FFFF7F00837910B51C
:1003B000002B29D01A4B01681C68CA4314401C60EA
:1003C0005C6822405A60027902F1804202F59E3256
:1003D00014682143116002689C68D1430C409C6002
:1003E000DC682140D9604179102906D19968114310
:1003F0009960D9680A43DA6010BD01F1804303F5C2
:100400009E3319680A4308E00379016803F18043C9
:1004100003F59E331A6822EA01021A6010BD00BF7C
:10042000003C014000230C22036003714271837180
:100430007047024B1A6902431A617047003C014041
:10044000034B5B6918420CBF00200120704700BFBE
:10045000003C0140014B5861704700BF003C014027
:10046000054B1A685B69034004D010420CBF0020A2
:100470000120704718467047003C0140014B58610D
:10048000704700BF003C01404FF0204318B943F2D1
:10049000DB021A6003E043F2D20243F820204FF05F
:1004A0002042411C6FF0704342F8213002F5827205
:1004B00042F82030704770B584684568C368C16AE7
:1004C000026825431D4303691D4343691D43836936
:1004D0001D43C3691D43036A1D43436A1D43836A69
:1004E0001D43036B0D431D434FF02043082C43F87D
:1004F000225005D153F8224044F0400443F82240F2
:10050000436B9E691D6835435E6845EA06159E6823
:1005100045EA0625DE6845EA06451E695B6945EA47
:100520000655541C45EA03654FF02043B1F5804F52
:1005300043F8245010D1836B9869196801435868B7
:1005400041EA0011986841EA002118695B6941EAB3
:10055000005141EA036101E06FF07041014B43F843
:10056000221070BD040100A0022242604FF48052AC
:100570004262416B4FF4005210B5826200230F2299
:10058000FF2403608360C360036143618361C361CF
:100590000362C36203630A604A608C60CA600A61D6
:1005A0004A618B61816B0A604A608C60CA600A6133
:1005B0004A618B6110BD4FF0204321B153F82020D8
:1005C00042F0010203E053F82010024A0A4043F8C7
:1005D00020207047FEFF0F0010280CBF064B074B72
:1005E0004FF040024FF0180119605A604FF0FC3292
:1005F0009A60DA60704700BF600000A0800000A031
:1006000030B5836844681C43C36844F008041C4345
:1006100003691C43436944EA4324836944EA43343D
:10062000C36999685A68090441EA02211A68DB68BB
:10063000114341EA0361036A9A685D68120442EA61
:1006400005221D68DB682A4342EA03620368102B17
:100650000CBF034B034B1C609960DA6030BD00BFD8
:10066000600000A0800000A010230360C269002386
:1006700043608360C360036143618361FC23136053
:1006800053609360D360026A136053609360D360D9
:10069000704741B110280CBF074B084B1A6842F055
:1006A00004021A60704710280CBF034A034A044B27
:1006B00011680B4013607047600000A0800000A02C
:1006C000FBFF0F0041B110280CBF084B084B1A6804
:1006D00042F040021A60704710280CBF034A044AD7
:1006E000044B11680B401360704700BF600000A00E
:1006F000800000A0BFFF0F00102802D1024B5869F4
:100700007047024B58697047600000A0800000A04D
:10071000054B18221A6000225A604FF0FC329A6092
:10072000DA601A61704700BFA00000A00268436849
:1007300042F0100242EA4322836842EA4332144BF9
:1007400010B51A60C26891685468090441EA04212E
:100750001468D268214341EA02629A600269916892
:100760005468090441EA04211468D268214341EA2B
:100770000262DA60426991685068090441EA002126
:100780001068D268014341EA02621A6110BD00BFDD
:10079000A00000A0C2680023036043608360FC23C4
:1007A000136053609360D360026913605360936079
:1007B000D3604269136053609360D3607047054B08
:1007C00018B11A6842F0040202E01968024A0A40AD
:1007D0001A607047A00000A0FBFF0F0062B1102854
:1007E00001D10E4B03E0B0F5807F03D10C4B5A686A
:1007F000114311E00B4BFAE7102804D1074B5A685C
:1008000022EA010108E0B0F5807F0CBF044B054BE4
:100810005A686FEA0101114059607047600000A0FA
:10082000800000A0A00000A0102801D1064B04E029
:10083000B0F5807F0CBF054B054B5B680B420CBFCE
:1008400000200120704700BF600000A0800000A0D1
:10085000A00000A0102804D1074B5A6822EA010129
:1008600008E0B0F5807F0CBF044B054B5A686FEA77
:100870000101114059607047600000A0800000A095
:10088000A00000A0102801D1084B04E0B0F5807F43
:100890000CBF074B074B5B6813EA010004D013EA57
:1008A000D1010CBF00200120704700BF600000A0F4
:1008B000800000A0A00000A0102804D1084B5A68B6
:1008C00022EAD10109E0B0F5807F0CBF054B064B51
:1008D0005A684FEAD10122EA01015960704700BF0E
:1008E000600000A0800000A0A00000A008B52C4B74
:1008F000984205D10120014600F048FC012048E063
:10090000284B984205D10220012100F03FFC022033
:100910003FE0254B984205D10420012100F036FC30
:10092000042036E0214B984205D10820012100F037
:100930002DFC08202DE01E4B984205D110200121EE
:1009400000F024FC102024E01A4B984205D120200E
:10095000012100F01BFC20201BE0174B984205D121
:100960004020012100F012FC402012E0134B98427D
:1009700005D18020012100F009FC802009E0104B06
:1009800098420BD14FF48070012100F0FFFB4FF42F
:1009900080700021BDE8084000F0F8BB08BD00BF32
:1009A000000002400004024000080240000C024027
:1009B000001002400014024000180240001C0240D7
:1009C000002002402DE9F0470023D1F800801A46AC
:1009D0004FF0010C03270CFA02F404EA0805A542C3
:1009E0002ED1066817FA03F4E443264006600E7918
:1009F000D0F8009006FA03FA013E4AEA0909012EEE
:100A0000C0F8009014D8866891F80590264086605A
:100A1000866809FA03F949EA06068660466826EA06
:100A2000050545608D7946689540ADB23543456012
:100A3000C5682C40C460CC79C5689C402C43C46018
:100A400001320233102AC6D1BDE8F0874FF6FF739A
:100A500003600023037143718371C371704782B0D7
:100A60004FF480330193019B0B430193019BC361BE
:100A7000C161019BC361C3690193C369019302B062
:100A80007047036919420CBF0020012070470069BC
:100A900080B27047436919420CBF002001207047A3
:100AA000406980B2704701837047418370470AB143
:100AB00001837047418370474161704743694B40F0
:100AC0004361704701F00703C908083130B59B0046
:100AD00050F821500F249C4025EA040440F821409E
:100AE00050F8214012FA03F31C4340F8214030BD76
:100AF00008B5134B984207D14FF40010012100F0C4
:100B000069FB4FF4001014E00E4B984207D14FF4EC
:100B10008000012100F05EFB4FF4800009E00A4BE9
:100B200098420BD14FF40000012100F053FB4FF429
:100B300000000021BDE8084000F04CBB08BD00BF2C
:100B40000054004000580040005C00407FB504465F
:100B5000868868460D4600F06DFA02992C482B688D
:100B600026F03F063604B1FBF0F0360C80B20643A7
:100B7000A680228822F001021204120C2280254A4B
:100B800093420AD85B00B1FBF3F301309BB280B211
:100B90002084032B98BF042321E0EE884BF6FF72DC
:100BA000964205D103225343B1FBF3F39BB206E017
:100BB00019225343B1FBF3F39BB243F480431A056C
:100BC0004FF4967208BF43F0010350434FF47A721A
:100BD00090FBF2F0013080B243F400432084A38301
:100BE00023886989AA889BB243F001032380238864
:100BF00023F4816323F002031B040A431B0C1343F9
:100C00009BB223802A89AB8913439BB223817FBD8A
:100C100040420F00A086010041F2883303600023A8
:100C200083804BF6FF72038143814FF48043C2807F
:100C300083817047038819B19BB243F0010303E03D
:100C400023F001031B041B0C03807047038819B1B8
:100C50009BB243F4807303E023F480731B041B0CEA
:100C600003807047038819B19BB243F4007303E01B
:100C700023F400731B041B0C0380704712B141F076
:100C8000010101E001F0FE0101827047038819B102
:100C90009BB243F4806303E023F480631B041B0CCA
:100CA0000380704783899BB201F0FE0123F0FE03AD
:100CB0000B4383817047838919B19BB243F00103D1
:100CC00003E023F001031B041B0C8381704703889E
:100CD00019B19BB243F0400303E023F040031B042F
:100CE0001B0C03807047038829B16FEA43436FEA06
:100CF00053439BB201E05B045B0C038070470388A5
:100D000019B99BB243F0800303E023F080031B0476
:100D10001B0C03807047B1F5804F838B04D023F404
:100D200080431B041B0C02E09BB243F4804383838B
:100D30007047B1F5006F038803D19BB243F40063A1
:100D400003E023F400631B041B0C03807047B1F520
:100D5000005F038803D19BB243F4005303E023F404
:100D600000531B041B0C03807047038819B19BB20E
:100D700043F0100303E023F010031B041B0C03805B
:100D8000704701827047008AC0B27047038819B16A
:100D90009BB243F4805303E023F480531B041B0CE9
:100DA00003807047B1F5006F038803D19BB243F411
:100DB000006303E023F400631B041B0C03807047F3
:100DC000038819B19BB243F0200303E023F0200312
:100DD0001B041B0C03807047008BC0F30720704777
:100DE000838819B19BB243F4006303E023F40063EA
:100DF0001B041B0C83807047838819B19BB243F49A
:100E0000805303E023F480531B041B0C8380704742
:100E100082B0002301930190019BCB180193019BA9
:100E2000188880B202B0704783889BB20AB1194318
:100E300001E023EA010181807047838A008B9BB225
:100E400043EA0040084020F07F40431A584240EBFC
:100E500003007047838A008B9BB243EA004020F076
:100E60007F40704782B00023009301930B0F0190E5
:100E70000093009B21F07F4113B1019B143302E0EA
:100E8000019B090C18330193019B1B6819420CBF8D
:100E90000020012002B07047C94389B281827047A7
:100EA0008388808A80B208409BB206D001F0E0615E
:100EB00013EA11410CBF002001207047C94389B2D9
:100EC000818270470A4B1A6842F001021A600022C0
:100ED0009A60196821F0847121F480311960054904
:100EE0005960196821F480211960DA60704700BFE9
:100EF0000038024010300024024B00221A70187093
:100F0000704700BF02380240034B1A6822F0F80213
:100F100042EAC0021A60704700380240014B186074
:100F2000704700BF00004742064B002201281A709C
:100F30001A7002D0042804D101E01870704705220D
:100F40001A70704770380240014B1860704700BF3C
:100F5000800E4742014341EA821200995B08013B3F
:100F600042EA016141EA0341014B5960704700BF09
:100F700000380240014B1860704700BF60004742D4
:100F80008001034B40EA0171C3F88410704700BF31
:100F900000380240014B1860704700BF68004742AC
:100FA000014B1860704700BF4C004742034B9A68E2
:100FB00022F0EC6202430A439A6070470038024014
:100FC000034B9A6822F0784202430A439A607047C2
:100FD00000380240034B9A6822F0030202439A60F1
:100FE000704700BF00380240024B986800F00C00C8
:100FF000704700BF00380240034B9A6822F0F002AD
:1010000002439A60704700BF00380240034B9A6861
:1010100022F4E05202439A60704700BF0038024059
:10102000034B9A6822F4604242EAC0029A60704719
:10103000003802401E4B9A6802F00C02042A10B5D8
:1010400003D0082A03D01B4B18E01B4B16E059684D
:101050005A6811F4800F596814BF174B154B02F0F2
:101060003F02B3FBF2F3124A5268C2F30142C1F3EA
:10107000881101324B435200B3FBF2F30C49036079
:101080008B680E4A0468C3F30313D35C34FA03F38A
:1010900043608C68C4F38224145D33FA04F48460E2
:1010A0008968C1F34231525CD340C36010BD00BFB8
:1010B000003802400024F40000127A0034030020BB
:1010C00000F44073B3F5407F084B08D1996820F0D5
:1010D000704221F4F81122F440720A439A601A6FA8
:1010E000000542EA10501867704700BF0038024000
:1010F000014B1860704700BF3C0E4742014B18601F
:10110000704700BF400E4742014B1860704700BF58
:101110005C014742044B1A6B09B1104301E022EA1B
:1011200000001863704700BF00380240044B5A6B40
:1011300009B1104301E022EA00005863704700BF84
:1011400000380240044B9A6B09B1104301E022EAD7
:1011500000009863704700BF00380240044B1A6CCF
:1011600009B1104301E022EA00001864704700BF93
:1011700000380240044B5A6C09B1104301E022EAE6
:1011800000005864704700BF00380240044B1A69E1
:1011900009B1104301E022EA00001861704700BF66
:1011A00000380240044B5A6909B1104301E022EAB9
:1011B00000005861704700BF00380240044B9A6934
:1011C00009B1104301E022EA00009861704700BFB6
:1011D00000380240044B1A6A09B1104301E022EAC8
:1011E00000001862704700BF00380240044B5A6A82
:1011F00009B1104301E022EA00005862704700BFC5
:1012000000380240044B1A6D09B1104301E022EA94
:1012100000001865704700BF00380240044B5A6D4B
:1012200009B1104301E022EA00005865704700BF91
:1012300000380240044B9A6D09B1104301E022EAE4
:1012400000009865704700BF00380240044B1A6EDA
:1012500009B1104301E022EA00001866704700BFA0
:1012600000380240044B5A6E09B1104301E022EAF3
:1012700000005866704700BF00380240044B1A78DF
:1012800009B1104301E022EA00001870704700BF66
:101290000D3802404309012B074A01D1136803E0CE
:1012A000022B0CBF136F536F00F01F0033FA00F0D6
:1012B00000F00100704700BF0038024007B500236E
:1012C00001933120FFF7E6FF019B01330193019B5E
:1012D000B3F5A06F01D00028F3D03120FFF7DAFF7B
:1012E000003018BF01200EBD024B5A6F42F08072D1
:1012F0005A67704700380240034BDB6818420CBF46
:1013000000200120704700BF00380240014B1870D8
:10131000704700BF0E38024008B5154B98420BD1FC
:1013200001214FF48050FFF761FF4FF480500021FE
:10133000BDE80840FFF75ABF0E4B984207D14FF463
:1013400080400121FFF746FF4FF4804009E00A4B3F
:1013500098420BD14FF400400121FFF73BFF4FF4BF
:1013600000400021BDE80840FFF734BF08BD00BFC2
:101370000030014000380040003C00400B880288EB
:1013800010B54C8823438C882343CC8823430C8995
:1013900023434C8923438C892343CC8902F4415253
:1013A000234313439BB20380838B23F400631B040A
:1013B0001B0C83830B8A038210BD838B23F47B6316
:1013C00023F00F031B041B0C8383022303848B680D
:1013D000F0B5858B022BADB238D0294A8E8894683F
:1013E000002E14BF02260126240203D5946824F49B
:1013F00000049460D2F88440D2F884705268DFF818
:1014000084C002F03F02BCFBF2F2C4F388145443E0
:10141000C7F30272B4FBF2F4CA88B2F5007F4FF052
:101420000A0201D1240A02E07601B4FBF6F4624319
:10143000B2FBF3F305330A229BB2B3FBF2F303F0E2
:1014400001021202C3F34F0392B200E000229C1E7D
:10145000A4B2FE2C28BF0022CC8828BF022313434D
:1014600023439BB203840B884A882B4343F40063D5
:1014700013438A8813438A8913439BB28383F0BD45
:101480000038024000127A000023038043808380EA
:10149000C380038143818381C38107230382704713
:1014A00000230222038043808380C3808260838183
:1014B0007047038819B19BB243F0400303E023F067
:1014C00040031B041B0C03807047838B19B19BB234
:1014D00043F4806303E023F480631B041B0C8383C9
:1014E0007047038823F400631B041B0C03800388EC
:1014F0009BB20B4303807047B1F5804F038803D143
:101500009BB243F4804303E023F480431B041B0C91
:10151000038070474FF6FF639942038803D09BB264
:1015200043F4807303E023F480731B041B0C0380DB
:101530007047838819B19BB243F0040303E023F0A2
:1015400004031B041B0C83807047838819B19BB272
:1015500043F0100303E023F010031B041B0C8380F3
:101560007047838B23F47B6323F00F031B041B0C56
:101570008383022303840B88828BB3F5007F10B52D
:1015800092B205D0002B0CBF4FF48073002301E012
:101590004FF480734C8822438C88898942F400621E
:1015A00022430A4392B21343838310BD808980B2E1
:1015B000704781817047038819B19BB243F400538F
:1015C00003E023F400531B041B0C038070470388C3
:1015D0009BB243F4805303807047012902D0008BF3
:1015E00080B27047808A80B27047008A80B27047AC
:1015F00083889BB20AB1194301E023EA010181808B
:101600007047090901238B409BB21AB1828892B2BC
:10161000134303E0828892B222EA03038380704777
:10162000038919420CBF002001207047C94389B2C9
:101630000181704710B584880089012301F00F02F1
:1016400080B213FA02F21040A4B205D009098B400F
:101650001C420CBF0020012010BD01F00F0101232E
:101660008B40DB439BB20381704700BF08B501216B
:101670004FF48040FFF7BAFD4FF480400021BDE8F1
:101680000840FFF7B3BD014B1860704700380140B8
:1016900001F0030289080A4B023130B5920053F879
:1016A00021500F24944025EA040443F8214053F8C4
:1016B000214010FA02F2144343F8214030BD00BF2C
:1016C00000380140014B1860704700BFDC00274222
:1016D000014B1860704700BF00042742024B186A94
:1016E000C0F30020704700BF0038014030B5048CC3
:1016F00024F001042404240C0484058B048CADB272
:10170000A4B225F0F305154324F00A0445EA0315B5
:1017100044F00104ADB20C430583048430BD30B500
:10172000048C24F010042404240C0484048B058C01
:1017300024F44074ADB22405240D25F0A00544EA3C
:10174000022445F0100544EA033445EA0115A4B229
:10175000ADB20483058430BD08B5474B984205D12E
:1017600001200146FFF742FD01203DE0B0F1804F2E
:1017700005D101200146FFF72DFD012076E03F4B0A
:10178000984205D102200121FFF724FD02206DE0DF
:101790003B4B984205D104200121FFF71BFD04209B
:1017A00064E0384B984205D108200121FFF712FD73
:1017B00008205BE0344B984205D110200121FFF74F
:1017C00009FD102052E0314B984205D12020012123
:1017D000FFF700FD202049E02D4B984209D102205F
:1017E0000121FFF703FD02200021BDE80840FFF7BB
:1017F000FDBC284B984207D14FF480300121FFF700
:10180000F5FC4FF48030EFE7234B984207D14FF4BB
:1018100000300121FFF7EAFC4FF40030E4E71F4BF2
:10182000984207D14FF480200121FFF7DFFC4FF4ED
:101830008020D9E71A4B984205D140200121FFF7BB
:10184000C9FC402012E0174B984205D180200121AD
:10185000FFF7C0FC802009E0134B98420BD14FF4F6
:1018600080700121FFF7B6FC4FF480700021BDE8C5
:101870000840FFF7AFBC08BD000001400004004075
:1018800000080040000C0040001000400014004020
:101890000004014000400140004401400048014074
:1018A00000180040001C0040002000401C4A038833
:1018B00090429BB212D002F5806290420ED0B0F1FD
:1018C000804F0BD0A2F58032904207D002F58062A3
:1018D000904203D002F58062904203D14A8823F0FF
:1018E000700313430F4A904208D002F58062904281
:1018F00004D023F440730A899BB2134303804B68DE
:10190000C3620B880385064B984203D003F58063BE
:10191000984201D18B7A038601238382704700BFEE
:1019200000000140001000404FF0FF3343600023EF
:1019300003800381438083727047018582827047F0
:10194000038823F070031B041B0C0B4303807047B8
:1019500041627047C1627047406A7047008D80B233
:101960007047038819B19BB243F0020303E023F0F0
:1019700002031B041B0C03807047038819B19BB240
:1019800043F0040303E023F004031B041B0C038057
:101990007047038819B19BB243F0800303E023F042
:1019A00080031B041B0C03807047038823F008038B
:1019B0001B041B0C038003889BB20B4303807047FE
:1019C000038823F440731B041B0C038003889BB221
:1019D0000B4303807047038819B19BB243F00103A6
:1019E00003E023F001031B041B0C03807047038CEE
:1019F00023F001031B041B0C038470B5038C848843
:101A0000028B0D884E8822F073021204120C2A43B6
:101A10008D8923F002031B0435431B0CADB22B430D
:101A20000E4DA842A4B203D005F58065A8420ED1A0
:101A3000CD894E8A23F008032B438D8823F00403BD
:101A40002B430D8A354324F44074ADB22C4384807B
:101A500002838A684263038470BD00BF00000140B6
:101A6000038C23F010031B041B0C0384038C82885B
:101A700030B5048B0D8824F4E6442404240C23F0B0
:101A8000200344EA05241B048D891B0C43EA05133B
:101A90004D8843EA0513134DA84292B2A4B29BB2FB
:101AA00003D005F58065A84215D1CD8923F08003C8
:101AB0009BB243EA05134FF6BF751D408B8845EA7C
:101AC00003130D8A22F4406242EA85024D8A42EAFB
:101AD00085029BB292B282808A6804838263038407
:101AE00030BD00BF00000140038C23F480731B0451
:101AF0001B0C0384038C828830B5848B0D8824F002
:101B000073042404240C23F400731B042C438D89D8
:101B10001B0C43EA05234D8843EA0523124DA842D6
:101B200092B29BB203D005F58065A84215D1CD894C
:101B300023F400639BB243EA05234FF6FF351D40B3
:101B40008B8845EA03230D8A22F4405242EA0512AB
:101B50004D8A42EA05129BB292B282808A688483DF
:101B6000C263038430BD00BF00000140038C23F436
:101B700080531B041B0C0384038C30B58488828B38
:101B80000D8822F4E6421204120C23F4005342EAB8
:101B900005221B048D891B0C43EA05334D8843EA5B
:101BA00005330B4DA842A4B292B29BB203D005F507
:101BB0008065A84205D10D8A24F4804444EA851446
:101BC000A4B2848082838A680264038430BD00BF2B
:101BD0000000014000230380438083808360838171
:101BE000C38103824382704730B5058C0124ADB2B6
:101BF0008C4025EA040400F11803048409B1082983
